:020000040800F2
:1000000088EA0024ED03000821E90008D1CE0008A9
:10001000F9E50008912F0008D954010800000000FC
:10002000000000000000000000000000C1070108FF
:10003000D94900080000000071EB0008E91B010825
:100040000B0400080B0400080B0400080B04000854
:100050000B0400080B0400080B0400080B04000844
:100060000B0400080B0400080B0400089942000868
:10007000A94200080B040008B94200080B0400085C
:100080000B0400080B0400080B040008414A000898
:10009000614A0008514A0008714A00080B04000830
:1000A0000B0400080B0400080B0400080B040008F4
:1000B000B11D01080B0400080B0400080B04000824
:1000C0000B0400080B0400080B0400080B040008D4
:1000D000390601080B0400080B0400080B04000893
:1000E000E14900080B040008000000000B040008B0
:1000F0000B0400080B0400080B0400080B040008A4
:100100000B0400080B0400080B0400080B04000893
:100110000B040008993001080B0400080B040008C8
:100120000B040008C9420008D94200080B0400086B
:100130000B0400080B0400080B0400080B04000863
:1001400000000000000000000000000000000000AF
:100150000B0400080B0400080B0400080B04000843
:100160000B0400080B0400080B0400080B04000833
:100170000B0400080B0400080B040008000000003A
:100180000B0400080B0400080B0400080B04000813
:100190000B0400080B0400080B0400080B04000803
:1001A0000B0400080B0400080B040008000000000A
:1001B0000B0400080B0400080B0400080B040008E3
:1001C0000B0400080B040008000000000000000001
:1001D00000000000000000000B0400080000000008
:1001E000000000000000000000000000000000000F
:1001F00000000000000000000B0400080B040008D1
:100200000B0400080B040008000000000B040008A9
:100210000B0400080B0400080B0400080B04000882
:100220000B040008000000000B04000800000000A0
:100230000B0400080B040008000000000B04000879
:100240000B0400080B0400080B0400080B04000852
:100250000B0400080B0400080B0400080B04000842
:100260000B0400080B0400080B0400080B04000832
:100270000B0400080B0400080B0400080000000039
:100280000B0400080B0400080B0400080B04000812
:10029000000000000B0400080B0400080000000030
:1002A000000000000B0400080B0400080B04000809
:1002B000C95401080B0400080B040008814A000817
:1002C000914A00080B0400080B04000800F002F833
:1002D00000F063F80AA090E8000C82448344AAF17D
:1002E0000107DA4501D100F058F8AFF2090EBAE87B
:1002F0000F0013F0010F18BFFB1A43F0010318475A
:10030000A4A80100C4A801000A444FF0000C10F892
:10031000013B13F0070408BF10F8014B1D1108BF83
:1003200010F8015B641E05D010F8016B641E01F823
:10033000016BF9D113F0080F1EBF10F8014BAD1C73
:100340000C1B09D16D1E58BF01F801CBFAD505E091
:1003500014F8016B01F8016B6D1EF9D59142D6D3EB
:10036000704700000023002400250026103A28BF13
:1003700078C1FBD8520728BF30C148BF0B60704717
:10038000732900F07282002070471FB519F083FFB7
:1003900000F055F91FBD10B510BD00F073FA1146FD
:1003A000FFF7F3FF15F0FCF800F091FA03B4FFF744
:1003B000F2FF03BC00F094FA0B49D1F800C04A6880
:1003C0005CF8043B1068184442F8040B8C4528BFC5
:1003D000A1F1DC0C8A4228BFA1F1DC02C1F800C007
:1003E0004A6020F000407047340600240A488047E5
:1003F0000A4880470A480047FEE7FEE7FEE7FEE7B7
:10040000FEE7FEE7FEE7FEE7FEE7FEE705480649F2
:10041000064A074B70470000114A0008D91C010822
:10042000CD02000888CA002488EA002488DA002463
:1004300088DA002453EA020C00F069802DE9F04BC1
:100440004FF00006002B1FBFB3FA83F503FA05F443
:1004500024FA05F65E4012BF1643B2FA82F502FA9C
:1004600005F4C5F120051EBF22FA05FC44EA0C0480
:10047000203556EA044C4FEA144418BF641C4FF070
:1004800000084FF00009904271EB030C39D30029AA
:1004900019BFB1FA81F701FA07F6B0FA80F700FA4E
:1004A00007F6C7F120071EBF20FA07FC46EA0C0634
:1004B0002037B6FBF4FCA7EB0507103F07F01F0B36
:1004C000CBF120062CFA06F60CFA0BFB44BFB34620
:1004D0000026202FA4BF5E464FF0000B5BEA060CFF
:1004E00008BF4FF0010B19EB0B0948EB0608ABFBFB
:1004F000027C06FB02CC0BFB03CCC01B71EB0C0196
:10050000C1E70B46024641464846BDE8F08B13B5AD
:10051000084318BF4FF0FF300146AFF30080BDE83D
:100520001C4070470FB41CB50C0007AA009001D006
:100530002044401E074B7B4469460190069800F01A
:1005400062F9002C03D06946002000F06FF91CBC52
:100550005DF814FBFD0200002DE9F0410E46044653
:10056000002020622046E168884730B3252805D066
:10057000D4E901219047206A401CF2E7E168204657
:1005800000278847050018D0A5F14100192802D896
:1005900020354FF400673246294620462760FFF792
:1005A000EFFE40B1012804D0F61D26F007060836FC
:1005B000D8E7361DD6E72846DAE7206ABDE8F0819D
:1005C00070B50C460546012A05D02878800600D56E
:1005D000EA69002302E0012305E05B1C934202D29A
:1005E000E05C0028F9D1A869E618C01AA861286A59
:1005F000184428622846AFF3008004E0D5E90121C1
:1006000014F8010B9047B442F8D32846AFF30080AA
:1006100070BD00000B4910B5A1F17C020A4CC2E983
:100620003712372106E000EB104342F82130074B28
:1006300000FB03400B1EA1F10101F4DC10BD012001
:10064000E8E70000D4050024E119D666CD0D0100CD
:10065000032A40F2308010F0030C00F0158011F8EE
:10066000013BBCF1020F624498BF11F801CB00F8C6
:10067000013B38BF11F8013BA2F1040298BF00F81A
:1006800001CB38BF00F8013B11F0030300F02580D7
:10069000083AC0F0088051F8043B083A51F804CBFE
:1006A000A0E80810F5E7121D5CBF51F8043B40F8C4
:1006B000043BAFF30080D20724BF11F8013B11F8CF
:1006C00001CB48BF11F8012B24BF00F8013B00F813
:1006D00001CB48BF00F8012B704710B5203AC0F09D
:1006E0000B80B1E81850A0E81850B1E81850A0E805
:1006F0001850203ABFF4F5AF5FEA027C24BFB1E89E
:100700001850A0E8185044BF18C918C0BDE81040E0
:100710005FEA827C24BF51F8043B40F8043B08BFE9
:100720007047D20728BF31F8023B48BF11F8012BB0
:1007300028BF20F8023B48BF00F8012B704702F0A9
:10074000FF0343EA032242EA024200F024B84FF0DA
:1007500000020429C0F0128010F0030C00F01B808E
:10076000CCF1040CBCF1020F18BF00F8012BA8BF9C
:1007700020F8022BA1EB0C0100F00DB85FEAC17C60
:1007800024BF00F8012B00F8012B48BF00F8012B13
:1007900070474FF0000200B5134694469646203944
:1007A00022BFA0E80C50A0E80C50B1F12001BFF42A
:1007B000F7AF090728BFA0E80C5048BF0CC05DF890
:1007C00004EB890028BF40F8042B08BF704748BFDE
:1007D00020F8022B11F0804F18BF00F8012B704752
:1007E00070477047704710B500F044F8006810BDBE
:1007F00010B5044600F03EF8046010BD01694A1CC3
:1008000002610878704700B58FB0CDE90131002151
:10081000059105497944CDE9031011466846FFF773
:100820009BFE0FB000BD0000E5FFFFFF0A6802F865
:10083000010B0A607047D1E900239A4202D2531C8F
:100840000B601070704710B5436913B1AFF30080AF
:1008500001E0FFF7B5FE012010BD127800F1240180
:100860000A7000224A700122EDE711684FF0FF3252
:10087000E9E70000004870473C0600240048704744
:100880003C0600247546FFF7F9FFAE4605006946B1
:10089000534620F00700854618B020B5FFF7B6FD97
:1008A000BDE820404FF000064FF000074FF0000871
:1008B0004FF0000BAC46ACE8C009ACE8C009ACE8AE
:1008C000C009ACE8C00921F007018D46704710B59A
:1008D0000446AFF300802046BDE81040FFF766BD38
:1008E00001491820ABBEFEE7260002007047000059
:1008F000B0B52DED028B044600284FF0FF005FD00D
:100900000D4600295CD095ED020A95ED032A20EEF4
:10091000001A95ED013A20EE020A95ED002AB7EE95
:10092000008A03EE031A02EE030A31EE011A30EEDA
:10093000000A78EE410A18F09BFE95ED002A95ED2D
:10094000014A95ED023A95ED035A22EE031A84ED21
:10095000010A05EE441A31EE011AB0EEC16AB4EE96
:10096000486AF1EE10FA0FDAB0EE410A18F018FCFE
:1009700095ED002A95ED014A95ED023A95ED035A61
:1009800084ED020A09E000BF11EE100A40F6DB71A7
:10099000C3F6C97161F31E00A06023EE030A24EEC2
:1009A000031A05EE050A02EE051A30EE002A31EEB2
:1009B000010A78EE420A18F05BFE002084ED000A7E
:1009C00040B2BDEC028BB0BDB0B500286ED0B7EE22
:1009D000001A04460D46002981EE000A80ED040A43
:1009E0004FF07E5020604FF00000C4E90100E0604D
:1009F00059D095ED010A95ED001AB7EEC00AB7EE91
:100A0000C11A18F051FD95ED001AB5EE401AF1EE3D
:100A100010FA0DD195ED011AB5EE401AF1EE10FA6B
:100A200006D195ED021AB5EE401AF1EE10FA41D05A
:100A3000B7EEC00B9FED351AB4EE410AF1EE10FA95
:100A40004CDCB5EE400AF1EE10FA47DB9FED302AA0
:100A5000B4EE420AF1EE10FA2CDCB4EE410AF1EEEB
:100A600010FA27DB9FED2B1AB4EE410AF1EE10FAD3
:100A700004DCB4EE420AF1EE10FA43DA40F2C5604B
:100A800044F62D21C3F64D70C3F60D4120604AF2A5
:100A90005640616044F2AD71CBF63930C3F619713E
:100AA000C4E90201002040B2B0BD00BFFF2040B247
:100AB000B0BD00BF40F2C56044F62D21C3F64D70B5
:100AC000C3F60D4120604AF25640616044F2AD71B8
:100AD000CBF63930C3F6197112E000BF45F66E103F
:100AE00045F20C31C3F67F70C3F6B011206048F6B2
:100AF000AB00616049F28551CBF6BB30C3F697512C
:100B0000C4E90201002040B2B0BD00BFDB0FC9BF85
:100B1000DB0F49C00000B4C200218160C0E90011B0
:100B20007047000000000000B0B52DED108B8EB0B6
:100B3000044600284FF0FF0003D0002918BF002A08
:100B400004D140B20EB0BDEC108BB0BD40F27005C8
:100B50004EF69E70C2F20045002BC3F62750286067
:100B600000F0D28193ED009A93ED01AAB5EE409A80
:100B700093ED028AF1EE10FA04BFB5EE40AAF1EE51
:100B800010FA00F0BB8192ED000A94ED011A92ED8B
:100B9000016A92ED027A94ED004A21EE405A60EE2D
:100BA000040A94ED022A66EE041A94ED033A67EE05
:100BB000042AD1ED004A06EE425AF5EE404A47EECD
:100BC000020A47EE411A46EE012A07EE435A46EE64
:100BD000430AB6EE006A40EE031A40EE422A91ED57
:100BE000010AF1EE10FA65EE063A91ED025A60EE56
:100BF000860A21EE867A22EE866A04BFB5EE400AA6
:100C0000F1EE10FA00F088818DED080A20EE000A5E
:100C10008DED0D6A8DED0C7A04EEA40ACDED0B3A44
:100C2000CDED0A0A8DED095A05EE050ACDED074A0C
:100C30000CF052F92AEE0A1A8DED060A09EE091A8D
:100C400008EE081AB0EE410A0CF046F994ED00CA1D
:100C500029EE00FA7CEE0CBA94ED03BA6AEE008A33
:100C600094ED013A28EE00EAD4ED029A2FEE2B0A19
:100C70002CEE0C8A8DED010A68EEABAA20EE0B0A71
:100C80002FEE081A2EEE2B2A08EE880A73EE03EADE
:100C90000AEECB1A03EE420A6FEE2ECA02EE291AB2
:100CA00023EE034A09EEAC0A8DED034A28EEAE2A84
:100CB0000FEE041A08EEC40A69EEA9FA39EEA99AF1
:100CC00009EE821A08EEAF0A2EEE2E2A2EEE094AFF
:100CD0002BEE0BDA02EE0B1A0BEE040A2CEE03AA33
:100CE0000FEE6F1A08EECD0A63EE0BDA0FEE4D1A17
:100CF00020EE000A01EE010A23EE291A8DED021AF8
:100D00003BEE0B1A8DED051A2CEE291A8DED041A07
:100D10000CF0E2F894ED011A94ED022A2AEE813AE1
:100D20009DED014ADDED031A28EE897A3DEEAD5ABC
:100D3000DDED070A04EE423A94ED034A3AEE0A6A00
:100D4000F6EE004A0BEEE95ADDED047A0EEE083AB3
:100D5000F0EE616A09EE0B6ADDED02AA7DEEE72A8C
:100D60009DED058A0CEE843A09EE8BAA4CEE4BAA57
:100D70000EEE613A07EE043A9DED067A00EEC75A90
:100D8000DDED080A00EEC76AF0EE473A0EEE6F3A64
:100D9000B7EE007A71EEA10A74EEEF1A0EEE0D3A7C
:100DA00087EE000A37EE607A7FEEAF0A28EE05BACA
:100DB00028EE068A37EE607A71EECD0A62EE831A6B
:100DC000DDED092A02EEE37A6AEE032A40EE201AEC
:100DD000F1EE000A0BEEC58A40EE2A2A61EE203AB7
:100DE00062EE200A0BEE86BA2EEE86AA00EEC78AC5
:100DF00074EEE60AF8EE004A2EEE85CA07EE63BAF4
:100E000070EEEF0A09EE45AA09EE06CA31EECF5A96
:100E100032EEE86A62EE031A61EE032A60EE043AEB
:100E200037EEAD7A60EE830A01EEC5AA72EEE35AA0
:100E300060EE244A40EE070A94ED007A05EE86AA99
:100E400044EE842A24EE034A60EE025A67EE036AF7
:100E500033EE033A20EE077A75EEA67A52EE246A54
:100E600041EE433A04EE05BA71EEC71A02EE437A38
:100E700030EECE2A20EE011A07EE86BA06EE858AFB
:100E800031EE040A03EE82BA02EE85CA00EE068A4B
:100E900005EE82AA01EE86CA07EE028A2BEE0B0A45
:100EA00001EE02CA0AEE0A0A08EE080A0CEE0C0A63
:100EB0000CF012F820EE0A1ADDED0A0A20EE0B2AD9
:100EC000DDED0B3A20EE083A9DED0C7A20EE0C0A8F
:100ED0009DED0D6A95ED004A44EE413A94ED011AFC
:100EE00044EE420A94ED022A04EE437A94ED033A6A
:100EF00004EE406A94ED004A14E000BFB5EE408A6B
:100F0000F1EE10FA7FF43FAE20460EB0BDEC108B30
:100F1000BDE8B04000F040B8B5EE405AF1EE10FA2E
:100F20007FF472AE94ED045A00EE851A03EE854A02
:100F300007EE052A06EE053A84ED011A84ED004A13
:100F400021EE010A84ED022A84ED033A04EE040A3C
:100F500002EE020A03EE030A0BF0BEFF94ED001A44
:100F600094ED012A94ED023A94ED034A20EE011A21
:100F7000002020EE022A84ED001A20EE031A84EDF0
:100F8000012A20EE040A84ED021A84ED030A40B21D
:100F90000EB0BDEC108BB0BDB0B52DED108B04467E
:100FA00000284FF0FF0003D0002918BF002A03D10A
:100FB00040B2BDEC108BB0BD40F2700542F602307D
:100FC000C2F20045C3F6075094ED011A92ED016A92
:100FD000286092ED027A92ED000A94ED003A21EE3B
:100FE000405A94ED022A60EE030A94ED034A66EE3D
:100FF000031A91ED00EA67EE032AB5EE40EA06EE29
:10100000425A91ED01DA47EE020A91ED02CA47EE2B
:10101000411A46EE012A07EE445A46EE440AB6EE5D
:10102000006A40EE041A40EE422AF1EE10FA04BFC4
:10103000B5EE40DAF1EE10FA25EE06AA20EE86BAF9
:1010400021EE869A22EE868A00F090802DEE0D0A1F
:101050000EEE0E0A0CEE0C0A0BF03EFFB1EE001A7B
:1010600094ED013A94ED034A94ED007A24EE046A7B
:10107000D4ED023A23EE015A67EE071A2EEE002A4B
:1010800074EE040A65EE062A61EE811A77EE074ACD
:1010900042EE602A61EEA35A63EE816A43EE212A92
:1010A0006DEE001A42EE245A2CEE000A41EEE42ABC
:1010B00046EE865A33EEA36A27EE017A41EEE05AF5
:1010C000F2EE000A22EE06DA32EEC5CA63EEA32A79
:1010D00063EE204A63EE037A07EE22DA63EEA00A9B
:1010E00004EEA7CA07EE27DA35EEE6EA04EEA2CA56
:1010F00027EE817A07EEA0EA33EE033A27EE04FAF0
:1011000000EE05CA00EEA2EA02EE43FA22EE811AD0
:1011100001EEC3DA00EE26EA04EE01FA2CEE0C0A28
:1011200001EEC6FA0DEE0D0A0EEE0E0A0FEE0F0AD4
:101130000BF0D2FE20EE0D1A95ED004A20EE0C2A9F
:1011400020EE0E3A20EE0F0A04EE41AA94ED011AA9
:1011500004EE42BA94ED022A04EE439A94ED003A6A
:1011600004EE408A94ED034A06E000BFB5EE40CAA3
:10117000F1EE10FA7FF46AAF94ED045A0BEE051A03
:101180000AEE053A09EE052A08EE054A84ED011A31
:1011900084ED003A21EE010A84ED022A84ED034A2F
:1011A00003EE030A02EE020A04EE040A0BF094FEB8
:1011B00094ED001A94ED012A94ED023A94ED034A5D
:1011C00020EE011A002020EE022A84ED001A20EE03
:1011D000031A84ED012A20EE040A84ED021A84ED3C
:1011E000030A40B2BDEC108BB0BD0000000000004F
:1011F000B1EE601A80FE602AB4EE401AF1EE10FAE9
:1012000031FE020A70470000F0B110B5044600F04C
:10121000E3FB207861680A2200F0DAFC207861683C
:1012200001310A2200F0D4FC2078616802310A22E0
:1012300000F0CEFC20780A22A16800F0C9FC002052
:10124000BDE8104040B27047FE2040B27047000039
:1012500030B1027080ED010A0181002040B2704778
:10126000FE2040B27047000070B588B000284FF0F3
:10127000FE0666D00C46002963D00546007801AA18
:101280000023696800F04CFB10B1FF2640E000BF6E
:101290009DF812009DF814209DF813109DF815304C
:1012A0009DF817609FED2E2A090341EA00510006C0
:1012B0009DF8160041EA021103F00F024FEA0040C8
:1012C00040EA02609DF8182040EA06204FF0000630
:1012D00041EA1311104448BF01F170411A0748BF99
:1012E00000F1704000EE101A9DF8111001EE100A86
:1012F000601C2170B8EEC00AB8EEC11A80EE020A76
:1013000081EE021A10EE102A11EE101A02604160EE
:1013100028786968013101AA002300F001FB40B977
:101320000026DDF81100DDF81510C4F81500C4F82A
:10133000111028786968023101AA002300F0F0FA40
:1013400010B170B208B070BD0026DDF81100DDF8F4
:101350001510C4F80D00C4F8091070B208B070BDC3
:101360008096184B00000000002818BF002901D10A
:10137000704700BF80B584B008228DF804208268D1
:1013800000924A68CDF805200A8900780978ADF8FE
:1013900009208DF80B1000218DF80C10694601F022
:1013A000DFF804B0BDE88040704700000000000096
:1013B00040F2E8700821C2F20040406814F0D0BB4F
:1013C00010B50120002101F07FFA40F2E87492206C
:1013D000C2F200440122002304F8010F002021463C
:1013E00001F066FBE11D00201322012301F02CFB1C
:1013F000002010BD00000000022001214FF0FF324C
:1014000014F0F2BB000000009FED010A704700BF1E
:101410000000C8430000000040F2E8701021C2F252
:101420000040406814F09CBB10B50520002101F07D
:101430004BFA40F2E8748220C2F2004401220023F9
:1014400004F8010F0020214601F032FB04F10E01E7
:1014500000200622012301F0F7FA002010BD000051
:10146000042001214FF0FF3214F0BEBB0000000049
:101470002DE9F04100284FF0FE0700F08F810E4665
:10148000002900F08B8140F2E8780546C2F200485E
:1014900098F8000020B1FD2778B2BDE8F08100BFC8
:1014A00014F056FC0028C8F8040000F07F81444680
:1014B0004BF27E60EE6224F8010F012001F01CFB6C
:1014C0000120002101F000FA002002220023214621
:1014D00001F0EEFA0120012101F0F6F94BF214605F
:1014E0002080012001F008FB0520002101F0ECF92B
:1014F000002002220023214601F0DAFA0520012112
:1015000001F0E2F91E2001F0F7FA012001F0F4FAEF
:101510000120002101F0D8F99E2020700020012236
:101520000023214601F0C4FA0020022200232146B4
:1015300001F08AFA0120012101F0C6F9012001F031
:10154000DBFA0120002101F0BFF900200122002375
:1015500021468026267001F0ABFA002002220023EB
:10156000214601F071FA0120012101F0ADF9607806
:101570001E2840F017810120012501F0BDFA052049
:10158000002101F0A1F9444600200122002304F8C3
:10159000016F214601F08CFA00200222002321462F
:1015A00001F052FA0520012101F08EF920780F2870
:1015B00040F0F880062001F0EFF8072001F0ECF889
:1015C00041F6C1020020C0F600020121002701F00F
:1015D0005FFA41F2B1310620C0F6000101F01CF9BA
:1015E00041F219410720C0F6000101F015F9444607
:1015F0004AF6402024F8010F012001F07DFA012075
:10160000002101F061F9002002220023214601F0AF
:101610004FFA0120012101F057F940F241102080DA
:10162000012001F069FA0120002101F04DF90020AC
:1016300002220023214601F03BFA0120012101F0A2
:1016400043F940F653002080012001F055FA0120B3
:10165000002101F039F9002002220023214601F087
:1016600027FA0120012101F02FF94FF48B6020802F
:10167000012001F041FA0120002101F025F90020AC
:1016800002220023214601F013FA0120012101F07A
:101690001BF940F27D402080012001F02DFA01204D
:1016A000002101F011F9002002220023214601F05F
:1016B000FFF90120012101F007F9322001F01CFAA5
:1016C00040F20F102080012001F016FA05200021C1
:1016D00001F0FAF8002002220023214601F0E8F987
:1016E0000520012101F0F0F84FF444702080012022
:1016F00001F002FA0520002101F0E6F800200222A4
:101700000023214601F0D4F90520012101F0DCF885
:1017100016202080012001F0EFF90520002101F0C2
:10172000D3F8002002220023214601F0C1F9052050
:10173000012101F0C9F84FF48C702080012001F0E4
:10174000DBF90520002101F0BFF800200222002370
:10175000214601F0ADF90520012101F0B5F848F26C
:1017600015002080012001F0C7F90520002101F0BB
:10177000ABF8002002220023214601F099F9052050
:10178000012101F0A1F80A2001F0B6F9062088F83D
:10179000005001F015F8072001F012F878B2BDE80A
:1017A000F08100BFFC2778B2BDE8F081FE2778B257
:1017B000BDE8F0810000000000283FD040F2E87151
:1017C0009FED203AC2F20041B1F90920B1F90DC0F4
:1017D000B1F90B3000EE102A02EE10CA01EE103AF9
:1017E0004FF60003CFF6FF73B8EEC00AB8EEC11A89
:1017F000B8EEC22A80EE030A81EE031A80ED040AD5
:1018000082EE030A80ED051A80ED060AB4EE001A96
:101810004A7EB3EE072A897ED20042EA51120021A5
:10182000B1EB922F18BF1A4300EE102AB8EEC00A8F
:1018300000EE012A80ED0A2A48B27047FE2148B224
:10184000704700BF00A0AA4590B340F2E8719FED39
:101850001A3AC2F200419FED194AB1F90F20B1F9CD
:101860001130B1F9131000EE102A01EE103A02EE19
:10187000101AC16AB8EEC00A91ED015AB8EEC11A49
:10188000B8EEC22A80EE030A81EE031A82EE032A22
:1018900091ED003A10EE043A91ED020A11EE045A6D
:1018A00012EE040A80ED073A80ED085A80ED090A2D
:1018B0006FF00100704700BF6F12034235FA8E3C93
:1018C00010B5012000F090FF40F2E874C2F200442D
:1018D00038B90120012100F0F7FF6068022114F0FF
:1018E0003FF9052000F080FF002818BF10BD05203B
:1018F000012100F0E9FF60680421BDE8104014F008
:101900002FB9000000000000182001214FF0FF3225
:1019100014F06AB9000000007047000000000000E9
:101920002DE9F04140F27874C2F2004427786FB19B
:1019300015467AB10E460746A0686421984614F011
:1019400033F858B1FB2040B2BDE8F081FD2040B231
:10195000BDE8F081FE2040B2BDE8F081606800E0A3
:10196000006978B30178B94202D14168B14217D019
:10197000006938B30178B94202D14168B1420FD051
:101980000069F8B10178B94202D14168B14207D08B
:101990000069B8B10178B942E2D14168B142DFD102
:1019A0008668A06814F06CF87EB1002230462946A3
:1019B000434613F0FDFE002818BF4FF0FF3040B241
:1019C000BDE8F081A06814F05BF8FC2040B2BDE8EF
:1019D000F0810000000000002DE9F04F89B040F2D6
:1019E0007877C2F20047387820B1FD2040B209B0C4
:1019F000BDE8F08F07F110006021FEF7CAFE43F248
:101A0000281041F29001C2F2004041F294020024F9
:101A1000C0F88045C0F88445C0F8084BC0F80C4BAE
:101A20004450845041F61910C0F60000F8600020C0
:101A300013F0E6FF0028B86000F0C48041F62005EE
:101A400001AEC2F2004541F21009284631464FF07E
:101A5000010A87F800A0CDE901444FF0020BC0F263
:101A60000209CDE903BACDE90544079405F060FB0E
:101A700028463146CDF808A04FF08048CDF80480C4
:101A8000CDE903BACDE90544079405F051FB0221E5
:101A9000022200232846009405F092FBA9F10F01D1
:101AA0000022284605F080FA387842F28951C0F6C3
:101AB000000128B141F6B9403961C0F60000F86173
:101AC00041F62000C2F2004006F0C2F941F6C0051E
:101AD00001AEC2F20045314628460024CDE901445A
:101AE000CDE903BBCDE90544079405F021FB01A82E
:101AF0003146CDE904B480E8000D2846CDE906441E
:101B000005F016FB0121012200232846009405F070
:101B100057FB00222846494605F046FA387842F23B
:101B2000390AC0F6000A30B142F28950C7F844A021
:101B3000C0F60000386341F6C000C2F2004006F073
:101B400087F941F660150DF10408C2F200454146DF
:101B500028460226CDE90144CDE90366CDE90544D6
:101B6000079405F0E5FA012002904FF080400190C3
:101B700028464146CDE90366CDE90544079405F0C2
:101B8000D7FA0221012200232846009405F018FB11
:101B900000222846494605F007FA387830B142F26B
:101BA0008950C7F864A0C0F60000386541F660109F
:101BB000C2F2004006F04CF9002040B209B0BDE886
:101BC000F08F00BFFF2040B209B0BDE8F08F0000E9
:101BD0002DE9F04140F27878C2F2004898F80030E0
:101BE00083B114460D460646002A08BF0A24D8F8D9
:101BF0000800642113F0D8FE40B1FB2040B2BDE8DC
:101C0000F08100BFFD2040B2BDE8F081D8F80400AB
:101C100001E000BF0069F8B10178B14202D141682A
:101C2000A94240D00069B8B10178B14202D14168FF
:101C3000A94238D0006978B10178B14202D1416837
:101C4000A94230D0006938B10178B142E2D141688F
:101C5000A942DFD127E000BF142000F04DFEB8B14B
:101C600007461C210022204613F0EAFDB860B8B1F7
:101C7000D8F804003861D8F808003E707D603C73E5
:101C8000C8F8047013F0FCFE002040B2BDE8F081FB
:101C9000D8F8080013F0F4FEFE2040B2BDE8F08151
:101CA000384600F075FDD8F8080013F0E9FEFF2073
:101CB00040B2BDE8F08100002DE9F04F93B06846D6
:101CC000402100F10D0941F62000C2F2004005F06C
:101CD000BFFA40F278780028C2F2004800F0848011
:101CE00041F620050DF1240AC2F200450DF11C0B4E
:101CF00006E000BF4021284605F0AAFA002873D06C
:101D00004021284652465B4605F0AEFA00286BD1CA
:101D10000A986FF0604100284FF0020608BF40F2B9
:101D2000FF71099AB0F1804F01EA020400F14041CD
:101D3000B1FA81F00B9B08BF0326D8F80C20B3F151
:101D4000005F18BF4609204612B120463146904731
:101D5000D8F8041001E000BF09690029CAD00A7848
:101D600012B94A68824218D009690029C2D00A789B
:101D700012B94A68824210D009690029BAD00A789B
:101D800012B94A68824208D009690029B2D00A789B
:101D9000002AE1D14A688242DED18F68002FA9D0A3
:101DA0000C994AF6382201F00F01C0F601028DF8B5
:101DB0000060525C09390194072902904FF000003D
:101DC00038BF0822C9F8040059468DF80C20D2B259
:101DD000C9F800004846FEF73BFC002200233846C5
:101DE000694613F079FD85E741F6C0004021C2F253
:101DF000004005F02DFA002800F0888041F6C0056B
:101E00000DF1240AC2F200450DF11C0B06E000BFE3
:101E10004021284605F01CFA002877D040212846AA
:101E200052465B4605F020FA00286FD10A986FF001
:101E3000604100284FF0020608BF40F2FF71099A86
:101E4000B0F1804F01EA020400F14041B1FA81F0A3
:101E50000B9B08BF0326D8F80C20B3F1005F18BF16
:101E60004609204612B1204631469047D8F8041062
:101E700001E000BF09690029CAD00A78012A02D10D
:101E80004A6882421AD009690029C1D00A78012A19
:101E900002D14A68824211D009690029B8D00A7873
:101EA000012A02D14A68824208D009690029AFD0CC
:101EB0000A78012ADED14A688242DBD18F68002F7E
:101EC000A6D00C994AF6382201F00F01C0F60102A3
:101ED0008DF80060525C09390194072902904FF097
:101EE000000038BF0822C9F8040059468DF80C20BC
:101EF000D2B2C9F800004846FEF7AAFB0022002330
:101F00003846694613F0E8FC82E700BF41F66010EE
:101F10004021C2F2004005F09BF9002800F08880C3
:101F200041F660150DF1240AC2F200450DF11C0BBB
:101F300006E000BF4021284605F08AF9002877D046
:101F40004021284652465B4605F08EF900286FD1A5
:101F50000A986FF0604100284FF0020608BF40F277
:101F6000FF71099AB0F1804F01EA020400F140418B
:101F7000B1FA81F00B9B08BF0326D8F80C20B3F10F
:101F8000005F18BF4609204612B1204631469047EF
:101F9000D8F8041001E000BF09690029CAD00A7806
:101FA000022A02D14A6882421AD009690029C1D0A6
:101FB0000A78022A02D14A68824211D009690029AE
:101FC000B8D00A78022A02D14A68824208D0096948
:101FD0000029AFD00A78022ADED14A688242DBD1DA
:101FE0008F68002FA6D00C994AF6382201F00F0115
:101FF000C0F601028DF80060525C0939019407298E
:1020000002904FF0000038BF0822C9F8040059467A
:102010008DF80C20D2B2C9F800004846FEF718FB34
:10202000002200233846694613F056FC82E700BFC1
:1020300013B0BDE8F08F00002DE9F04F93B0684673
:10204000412100F10D0941F62000C2F2004005F0E7
:10205000FFF840F278780028C2F2004800F084804F
:1020600041F620050DF1240AC2F200450DF11C0BCA
:1020700006E000BF4121284605F0EAF8002873D0A9
:102080004121284652465B4605F0EEF800286BD108
:102090000A986FF0604100284FF0020608BF40F236
:1020A000FF71099AB0F1804F01EA020400F140414A
:1020B000B1FA81F00B9B08BF0326D8F80C20B3F1CE
:1020C000005F18BF4609204612B1204631469047AE
:1020D000D8F8041001E000BF09690029CAD00A78C5
:1020E00012B94A68824218D009690029C2D00A7818
:1020F00012B94A68824210D009690029BAD00A7818
:1021000012B94A68824208D009690029B2D00A7817
:10211000002AE1D14A688242DED18F68002FA9D01F
:102120000C994AF6382201F00F01C0F601028DF831
:102130000060525C09390194072902904FF00000B9
:1021400038BF0822C9F8040059468DF80C20D2B2D5
:10215000C9F800004846FEF77BFA00220023384603
:10216000694613F0B9FB85E741F6C0004121C2F290
:10217000004005F06DF8002800F0888041F6C005A9
:102180000DF1240AC2F200450DF11C0B06E000BF60
:102190004121284605F05CF8002877D041212846E7
:1021A00052465B4605F060F800286FD10A986FF040
:1021B000604100284FF0020608BF40F2FF71099A03
:1021C000B0F1804F01EA020400F14041B1FA81F020
:1021D0000B9B08BF0326D8F80C20B3F1005F18BF93
:1021E0004609204612B1204631469047D8F80410DF
:1021F00001E000BF09690029CAD00A78012A02D18A
:102200004A6882421AD009690029C1D00A78012A95
:1022100002D14A68824211D009690029B8D00A78EF
:10222000012A02D14A68824208D009690029AFD048
:102230000A78012ADED14A688242DBD18F68002FFA
:10224000A6D00C994AF6382201F00F01C0F601021F
:102250008DF80060525C09390194072902904FF013
:10226000000038BF0822C9F8040059468DF80C2038
:10227000D2B2C9F800004846FEF7EAF9002200236E
:102280003846694613F028FB82E700BF41F660102C
:102290004121C2F2004004F0DBFF002800F08880FA
:1022A00041F660150DF1240AC2F200450DF11C0B38
:1022B00006E000BF4121284604F0CAFF002877D07D
:1022C0004121284652465B4604F0CEFF00286FD1DC
:1022D0000A986FF0604100284FF0020608BF40F2F4
:1022E000FF71099AB0F1804F01EA020400F1404108
:1022F000B1FA81F00B9B08BF0326D8F80C20B3F18C
:10230000005F18BF4609204612B12046314690476B
:10231000D8F8041001E000BF09690029CAD00A7882
:10232000022A02D14A6882421AD009690029C1D022
:102330000A78022A02D14A68824211D0096900292A
:10234000B8D00A78022A02D14A68824208D00969C4
:102350000029AFD00A78022ADED14A688242DBD156
:102360008F68002FA6D00C994AF6382201F00F0191
:10237000C0F601028DF80060525C0939019407290A
:1023800002904FF0000038BF0822C9F804005946F7
:102390008DF80C20D2B2C9F800004846FEF758F973
:1023A000002200233846694613F096FA82E700BF00
:1023B00013B0BDE8F08F00002DE9F0478CB040F27B
:1023C0007877C2F200473F7847B1044602280BD91C
:1023D000FF2250B20CB0BDE8F08700BFFD2250B222
:1023E0000CB0BDE8F08700BF01F0FE001D461746A7
:1023F0000E46022806D02DB9FE2250B20CB0BDE820
:10240000F08700BFDDF850A0BAF1080FE0D80DF159
:1024100004082C214046FEF7BCF9032ED8D860B240
:102420004AF2EC32C0F6010252F82090DFE806F0E2
:1024300002060A100197002100200EE001970020FB
:1024400009E000BF01974FF00050002105E000BFF8
:102450004FF0005001974FF080410390D9F80800E9
:102460000291B0F5407F07D0B0F5807F0AD14FF4DC
:102470000010002108E000BF4FF400104FF480115D
:1024800002E000BF0021002008F12407CDF810A0D1
:10249000CDE90610002005904FF4000008900120BF
:1024A000099038465146FEF774F9002D18BFBAF16D
:1024B000000F05D1484605F02BF850B90FE000BFDA
:1024C000384629465246FEF7C3F8484605F020F83C
:1024D00028B101A948463A4604F0AEFDD0B343F214
:1024E00028134FF4B167C2F2004314FB0732D2F84D
:1024F0008005D2F88415013000F01F00884220D0FA
:1025000002F5B06214FB07332C27166806FB07F5AB
:1025100006FB0737019E5E510A9B7B620B9BBB62E9
:10252000029B7B60039BBB60049BFB60059B3B6144
:10253000069B7B61079BBB61089BFB61099B3B6220
:1025400010600022884208BF4FF0FF3250B20CB03A
:10255000BDE8F087002250B20CB0BDE8F087000063
:1025600061B180B582B091F804C00A684B1D0021AA
:10257000CDF800C0FFF720FF02B080BD6FF0010072
:1025800070470000000000002DE9F04796B001A858
:1025900041F6200500F12409C2F200450CAE00BF4F
:1025A0002846314604F054FF0028F9D043F228179A
:1025B00041F62005C2F20047C2F200452C2401AECC
:1025C000D7F88005D7F88415884234D0284604F01F
:1025D0009FFF00281EBFD7F88005D7F884158842D2
:1025E00029D0D7F884054A4600FB04F100FB0470AB
:1025F000795801914168029181680391C168049101
:102600000169059141690691816A0B91416A0A91BC
:10261000016A0991C169089180690790D7F884051A
:102620003146013000F01F00C7F88405284604F049
:1026300003FD0028C4D041F6C0050CAEC2F200452F
:102640002846314604F004FF0028F9D041F6C005C1
:102650002C24C2F2004501AED7F8080BD7F80C1BAA
:1026600088423DD0284604F053FF00281EBFD7F80B
:10267000080BD7F80C1B884232D0D7F80C0B4A460F
:1026800000FB0470D0F888150191D0F88C150291E8
:10269000D0F890150391D0F894150491D0F89815BE
:1026A0000591D0F89C150691D0F8B0150B91D0F893
:1026B000AC150A91D0F8A8150991D0F8A415089185
:1026C000D0F8A0050790D7F80C0B3146013000F088
:1026D0001F00C7F80C0B284604F0AEFC0028BBD046
:1026E00041F660150CAEC2F2004500BF28463146E7
:1026F00004F0AEFE0028F9D041F6601541F29006D4
:1027000041F29404C2F200454FF02C0A0DF1040886
:10271000B8593959884238D0284604F0F9FE0028C3
:102720001EBFB859395988422FD038594A4600FB44
:102730000A70D0F8101B0191D0F8141B0291D0F848
:10274000181B0391D0F81C1B0491D0F8201B059195
:10275000D0F8241B0691D0F8381B0B91D0F8341B0D
:102760000A91D0F8301B0991D0F82C1B0891D0F8B1
:10277000280B079038594146013000F01F003851AE
:10278000284604F059FC0028C2D016B0BDE8F087F6
:1027900014F0CEBC0000000007284FF0FF010CD859
:1027A000012202FA00F010F0C10F06D080B52820F7
:1027B00005F01EFE0021BDE8804048B270470000D1
:1027C00007284FF0FF010CD8012202FA00F010F0A8
:1027D000C10F06D080B5282005F01EFE0021BDE8FF
:1027E000804048B270470000072801D90020704798
:1027F00080B54AF21441C0F6010101EBC00231F884
:102800003010506805F030FD0138B0FA80F0400912
:1028100080BD00000000000021B1072806D9FF207C
:1028200040B27047FE2040B2704700BF4AF21442E7
:10283000C0F6010232F83000C2071FD182071FD450
:1028400042071FD402071FD4C2061FD482061FD41A
:1028500042061FD402061FD4C2051FD482051FD40E
:1028600042051FD402051FD4C2041FD482041FD402
:1028700042041FD4000424D50F201CE000201AE0DD
:10288000012018E0022016E0032014E0042012E0EA
:10289000052010E006200EE007200CE008200AE0EA
:1028A000092008E00A2006E00B2004E00C2002E0EA
:1028B0000D2000E00E2040F69C32C2F2004242F8A9
:1028C0002010002040B27047072803D9FF2040B2F3
:1028D000704700BF80B50A464AF21441C0F60101B4
:1028E00001EBC00331F83010586805F0C5FC00203A
:1028F000BDE8804040B2704714F0EAB90000000023
:10290000012803D9FF2040B2704700BF4AF20C51A2
:10291000B7EE001AC0F6010151F8301080FE410AEE
:102920009FED131A0A6880FE010AD16A01F10101C4
:1029300001EE101AB8EE411A20EE010ABCEEC00AF0
:1029400010EE101A40B101280CD102F138000160DC
:10295000002040B2704700BF02F14000016000203B
:1029600040B2704702F15C000160002040B2704745
:10297000000000000000000010B52DED028B0128C2
:1029800004D9FF2040B2BDEC028B10BD0446B0EE6E
:10299000408A06F0DDFD4AF20C51BFEE001AC0F687
:1029A000010151F834104A680132B0FBF2F000EE38
:1029B000100A0022B8EE400A80EE080A30EE010A42
:1029C000BCEEC00A10EE100AB2EB104F04D0FF208C
:1029D00040B2BDEC028B10BD0A68D062C860002016
:1029E00040B2BDEC028B10BD012803D9FF2040B2DC
:1029F000704700BF80B54AF20C52C0F6010202EBEC
:102A0000C00152F83000898808F0BAFF0020BDE804
:102A1000804040B270470000012803D9FF2040B237
:102A2000704700BF80B54AF20C52C0F6010202EBBB
:102A3000C00152F83000898809F072F80020BDE822
:102A4000804040B27047000080B5012814D841F69C
:102A5000882E8446C2F2004E41F6002018BF4FF087
:102A6000000EC2F20040BCF1000F18BF704618B152
:102A700033B107F0F1FD06E0FF2040B280BD00BF9A
:102A8000142307F0EDFB002818BF012040B280BDE1
:102A900052B140F66043C2F2004303EB401040F8ED
:102AA0002120002040B27047FE2040B27047000055
:102AB00080B5012814D841F6882E8446C2F2004E13
:102AC00041F6002018BF4FF0000EC2F20040BCF1EA
:102AD000000F18BF704618B133B108F089F806E04E
:102AE000FF2040B280BD00BF142307F0C5FE0028C0
:102AF00018BF012040B280BD70B5044612F0E0FD61
:102B00000546FF2612F0C0FD411C05290CD8012006
:102B1000884010F0310F0CD110F0060F0CD0204679
:102B200004F02EFA13E000BF6FF00041884218BF96
:102B3000002670B270BD00BF4FF47A70B0FBF5F1A3
:102B4000B4FBF1F0A14288BF012012F071FD002614
:102B500070B270BD0000000015F0D2BF0000000090
:102B60002DE9F04112F0ACFD044615F0C9FF4EF21C
:102B700018074FF47A78CEF20007B8FBF4F404FBA0
:102B800000F63D6815F0BCFF60433968864200FBE3
:102B900008F008BF294657F8042C01FB08F1013260
:102BA000B1FBF2F1401A002100F57A70BDE8F08126
:102BB00041F6F43241F68841C2F20042012818BFC2
:102BC0000022C2F20041002818BF11460846704793
:102BD0000068C169C90658BF704745F20001042367
:102BE000C4F2000101F54C42904240F6A04208BFF9
:102BF0000123411AC2F2004218BF194601EBC1017C
:102C000002EB810110220262086A08B1004700BF8E
:102C1000704700000000000080B5022802D9FF20A4
:102C200040B280BD8446FE20002918BF002A01D191
:102C300040B280BD41F6F43E41F68840C2F2004EFB
:102C4000BCF1010F18BF4FF0000EC2F20040BCF102
:102C5000000F18BF70461BB109F062FE40B280BD84
:102C600009F056FF40B280BD32B1FF23022898BF61
:102C7000082905D958B27047FE2358B2704700BFE3
:102C800000EBC00040F6A043C2F2004303EB80001B
:102C9000002340F8212058B27047000000000000D7
:102CA00080B5022802D9FF2040B280BD8446FE20B4
:102CB000002918BF002A01D140B280BD41F6F43E80
:102CC00041F68840C2F2004EBCF1010F18BF4FF030
:102CD000000EC2F20040BCF1000F18BF70461BB1DD
:102CE00009F0AEFF40B280BD0AF01AF840B280BDD4
:102CF000B0B578B10446017401202070FFF72CFFB5
:102D0000217C0025C4E902050846FFF785FE68B26C
:102D1000B0BD00BFFF2568B2B0BD000000000000DC
:102D20002DE9F0472DED0A8B002800F0B080044615
:102D30000078FF25002800F09780022900F2948097
:102D400048B256A158A2B2EE08AAB6EE008A51F8CF
:102D5000201052F820004F1C451E4FF001094FF083
:102D6000000A9FED54BA9FED54CA00BF17F8010C3A
:102D7000B7F80180FF283ED0397801EB410100EB24
:102D800081000C3000EE100AB8EEC00A30EE0B0ADB
:102D900080EE0A0A16F06AFE20EE0C9A2078B5EE54
:102DA000409AF1EE10FA25DD002870D084F80090EA
:102DB000FFF7D2FE217CB0EE490AC4E9020A0846B8
:102DC000FFF7DAFD217CB0EE480A06460846FFF719
:102DD00097FD30434ED12078002858D084F80090D9
:102DE000FFF7BAFE217CC4E9020A0846FFF7FCFDA2
:102DF00058B13FE048B184F80090FFF7ADFE217C68
:102E0000C4E9020A0846FFF707FE4046FFF774FED2
:102E1000207848B184F80090FFF79EFE217CC4E939
:102E2000020A0846FFF7F8FD1420FFF765FE207838
:102E300045B1002807F10407A5F1010596D1FF254A
:102E400012E000BF4FF0000570B101202070FFF7C5
:102E500083FE217CC4E902050846FFF7DDFD68B268
:102E6000BDEC0A8BBDE8F08768B2BDEC0A8BBDE80B
:102E7000F08700BF207850B101202070FFF76CFE72
:102E8000217C0022C4E902020846FFF7C5FDFF25A8
:102E900068B2BDEC0A8BBDE8F08700BF1CA5010835
:102EA000D8A4010854A401080D0000000D00000082
:102EB0002100000000008AC20000DC430000000086
:102EC00010B52DED048B18B30446007800B3B0EEB6
:102ED000608AB0EE409A01202070FFF73DFE217C11
:102EE000B0EE490A0022C4E902020846FFF744FD99
:102EF000217CB0EE480A04460846FFF701FD204356
:102F000018BF4FF0FF3040B2BDEC048B10BD00BFC6
:102F1000FF2040B2BDEC048B10BD0000000000009B
:102F200010B598B10446007880B101202070FFF7F9
:102F300013FE217C0022C4E902020846FFF754FD7B
:102F4000002818BF4FF0FF3040B210BDFF2040B244
:102F500010BD00000000000010B598B104460078D4
:102F600080B101202070FFF7F7FD217C0022C4E929
:102F700002020846FFF750FD002818BF4FF0FF304F
:102F800040B210BDFF2040B210BD000000000000A4
:102F9000FEE700000000000030B380B584B040F6CA
:102FA000E4328378C2F2004240F20F3100910821EE
:102FB00012788DF804100188C078ADF80510991AC0
:102FC0008DF807108DF808000020CDF8090069463B
:102FD0000220FFF7C5FA002818BF4FF0FF3004B0F9
:102FE000BDE8804040B27047FE2040B2704700000C
:102FF00003284FF0FF020FD871B141F23022C2F224
:10300000004252F8200018B102690AB180681047E6
:10301000007900220A54FC2250B2704700000000E0
:1030200010B540F2100041F23024C2F20040C2F26A
:1030300000440179032998BF44F82100017F032946
:103040000AD990F8341003290ED990F84C100329AE
:1030500012D92068A8B918E000F1180244F821201C
:1030600090F834100329F0D800F1300244F8212000
:1030700090F84C100329ECD8483044F8210020681F
:1030800018B1C16809B180688847606818B1C16823
:1030900009B180688847A06818B1C16809B1806823
:1030A0008847E06818B1C16809B180688847002086
:1030B00010BD0000000000000146006890ED030A0A
:1030C00091ED4D1A20EE011A002081ED4D1A91ED7F
:1030D0004E1A20EE010A81ED4E0A704700000000F2
:1030E000817C51B190F82811012906D1022180F884
:1030F000401180F86C1180F88011002070470000AA
:103100000146006890ED020A91ED4E1A31EE400A38
:10311000002081ED4E0A704790F82811012903D054
:1031200059B9012101E000BF002180F8281180F881
:103130002C1180F8401180F86C11002070470000BD
:1031400001460020012281F86F2170470000000035
:10315000014690F86D01421C002002F0030281F844
:103160006D217047000000000146006890ED020AE2
:1031700091ED4E1A30EE010A002081ED4E0A7047A3
:103180000146006890ED020A91ED4D1A31EE400AB9
:10319000002081ED4D0A704740F698010020C2F2F0
:1031A00000410A7882F001020A70704700000000B6
:1031B0000146006890ED020A91ED4D1A30EE010AC9
:1031C000002081ED4D0A704701464FF40170022244
:1031D000A1F83001002081F8442170470000000070
:1031E00000207047000000002DE9F04381B08046C8
:1031F00000284FF0FF0000F076800F46002900F015
:1032000072804AF648291D4616460024C0F6010978
:1032100007E000BFC1684046884700BF1034B02CAB
:1032200060D009EB0400417A2942F7D0426882F06D
:103230000041D30043EA517106291BD8DFE801F0B1
:10324000061A1A1A04102E00E8E700BF97F8221099
:10325000002918BF0121BEB396F8222026E000BF46
:1032600097F82410002918BF01216EB396F8242086
:103270001CE000BFB96A01EA0201A1EB0201B1FA48
:1032800081F14FEA5111FEB1B36A13409A1AB2FAB2
:1032900082F25209037A73B91AE000BF97F823103B
:1032A000002918BF01217EB196F82320002A18BFFB
:1032B0000122037A63B1022B0ED0012BAED182F032
:1032C00001021142A6D1A9E70022037A002BF2D114
:1032D00000297FF49FAFA1E781F001010A423FF48A
:1032E0009DAF97E7002040B201B0BDE8F083000039
:1032F00001F01EBA000000000078704700000000D6
:103300000022C1E90722C1E9092202784A70D0F8F7
:103310003A20CA61B0F840204A84C28B00208A62F9
:103320007047000000000000B0B500230246C1E96C
:103330000133C1E90333C1E90533007840F20135B7
:10334000087092F839C0506A4860906A8860D06A04
:10335000C860ACF10100C0F20205C0B2D2F830E0A2
:103360004FEAC00C03284FF00000C1F810E038BF4E
:1033700025FA0CF0087592F838000138C0B2C40084
:10338000032838BF25FA04F300204B75526B8A617D
:10339000B0BD00000000000070B52DED028B78B3C9
:1033A0000446FFF7DDFB05460E4616F044FF00EE2F
:1033B000100AE0689FED378A281A66F1000180EE56
:1033C000080A84ED010A16F036FF00EE100A94F8A0
:1033D0002801E560042880EE080A84ED020A15D36E
:1033E000002084F8300184F8440184F86D0184F8E9
:1033F000740184F88101FC2040B2BDEC028B70BDE9
:10340000FF2040B2BDEC028B70BD00BF94F84001BC
:1034100040F2E045C2F20045C0EBC00005EB800081
:10342000816809B12046884794F82C01C0EBC000A0
:1034300005EB8000416809B12046884794F86C018B
:10344000C0EBC00005EB8000C16809B12046884789
:1034500094F87001C0EBC00005EB8000016909B170
:103460002046884794F88001C0EBC00005EB80003F
:10347000816939B120468847002040B2BDEC028BFB
:1034800070BD00BF002084F8810140B2BDEC028B0A
:1034900070BD00BF00247449B0B5044600284FF049
:1034A000FF000CD00D4651B1201D4FF4E271FDF725
:1034B00070F92560FFF7B4FDFFF792FE002040B2DF
:1034C000B0BD0000000000000020704700000000B8
:1034D000817C99B1D0E91012C0F85411816CC0F808
:1034E0005821426DC0F85C21026DC0F86021C26CA9
:1034F000C0E95921032180F844117047002180F868
:103500004411704700000000817C49B190F83C20D4
:103510000121002A08BF022180F88111704700BFF5
:10352000022180F881117047817C99B190F83C109C
:10353000022917D318BF704790F8281171B10129DB
:1035400010D190F8321069B140F20111A0F86E115B
:10355000704700BF002180F86D11704790F825106A
:103560000329F1D00121A0F86E117047000000007E
:10357000024601208870107881F82C00506808639A
:1035800090684863D06888631069C86350690864AC
:10359000002092694A6470470120704700000000D3
:1035A000417C79B100F11001022280F8302100F154
:1035B0009C0202234FF0000CC0F834C1C0F838C19F
:1035C000FFF712BE002180F83011704700000000A4
:1035D000417C69B3B0F92E1090ED022AB0F92C208D
:1035E000B7EE083A4942042300EE101A524201EEA7
:1035F000102A0168012280F84421B8EEC00A00F1C7
:103600009C02B8EEC11A22EE000A22EE011A91EDD8
:10361000012A00F1100122EE000A22EE011A80EDCB
:10362000521A20EE030A80ED530AFFF7DDBD00BFFA
:10363000002180F844117047417C69B100F110010C
:10364000012280F86E2190F832C000F19C0208231C
:1036500080F86FC1FFF7C8BD002180F86D11704779
:10366000417C79B100F11001012280F8742100F150
:103670009C0210234FF0000CC0F878C1C0F87CC148
:10368000FFF7B2BD002180F87411C0E95E117047E8
:1036900090F824200168032A06D0022A06D0012AC5
:1036A00008D1143103E000BF163100E0153109786C
:1036B00001E000BF002180F83011C169C0F8341169
:1036C000016AC0F838114169C0F83C117047000028
:1036D00090F824200168032A06D0022A06D0012A85
:1036E00008D1173103E000BF193100E01831097823
:1036F00001E000BF0021B8EE000AB8EE041A90ED18
:10370000052A80F8441122EE000A90ED062A22EEE6
:10371000011A80ED520A80ED531A70470000000034
:1037200090F82510027C80F86D21032908D0022929
:103730000ED10022012180F86E1180F86F217047B0
:103740000121012280F86E1180F86F21704700BFBF
:103750000021002280F86E1180F86F217047000070
:10376000014611F8102F2AB390ED080A80F8742151
:10377000B5EE400AF1EE10FA16DB30EE000AB7EEB5
:10378000001A80ED5E0AB0EEC02AB4EE412AF1EED6
:1037900010FA09DDBFEE002AB5EE400AF1EE10FA8C
:1037A00031FE020A80ED5E0A00F19C021023FFF751
:1037B0001BBD00BF002180F87411C0E95E11704785
:1037C000002070470000000080B50346007808B173
:1037D00001200FE093F8400010B101200AE000BF83
:1037E00093F8300010B1012004E000BF187B0028DE
:1037F00018BF0120C87001F1480044221946FCF7A7
:103800006CFF002080BD0000017829B990F84010BD
:1038100011B990F8301009B101207047007B0028E1
:1038200018BF01207047000030B370B500F19C054F
:1038300000F1100604468C2228463146FCF74DFF65
:1038400000203146FFF7D4FB01203146FFF7D0FBC3
:1038500002203146FFF7CCFB03203146FFF7C8FBBF
:1038600094F82801022802D82118097C79B9207C13
:1038700030B1002009E000BF4FF0FF30704700BFBB
:10388000617C0120002908BF042084F8280184F805
:103890002C01012384F84001314684F86C012A464A
:1038A00084F8700184F880012046FFF79DFCA07C1D
:1038B00068B194F8280150B994F82400032806D17F
:1038C000022084F8400184F86C0184F880012046CD
:1038D000FFF762FD054604F5C27004F15801442269
:1038E000FCF7FBFE284670BD70B5002951D04AF2A6
:1038F000F46311F0030EA1F1010CC0F6010320D016
:10390000D6B20446BEF1010F14F8015B85EA060544
:1039100033F8155085EA122206D161462046BCF1E3
:10392000030F36D310E000BFD2B24478BEF1020FCD
:1039300082EA040233F8124084EA15222CD10239BB
:103940000230BCF1030F24D3043800BFD5B210F805
:10395000046F92B244786E40043933F81660F5B2C1
:1039600085EA1222857882EA040233F81220D4B262
:1039700084EA162686EA0506C57833F81660F4B29E
:1039800084EA122282EA050233F8122082EA162221
:10399000DCD190B270BD00BFD2B28678033003395B
:1039A000724033F8122082EA1422BCF1030FF0D3E4
:1039B000CAE7000000000000022901D20020704781
:1039C000F0B58A1E4FF6FF7354D0CD1E4AF2F46E46
:1039D000032D02F0030CC0F6010E01D2024629E0CD
:1039E00022F0030254420246DEB212F8045B0434B1
:1039F00085EA060512F8036C3EF81550EFB287EA27
:103A0000132383EA060312F8026C3EF81330DFB288
:103A100087EA152585EA060512F8016C3EF815506F
:103A2000EFB287EA132383EA06033EF8133083EAF2
:103A30001523D9D1BCF1000F1CD0DDB21478BCF134
:103A4000010F84EA05043EF8144084EA132311D0E0
:103A5000DBB25578BCF1020F83EA05033EF8135040
:103A600085EA142306D0DBB292785A403EF8122041
:103A700082EA152301F0010221F0010110440844FB
:103A800030F8020C181AB0FA80F04009F0BD0000BE
:103A9000B0B5C9B34AF6F40311F0030EA1F1010C5D
:103AA000C0F6010317D00446BEF1010F14F8015B04
:103AB00082EA05029A5C05D161462046BCF1030FFB
:103AC00022D30BE04478BEF1020F82EA04029A5C32
:103AD0001CD102390230BCF1030F15D3043800BFEA
:103AE000D2B210F8045F043982EA050245789A5C84
:103AF00082EA050285789A5C82EA0502C5789A5CBA
:103B000082EA05029A5CEBD1D0B2B0BD8578033071
:103B100003396A409A5CBCF1030FF5D3DEE700007D
:103B2000022901D200207047B0B58A1EA1F1010E12
:103B3000032A4AF6F4020EF0030CC0F6010203D287
:103B4000FF2301461CE000BF2EF00301FF234C427F
:103B5000014600BF11F8045B043483EA050311F841
:103B6000035CD35C83EA050311F8025CD35C83EA4F
:103B7000050311F8015CD35C83EA0503D35CE9D14A
:103B8000BCF1000F10D00C78BCF1010F83EA0403E4
:103B9000D35C09D04C78BCF1020F83EA0403D35CF8
:103BA00002D089785940535C10F80E00181AB0FA08
:103BB00080F04009B0BD00002DE9F04381B02DED4B
:103BC000068B804600284FF0FE0000F02A810D464B
:103BD000002900F02681D8E90001101A4FF00004F6
:103BE00064EB0101914616F026FB00EE100A9FEDF2
:103BF000AE1AC8E9009480EE011A9FEDAC0A88ED78
:103C0000021AB5EE401AF1EE10FA0DDD11EE100AAF
:103C100000F0FF40B0F1FF4F06D09FEDA50AB4EED3
:103C2000401AF1EE10FA47DA88ED020A2F7898F878
:103C30001000B8424ED1052F00F08880012F03D12B
:103C40000020C8F8140085E098ED0C0A98EDB71A2A
:103C500031EE408AB0EE480A15F060FEB0EE409AB0
:103C6000B0EE480A15F0E6FF95ED011A95ED022A2F
:103C700029EE013A98F8100029EE024A062800EED3
:103C8000423A00EE014A88ED053A88ED064A67D8C7
:103C90009FED890ADFE810F0620062000800D4009E
:103CA000E6006200040100BF08F59C70D8ED021A1E
:103CB00098ED0C0ACEE000BF9FED7E0AB4EE401AEC
:103CC000F1EE10FAC8BF88ED020A2F7898F81000BC
:103CD000B842B0D0042F11D104280FD04846FCF7C9
:103CE00099FCFCF769FBC0074FF0FF3008BF0120CB
:103CF00000EE100AB8EEC00A88ED0D0A98F911001E
:103D000001281EDB00269FED6C8A0024C6EB0610FE
:103D100008EB800048300AF003FFB0EE480A08EBD9
:103D2000461606F5C67009F07FF9B0EE480A06F5AA
:103D3000037009F079F9013498F91100E6B286426E
:103D4000E4DB88F81070052F7FF478AF6868C8F856
:103D50001400A868C8F818009FED570A88ED070AF4
:103D600098F9113008F1120008F1140108F1380235
:103D70009FED560A0AF044FC98F91100012857DB20
:103D800000249FED4D8A9FED52AA002529E000BF37
:103D9000C4EB0410F0EE400AB0EE481A99ED000AA8
:103DA00008EB8000D8ED021A48300AF0BDFDB0EEF5
:103DB000409AB0EE490A07F5037009F0ADF8D8F85B
:103DC0000C0086EDA30AD0ED1F0A06F52370B1EEB4
:103DD000600A00F045FA013598F91100ECB284420E
:103DE0001EDA08EB041108EB441708EB840607F50C
:103DF000C67091EDA80A06F1380909F08DF898F817
:103E00001000411E0529C3D330B10628D1D199ED48
:103E1000000A80EE0A9ACCE7B0EE489AC9E700BFE4
:103E2000002040B2BDEC068B01B0BDE8F08300BFBE
:103E3000002040B2BDEC068B01B0BDE8F08300BFAE
:103E400098ED0C0A9FED201A30EE010A08F59C70DF
:103E5000D8ED021AD8EDB70A9FED171A0AF064FDE3
:103E60007CE700BF00EE109A9FED101A98ED0D8AC6
:103E7000B8EE400A20EE010A15F0DCFE9FED0F1AA5
:103E800020EE010A9FED0E1AB0EEC00A30EE010AD4
:103E90009FED0C1A80FE410A28EE000A5EE700BF83
:103EA00095ED030A5AE700BF00007A446F12833A87
:103EB0006F12033ACDCC4C3D00000000CDCC4C3EFF
:103EC0009A99193FCDCC4C3FAB611C3F0000FA439F
:103ED00000C0DA45000000002DE9F04F81B02DED63
:103EE000028BE8B18346B0EE408A8A46FDF774FD46
:103EF0009AF86080FC21CBF80CA00020B8F1060FE6
:103F00008BF8100000F26E800420DFE808F0121237
:103F100005120B6B0F0000BF02204FF0020808E0F3
:103F2000FE215FE004204FF0040802E04FF0050896
:103F3000012000260AF12009002500278BF8110036
:103F4000CBE90066CBF80860C5EB0510B0EE480A77
:103F500000214A460BEB800048300AF095FDB0EE98
:103F6000480A0BEB451404F5C670DAED190A09F09E
:103F700003F8B0EE480A04F50370DAED1A0A08F007
:103F8000FBFF01379BF911100BEB0510FDB28D42C1
:103F9000C0F89C62C0F8A062C0E9A966D4DBB0EEAC
:103FA000480A0BF59C700AF1400201210AF06CFDF1
:103FB0000BF1120041460AF0A7FC9BF91100002109
:103FC000CBE905110128CBF81C100BDB411E00F0DA
:103FD000030CC9B2002203290AD20123BCF1000F4D
:103FE0002AD141E048B2BDEC028B01B0BDE8F08FB0
:103FF00000F0FC030BF51F770BF52376002100BFC3
:104000000D4641F00101C9B247F8102F45F00304F5
:10401000043BE4B246F8212045F00201C9B246F85B
:10402000242046F82120190605F10401E8D1CAB27E
:104030006B1DBCF1000F17D00BEB8202BCF1010F1E
:104040004FF00001C2F88C120ED0DAB2BCF1020FB0
:104050000BEB8202C2F88C1206D0591C0022C9B2A6
:104060000BEB8101C1F88C2201280CDB0025002616
:10407000DBF80C00284409F083FC9BF911000136A1
:1040800008358642F4DB002148B2BDEC028B01B05A
:10409000BDE8F08F00000000002808BF7047B0B5F1
:1040A00090F911100446012912DB0020002504E0DC
:1040B0004AB20135E8B290420ADA04EB8002106A93
:1040C0000028F5D092EDA30A09F0EEFC617CEFE741
:1040D000206ABDE8B04008B109F082BB704700001B
:1040E00070B52DED028B8EB00446006A04F12403F6
:1040F0000AAEC0680A900ECBB0EE408A04F5237574
:10410000C8680B90D0680C90217CDA6840F29C0360
:1041100040F28000C2F20043C2F2004004290D9236
:1041200008BF1846D4F88C120591D4F89012069165
:10413000D4F894120791D4F89812089105A9324640
:10414000099011F0DDFEB0EE480A09A8012112F035
:10415000F3F80998D4F88C120191D4F890120291D6
:10416000D4F894120391D4F89812049101A932461C
:104170002B4612F035F80EB0BDEC028B70BD00007E
:1041800070B5044690F91100012820DB00260025B7
:10419000E06800EBC60009F013FDE06800EBC60024
:1041A00009F0A6FB04EB8601086298B104EB061146
:1041B00000F1080C406901359CE80C10C1E9A72307
:1041C000EEB294F91120C1E9A9C09642E0DB0020CB
:1041D00040B270BDFE2040B270BD00000000000083
:1041E00090ED001AF5EE400A31EE000AF1EE10FAF9
:1041F0000BDDB4EE600AF1EE10FA09DAB5EE400A12
:10420000F1EE10FA01DA30EE200A80ED000A704774
:1042100030EE600A80ED000A7047000000000000E8
:1042200030EE600AB5EE401AF1EE10FA16DDB6EE89
:10423000002A21EE022AB4EE420AF1EE10FA03DD62
:1042400030EE410A704700BFB1EE422AB4EE420A96
:10425000F1EE10FAA8BF704730EE010A7047000077
:1042600090ED002A82FE601AB4EE602AF1EE10FA98
:1042700005DCB4EE401AF1EE10FAA8BF704781FEDB
:10428000000A80ED000A704740F2B800C2F2004018
:10429000704700000000000041F2C850C2F2004028
:1042A00001F03ABD0000000041F24060C2F200405F
:1042B00001F032BD0000000041F2B860C2F20040DF
:1042C00001F02ABD0000000041F23070C2F200404F
:1042D00001F022BD0000000041F2A870C2F20040CF
:1042E00001F01ABD0000000040F20F42D0F800C0FB
:1042F000C4F20202944511DC6F22C4F2020294451A
:1043000022DC3F22C4F20202944539DC1022C4F2BE
:10431000020294455AD0282254E000BF40F26F4276
:10432000C4F2020294451BDC40F23F42C4F2020296
:1043300094452DDC40F21042C4F20202944545D06F
:1043400040F228423EE000BF9F22C4F202029445A0
:1043500028DC7022C4F20202944537D0882231E072
:1043600040F29F42C4F20202944523DC40F27042C4
:10437000C4F20202944529D040F2884222E000BFF4
:104380004022C4F20202944520D058221AE000BF15
:1043900040F24042C4F20202944517D040F2584223
:1043A00010E000BFA022C4F2020294450ED0B82251
:1043B00008E000BF40F2B842C4F20202944505D0C2
:1043C00040F2A042C4F20202944519D16FF00F02EC
:1043D0004AF6AB2352FA8CF2CAF6AA23A2FB0331A7
:1043E0000AA35F2AC1F302115B5C40F2FF312CEAA1
:1043F0000101C36588BF043181650846704700BF6D
:104400002CF0FF0181650846704700BF00061016BA
:10441000000610160000000070B540F26F44D0F89E
:1044200000C0C4F20204D0F858E0A4451ADC9F256D
:10443000C4F20205AC4533DC5725C4F20205AC4595
:104440005ADC1025C4F20205AC4500F098802825FE
:10445000C4F20205AC4500F092804025C4F202058A
:104460008AE000BF45F22F45C5F60205AC452DDCBC
:1044700040F2B745C4F20205AC454BDC40F2704552
:10448000C4F20205AC457AD040F28845C4F2020578
:10449000AC4574D040F2A045C4F202056CE000BF08
:1044A00040F22745C4F20205AC4543DCA025C4F226
:1044B0000205AC4563D0B825C4F20205AC455ED018
:1044C00040F21045C4F2020556E000BF45F26B45CC
:1044D000C5F60205AC453FDC45F23045C5F60205A0
:1044E000AC454CD045F24445C5F60205AC4546D036
:1044F00045F258453EE000BF5825C4F20205AC45E0
:104500003DD07025C4F20205AC4538D08825C4F2F0
:10451000020531E040F2B845C4F20205AC452ED0A8
:1045200045F20845C5F60205AC4528D045F21C45C4
:1045300020E000BF40F22845C4F20205AC451ED081
:1045400040F24045C4F20205AC4518D040F258454F
:10455000C4F2020510E000BF45F26C45C5F6020545
:10456000AC450CD045F29445C5F60205AC4506D0E5
:1045700045F28045C5F60205AC4540F0D580456E54
:10458000C66E002E866E6E601CBFD0E91C566E6033
:10459000A44515DC9F24C4F20204A4452CDC572456
:1045A000C4F20204A44551DC1024C4F20204A44560
:1045B0007AD02824C4F20204A44575D040246FE0C8
:1045C00045F22F44C5F60204A44529DC40F2B74465
:1045D000C4F20204A44545DC40F27044C4F2020473
:1045E000A44561D040F28844C4F20204A4455BD0E3
:1045F00040F2A04454E000BF40F22744C4F2020459
:10460000A4453FDCA024C4F20204A4454CD0B82445
:10461000C4F20204A44547D040F2104440E000BF79
:1046200045F26B44C5F60204A44555DC45F230441E
:10463000C5F60204A44561D045F24444C5F602041F
:10464000A4455BD045F2584454E000BF5824C4F25E
:104650000204A44528D07024C4F20204A44523D047
:1046600088241DE040F2B844C4F20204A4451BD0E3
:1046700045F20844C5F60204A4453FD045F21C4467
:1046800038E000BF40F22844C4F20204A4450BD035
:1046900040F24044C4F20204A44505D040F258441C
:1046A000C4F20204A4453FD18468C06D00F01F002D
:1046B0003F2505FA00F0CEF80800DCF80000402C99
:1046C00020F48020CCF80000CCF8043023D0CCF8C3
:1046D0000810CCF80C2070BD45F26C44C5F60204FD
:1046E000A4450BD045F28044C5F60204A44505D08C
:1046F00045F29444C5F60204A44515D1C46D806802
:1047000004F01F040125402805FA04F4CEF8044003
:10471000CCF8043004D1CCF80820CCF80C1070BDD3
:10472000CCF80810CCF80C2070BD00000000000090
:10473000B0B5D8B140F60404C2F20044207818B1F4
:10474000FD2568B2B0BD00BF11F002FB606068B12A
:1047500044F691120020C0F6000203210025FEF766
:1047600083FA0120207068B2B0BD00BFFE2568B298
:10477000B0BD00000000000010B538B134210024A5
:1047800000F8244BFCF705F860B210BDFE2460B2BF
:1047900010BD000000000000B0B508B30546044697
:1047A00055F8100F01466FF3DF21A1F5B671B1F591
:1047B000A56F11D8C0F3CA21A1F5B671B1F5A56FE7
:1047C0000AD8A988800D40EA81206FF3DF20A0F588
:1047D000B670B0F5A56F07D9FF2040B2B0BD00BFDD
:1047E000FE2040B2B0BD00BF11F4405F4FF0FF00AB
:1047F00000F0C5808AB2B2F5804FC0F0C080C1F32E
:104800004A01A1F5B671B1F5A56F00F2B88001209B
:104810002070FEF7A5F92A6894F81CC013466FF3C0
:10482000DF23BCF1000F00EE103AA369C4E90201D6
:10483000C2F3CA20A988B8EE401A9FED520AE3637A
:1048400031EE001A31EE012A01EE100A4FEA9250C1
:1048500040EA81206FF3DF20B8EE413A04EE100AFF
:104860009FED491AC1F34A0082EE012A05EE100AB3
:1048700033EE003AB8EE444A84ED0B2A4FEA913207
:1048800084F83920B8EE455AE28A34EE004A4FF0F7
:10489000000033EE033A6065C1F3013135EE005A92
:1048A00034EE044A84F8381083EE013A628735EE1C
:1048B000052A84ED0C3A84EE013A627F84ED093AD0
:1048C00082EE012A84ED0A2A18BF4FF0010C002A5B
:1048D00084F840C018BF0122E38B84F852C084F8EA
:1048E0004120DDB203F0010184F84210C5F340011C
:1048F00084F84310C5F3800184F84410C5F3C00167
:1049000084F84510C5F3001184F84610C5F3401132
:1049100084F84710C5F3801184F84810E90984F839
:104920004910C3F3002184F84A10C3F3402184F8EE
:104930004B10C3F38025218C84F84C5002EE101AE2
:1049400084F85320C3F3C02184F84D10C3F3003121
:1049500084F84E10C3F34031B8EE422A84F84F1069
:10496000C3F3803184F8501032EE000AD90B84F87A
:10497000511030EE000A80EE010A84ED0D0A40B2BB
:10498000B0BD00BF000080C40000A54400000000CE
:1049900040F604000121C2F20040406811F0E0B886
:1049A00010B504460020FEF703F904F110011222AD
:1049B00007F0B6FF002818BF4FF0FF3010BD000011
:1049C00080B502460120012111F00EF90138B0FA3C
:1049D00080F0400980BD000070470000000000002A
:1049E00080B54FF4806003F03FFB4FF4805003F03C
:1049F0003BFB4FF40040BDE8804003F035BB0000B6
:104A0000EFF3108072B600BFFEE700000000000068
:104A100044F60400C5F60200816841F0020181609D
:104A20000168890409D4016889045CBF01685FEAF0
:104A3000814102D401688904F2D57047000000006A
:104A400041F62000C2F2004002F06EBD00000000FE
:104A500041F62000C2F2004002F066BD00000000F6
:104A600041F6C000C2F2004002F05EBD000000004E
:104A700041F6C000C2F2004002F056BD0000000046
:104A800041F66010C2F2004002F04EBD000000008E
:104A900041F66010C2F2004002F046BD0000000086
:104AA00070B54FF0FE0608B30C46F9B15821054623
:104AB000FBF76FFE20890A222883002620686168A0
:104AC0006961286120782E706188FDF781F820786F
:104AD000A1880A22FDF77CF82078E1880A22FDF7F8
:104AE00077F820780A222189FDF772F870B270BD3C
:104AF000B0B5002818BF002A00D1B0BD438A8B4250
:104B000046D192F800C015795378547991789FED89
:104B10009A2A5B0192F803E043EA4C339FED904AF6
:104B200043EAD10C4FEA8E2300EE10CA61F394439E
:104B300043EA85019379D27941EA9411DB0101EED0
:104B4000101A64F3D433B8EE400A43EA520203EE7B
:104B5000102AB8EE411A20EE020AB8EE433A21EECE
:104B6000021A80EE040A23EE022A9FED843A81EEB7
:104B7000041A30EE030A82EE042A80ED070A31EEB1
:104B8000031A80ED081A32EE030A80ED090AB0BD5F
:104B9000838A8B4244D111789FED752A53789FED1B
:104BA000704A9578D4785B0143EA41311379A402C5
:104BB00041EAD50C517965F394449579D27944EA68
:104BC0008303ED0100EE10CA61F3D43543EA91137B
:104BD00045EA520101EE103A03EE101AB8EE400A0F
:104BE000B8EE411AB8EE433A20EE020A21EE021A5C
:104BF00023EE022A9FED5F3A80EE040A81EE041A4A
:104C000082EE042A30EE030A31EE031A80ED0A0A1E
:104C100032EE030A80ED0B1A80ED0C0AB0BD00BF26
:104C2000C38A8B4248D111789FED4C2A53789578EE
:104C3000D4785B0143EA41311379A40241EAD50CEF
:104C4000517965F394449579D27944EA8303ED016F
:104C500000EE10CA43EA911361F3D43501EE103A25
:104C600045EA5201B8EE400A03EE101AB8EE411AB6
:104C700020EE020A9FED3C2AB8EE433A21EE021ADA
:104C800023EE022A9FED363A80EE030A81EE031AE4
:104C900082EE032A9FED333A30EE030A9FED333A5A
:104CA00080ED0E0A31EE030A80ED0D0A32EE030AA2
:104CB00080ED0F0AB0BD00BF038B8B4218BFB0BDA3
:104CC00051789FED251A9378BFEE005AD4789D084D
:104CD00045EA8111157900EE101A210163F30D31B7
:104CE0005379947941EA15119B00D27965F38D23AC
:104CF00002EE101A43EA9413B8EE400A64F30D2250
:104D000003EE103A04EE102AB8EE422A30EE000A02
:104D1000B8EE433AB8EE444A32EE022A33EE033A92
:104D200080EE010A34EE044A82EE012A83EE013A53
:104D300084EE011A30EE050A80ED100A32EE050A03
:104D400080ED110A33EE050A80ED120A31EE050AF4
:104D500080ED130AB0BD00BF00FC7F460000344365
:104D6000F8FFFF490000B4C20000B443000034C3A0
:104D70001F858B421F850BC23333EB4233336BC22B
:104D8000002869D0F0B587B00446007C6D4600234A
:104D9000618A2A46FCF7C4FDB0FA80F14FEA511748
:104DA00078B905F10D0600BF618A20463246FFF74B
:104DB0009FFE207C0023618A2A46FCF7B1FD002873
:104DC000F2D0207CA18A6D4600232A46FCF7A8FD7C
:104DD00080B905F10D0600BFA18A20463246FFF7D3
:104DE00087FE207CA18A00232A46FCF799FD002833
:104DF000F2D00127207CE18A6D4600232A46FCF789
:104E00008FFD78B905F10D06E18A20463246FFF79D
:104E10006FFE207CE18A00232A46FCF781FD0028F2
:104E2000F2D00127207C6D46218B00232A46FCF717
:104E300077FDA8B11FBBFDF793FED4E90223801ACA
:104E400048F2A162C0F201029941801A71F100009A
:104E50001BD30020207018E0FE2040B2704700BF36
:104E600005F10D06218B20463246FFF741FE207CDE
:104E70000023218B2A46FCF753FD0028F2D00120A5
:104E80002070FDF76DFEC4E90201002007B0BDE807
:104E9000F04040B270470000F0B581B02DED068BB8
:104EA000044600284FF0FF0000F023810D46002942
:104EB00000F01F81FDF754FED4E90023801A9941C8
:104EC00015F0B9F900EE100A9FEDEC1A80EE010A18
:104ED00084ED020AFDF744FE2E78227CC4E900012D
:104EE000B24261D004F1200009F01AFE04F15C0026
:104EF00009F016FE04F1980009F012FE04F1D40046
:104F000009F00EFE04F5887009F00AFE04F5A6709B
:104F100009F006FE04F5C47009F002FE04F5E27023
:104F200009F0FEFD04F5007009F0FAFD04F50F70BC
:104F300009F0F6FD04F51E7009F0F2FD04F52D7080
:104F400009F0EEFD9FEDCE8A04F54070B0EE480A00
:104F500008F06AF8B0EE480A04F5487008F064F802
:104F6000E068083008F098F8E06808F095F804F177
:104F70001400FBF7D1FD032ED4F87403A06107D011
:104F8000022E0DD0012E0ED1D4F864030AE000BF2A
:104F9000D4F858036061D4F85C03A06103E000BF5B
:104FA000D4F8580360612674E868C4F8480395EDA6
:104FB000010A94ED021A20EE010AB7EE081AE06821
:104FC00090ED682A20EE018AB5EE402AF1EE10FA43
:104FD00040DD022E06D194EDD60A94EDD91A31EEB9
:104FE000400A01E09FEDA60A9FEDA61A30EE011AD5
:104FF0009FEDA52AB4EE420A9FEDA49AF1EE10FAB5
:105000009FEDA32A31FE000A30EE091AB4EE402AC1
:10501000F1EE10FA31FE00AA94ED050AB0EE491A3D
:1050200030EE0A0A78EE000A94EDBC0AFFF7F8F8B1
:1050300094ED051A3AEE011AB0EE40AA94EDBD0ABD
:1050400078EE010AB0EE491AFFF7EAF888FE4A1A2C
:1050500081FE008AB0EE480A04F11406DFED8B0AE7
:105060003046FFF7BDF8E06895ED020A94ED021AAC
:1050700090ED692A20EE018AB5EE402AF1EE10FA91
:105080001BDD94ED060A9FED819A78EE000AB0EEE2
:10509000491A94EDBE0AFFF7C3F894ED061AB0EE74
:1050A00040AA78EE010AB0EE491A94EDBF0AFFF764
:1050B000B7F888FE4A1A81FE008AB0EE480A04F169
:1050C0001807DFED720A3846FFF78AF828780328B8
:1050D00003D12869306068693860207C032800F2B9
:1050E0007B80DFE800F0030B377F00BF0020C4E9BE
:1050F000D00040B2BDEC068B01B0F0BD9FED608AE0
:1051000004F12000B0EE481AD4ED021A94ED050A1D
:10511000D4EDD90A09F008FCB0EE481A04F15C009D
:10512000D4ED021AD4EDD50A09F0FEFBB0EE481A10
:1051300084EDD00A04F19800D4ED021A94ED060A29
:10514000D4EDDD0A09F0F0FBB0EE481A04F1D4000A
:105150002AE000BF9FED4A8A04F58870B0EE481A35
:10516000D4ED021A94ED050AD4EDD60A09F0DCFB61
:10517000B0EE481A04F5A670D4ED021AD4EDD50AA3
:1051800009F0D2FBB0EE481A84EDD00A04F1980081
:10519000D4ED021A94ED060AD4EDDD0A09F0C4FB41
:1051A000B0EE481A04F5E270D4ED021AD4EDD30A39
:1051B00009F0BAFB84EDD10A04F5407094EDD00AF1
:1051C00007F0AAFE84EDD00A04F5487094EDD10AE8
:1051D00007F0A2FE84EDD10A002040B2BDEC068BA0
:1051E00001B0F0BD9FED268A04F50070B0EE481ABC
:1051F000D4ED021A94ED050AD4EDD60A09F094FB19
:1052000095ED061A04F50F7030EE010AB0EE481A5B
:10521000D4ED021AD4EDD50A09F086FB95ED081AF3
:105220009FED1C2A01EE020AB0EE481A04F51E702A
:10523000D4ED021AD4EDD70A84EDD00A94ED060A13
:1052400009F072FB95ED071A04F52D7030EE010A96
:10525000B0EE481AD4ED021AD4EDD30A09F064FB7B
:1052600095ED091A9FED0C2A01EE020A002084ED4B
:10527000D10A40B2BDEC068B01B0F0BD00247449E8
:1052800000000000DB0FC9C0DB0F4940DB0FC94045
:10529000DB0F49C0CDCC4C3D8FC2F53C0000000077
:1052A000B0B52DED028B002800F0B6800446C16039
:1052B00000250574203001F130020121B0EE408A52
:1052C00009F0E2FBB0EE480AE16804F15C0001F18C
:1052D0001002012109F0D8FBB0EE480AE16804F1A0
:1052E000980001F17002012109F0CEFBB0EE480AEE
:1052F000E16804F1D40001F15002012109F0C4FB7E
:10530000B0EE480AE16804F5887001F1B0020121AD
:1053100009F0BAFBB0EE480AE16804F5A67001F1A5
:105320009002012109F0B0FBB0EE480AE16804F5F3
:10533000C47001F1F002012109F0A6FBB0EE480AA9
:10534000E16804F5E27001F1D002012109F09CFB53
:10535000B0EE480AE16804F5007001F59872022188
:1053600009F092FBB0EE480AE16804F50F7001F510
:105370008872022109F088FBB0EE480AE16804F562
:105380001E7001F5B872022109F07EFBB0EE480AEA
:10539000E16804F52D7001F5A872022109F074FB93
:1053A000E168B0EE480A04F54070D1ED640A07F0F8
:1053B000E3FDE168B0EE480A04F54870D1ED640AF7
:1053C00007F0DAFDE06890ED660A90ED672A90ED4F
:1053D000681A90ED693A30EE011A84EDBD0A84ED49
:1053E000BC1A32EE031A84EDBE1A84EDBF2AFCF714
:1053F000F3FAE06807F0F8FFE068083007F0F4FF20
:10540000E06807F049FEE068083007F045FE68B242
:10541000BDEC028BB0BD00BFFF2568B2BDEC028BB6
:10542000B0BD000000000000B0B58AB0B1EE040AC3
:10543000044690EDD11A4FF07E500990E06821EEBD
:10544000000A05A900250695CDE907558DED050A49
:1054500007F09AFEB2EE000A49F69A1094EDD01ABF
:10546000C3F619700490E06821EE000A083069461E
:105470000395CDE901558DED000A07F085FE0AB0D0
:10548000B0BD00000000000010B538B30446C0688D
:1054900008F032F8E06807F04BFE48B100F11C0359
:1054A00004F55D7C806A0ECB8CE80E00C4F88003A6
:1054B000E068083008F020F8E068083007F038FEAF
:1054C00048B100F11C0304F5597C806A0ECB8CE8CE
:1054D0000E00C4F87003002040B210BDFF2040B29F
:1054E00010BD00000000000080B1D1E900C38A684F
:1054F000C0F85423C0E9D3C3D1E903234969C0F8F4
:105500006013C0E9D623002040B27047FF2040B2AC
:1055100070470000000000002DE9F041044602F051
:10552000B3FE0CB3054694F83500022820D140F2B2
:105530000F472668C4F2020740F26F48BE42C4F229
:1055400002081DDC6F20C4F2020086422ADC3F20E4
:10555000C4F20200864241DC1020C4F202008642FE
:1055600063D028205CE000BF0120BDE8F08100BFCF
:10557000802060650120002184F83410BDE8F081AE
:1055800046451BDC40F23F40C4F2020086422DDC5F
:1055900040F21040C4F20200864246D040F2284059
:1055A0003EE000BF9F20C4F20200864228DC70204B
:1055B000C4F20200864238D0882031E040F29F4099
:1055C000C4F20200864223DC40F27040C4F20200C2
:1055D00086422AD040F2884022E000BF4020C4F238
:1055E0000200864221D058201AE000BF40F240401D
:1055F000C4F20200864218D040F2584010E000BFCA
:10560000A020C4F2020086420FD0B82008E000BFFC
:1056100040F2B840C4F20200864206D040F2A040F8
:10562000C4F20200864240F099813146306820F091
:105630001E0041F8140B6FF080000A68464500EA2E
:10564000020008601ADC9F20C4F20200864233DCAC
:105650005720C4F2020086425ADC1020C4F2020035
:10566000864200F097802820C4F20200864200F0B3
:1056700091804020C4F202008AE000BF45F22F4032
:10568000C5F6020086422DDC40F2B740C4F20200AB
:1056900086424BDC40F27040C4F20200864279D070
:1056A00040F28840C4F20200864273D040F2A0402B
:1056B000C4F202006CE000BF40F22740C4F20200D6
:1056C000864243DCA020C4F20200864262D0B820A9
:1056D000C4F2020086425DD040F21040C4F20200E3
:1056E00056E000BF45F26B40C5F6020086423FDC43
:1056F00045F23040C5F6020086424BD045F24440A8
:10570000C5F60200864245D045F258403EE000BF53
:105710005820C4F2020086423CD07020C4F202003D
:10572000864237D08820C4F2020031E040F2B8400F
:10573000C4F2020086422DD045F20840C5F60200B0
:10574000864227D045F21C4020E000BF40F22840AE
:10575000C4F2020086421DD040F24040C4F2020072
:10576000864217D040F25840C4F2020010E000BF59
:1057700045F26C40C5F6020086420BD045F29440DB
:10578000C5F60200864205D045F28040C5F602000B
:10579000864204D1206E016821F480710160306876
:1057A00020F00100306000BF3068C00710D002F068
:1057B0006BFD401B0628F7D320206065032084F88A
:1057C00035000120002184F83410BDE8F08100BFCD
:1057D0002068B84210DC6F21C4F2020188421DDC4F
:1057E0003F21C4F20201884234DC1021C4F20201DC
:1057F000884255D028214FE040451BDC40F23F4114
:10580000C4F2020188422DDC40F21041C4F20201D0
:10581000884245D040F228413EE000BF9F21C4F2BB
:105820000201884228DC7021C4F20201884237D08C
:10583000882131E040F29F41C4F20201884223DC1A
:1058400040F27041C4F20201884229D040F28841FE
:1058500022E000BF4021C4F20201884220D058213A
:105860001AE000BF40F24041C4F20201884217D062
:1058700040F2584110E000BFA021C4F2020188426A
:105880000ED0B82108E000BF40F2B841C4F20201D6
:10589000884205D040F2A041C4F20201884261D1A1
:1058A000D4E9161202F01F023F2303FA02F28A60C3
:1058B000404561DC9F21C4F20201884214DC57217B
:1058C000C4F20201884227DC1021C4F2020188429E
:1058D00000F0A8802821C4F20201884200F0A280D2
:1058E0004021C4F202019BE040F22741C4F20201D0
:1058F000884221DCA021C4F20201884200F092809B
:10590000B821C4F20201884200F08C8040F21041BC
:10591000C4F2020184E000BF5821C4F202018842AF
:1059200000F080807021C4F2020188427AD0882180
:10593000C4F2020174E000BF40F22841C4F2020147
:1059400088426FD040F24041C4F20201884269D0DF
:1059500040F25841C4F2020162E000BF6FF00E0055
:1059600031466AE6D4E9161202F01F02012303FA57
:1059700002F24A6040459DDD45F22F41C5F6020125
:10598000884217DC40F2B741C4F20201884227DCAA
:1059900040F27041C4F20201884243D040F2884193
:1059A000C4F2020188423DD040F2A041C4F202019B
:1059B00036E000BF45F26B41C5F6020188421FDCAC
:1059C00045F23041C5F6020188422BD045F24441F0
:1059D000C5F60201884225D045F258411EE000BFBD
:1059E00040F2B841C4F2020188421BD045F208419E
:1059F000C5F60201884215D045F21C410EE000BFF9
:105A000045F26C41C5F6020188420BD045F2944143
:105A1000C5F60201884205D045F28041C5F6020173
:105A200088420BD1616EA26EE06E4A6030B10168AF
:105A300021F480710160D4E91C014160012084F8E7
:105A400035000020002184F83410BDE8F08100000A
:105A500080B5D8B190F83510022919D140F20F4223
:105A60000168C4F20202914216DC6F23C4F2020301
:105A7000994227DC3F23C4F2020399423EDC102303
:105A8000C4F2020399425FD0282359E0012080BD6F
:105A900080214165012080BD40F26F43C4F20203C2
:105AA00099421BDC40F23F43C4F2020399422DDCD1
:105AB00040F21043C4F20203994245D040F2284319
:105AC0003EE000BF9F23C4F20203994228DC70230A
:105AD000C4F20203994237D0882331E040F29F4359
:105AE000C4F20203994223DC40F27043C4F2020381
:105AF000994229D040F2884322E000BF4023C4F2FB
:105B00000203994220D058231AE000BF40F24043DC
:105B1000C4F20203994217D040F2584310E000BF8C
:105B2000A023C4F2020399420ED0B82308E000BFBC
:105B300040F2B843C4F20203994205D040F2A043B8
:105B4000C4F20203994275D191424FF0040280F8E9
:105B5000352011DC6F20C4F20200814222DC3F209C
:105B6000C4F20200814239DC1020C4F202008142FA
:105B700059D0282054E000BF40F26F40C4F2020028
:105B800081421BDC40F23F40C4F2020081422DDC26
:105B900040F21040C4F20200814244D040F228405A
:105BA0003EE000BF9F20C4F20200814228DC70204A
:105BB000C4F20200814236D0882031E040F29F409A
:105BC000C4F20200814223DC40F27040C4F20200C1
:105BD000814228D040F2884022E000BF4020C4F239
:105BE000020081421FD058201AE000BF40F240401E
:105BF000C4F20200814216D040F2584010E000BFCB
:105C0000A020C4F2020081420DD0B82008E000BFFD
:105C100040F2B840C4F20200814204D040F2A040F9
:105C2000C4F202008142086820F0010008600020F0
:105C300080BD00BF0A6822F00E020A6045F257429A
:105C4000C5F6020291420A6822F001020A600FDCE6
:105C500045F22F42C5F60202914219DC45F2084294
:105C6000C5F60202914229D045F21C4222E000BF53
:105C700045F27F42C5F60202914213DC45F25842DA
:105C8000C5F60202914219D045F26C4212E000BF03
:105C900045F23042C5F6020291420FD045F244422D
:105CA00008E000BF45F29442C5F60202914205D0D9
:105CB00045F28042C5F6020291421AD1D0E9181C81
:105CC000D0E916E30A6822F480720A6003F01F012B
:105CD000012202FA01F1CEF80410816ECCF8041012
:105CE000C16E31B10A6822F480720A60D0E91C12D8
:105CF0004A60012180F83510026D002180F83410CF
:105D00000AB190470021084680BD00000000000055
:105D1000406D7047000000002DE9F04782B000217F
:105D2000019140F208010446C2F2004148F2B51266
:105D3000C1F64E32A56D096840F26F490068C4F2A1
:105D40000209A1FB021848452E68296816DC9F212C
:105D5000C4F2020188422DDC5721C4F202018842BC
:105D600052DC1021C4F2020188427BD02821C4F207
:105D70000201884276D0402170E000BF45F22F42F8
:105D8000C5F60202904229DC40F2B742C4F2020298
:105D9000904245DC40F27041C4F20201884261D079
:105DA00040F28841C4F2020188425BD040F2A04137
:105DB00054E000BF40F22741C4F2020188423FDCB8
:105DC000A021C4F2020188424CD0B821C4F20201E1
:105DD000884247D040F2104140E000BF45F26B429C
:105DE000C5F60202904275DC45F23042C5F6020269
:105DF000904200F0818045F24442C5F60202904292
:105E00007AD045F2584273E05821C4F20201884228
:105E100028D07021C4F20201884223D088211DE0DD
:105E200040F2B842C4F2020290421BD045F208424E
:105E3000C5F6020290425FD045F21C4258E000BF16
:105E400040F22841C4F2020188420BD040F24041A6
:105E5000C4F20201884205D040F25841C4F2020166
:105E6000884261D1E16D082201F01F0140F20F4A22
:105E70008A40C4F2020A324200F0E98050454FF0F5
:105E8000040313DC6F27C4F20207B8426CDC3F271F
:105E9000C4F20207B84200F3A7801027C4F2020739
:105EA000B84200F0C8802827C0E000BF484567DC42
:105EB00040F23F47C4F20207B84200F39D8040F22F
:105EC0001047C4F20207B84200F0B58040F22847FC
:105ED000ACE000BF45F26C42C5F6020290420BD026
:105EE00045F28042C5F60202904205D045F2944246
:105EF000C5F60202904217D10268E36D570703F01E
:105F00001F0315D504279F4017EA010610D011047E
:105F10006F6045D4910603D4016821F0040101604B
:105F2000216C002940F0F68202B0BDE8F08700BF86
:105F300097073DD502279F4017EA010638D0110484
:105F40006F6000F1ED82910609D4016821F00A0129
:105F50000160012084F83500002084F83400E16BF2
:105F6000002940F0D782DFE79F27C4F20207B8423A
:105F70004CDC7027C4F20207B8425CD0882755E099
:105F800040F29F47C4F20207B84247DC40F2704734
:105F9000C4F20207B8424ED040F2884746E000BF44
:105FA000D00300F1C382A16C002940F0B382BBE7AB
:105FB0001207B9D508229A401140B5D0016821F0E6
:105FC0000E010160012000FA03F16960606584F848
:105FD00035000020E16C84F834000029A4D020466C
:105FE000884702B0BDE8F0874027C4F20207B842F4
:105FF00021D058271AE000BF40F24047C4F2020700
:10600000B84218D040F2584710E000BFA027C4F2B1
:106010000207B8420FD0B82708E000BF40F2A047FF
:10602000C4F20207B84206D040F2B847C4F20207F1
:10603000B84218BF082307681F4208D0036823F03E
:1060400004030360AA60626D42F0010262650122EE
:106050008A4032426FD0504510DC6F23C4F20203F5
:1060600098421DDC3F23C4F20203984234DC102323
:10607000C4F20203984256D028234FE048451BDC67
:1060800040F23F43C4F2020398422DDC40F2104339
:10609000C4F20203984246D040F228433EE000BFDB
:1060A0009F23C4F20203984228DC7023C4F2020347
:1060B000984238D0882331E040F29F43C4F2020373
:1060C000984223DC40F27043C4F2020398422AD083
:1060D00040F2884322E000BF4023C4F2020398420A
:1060E00021D058231AE000BF40F24043C4F202031B
:1060F000984218D040F2584310E000BFA023C4F2E9
:10610000020398420FD0B82308E000BF40F2A0433A
:10611000C4F20203984206D040F2B843C4F202032C
:10612000984240F00B8243691B0604D5AA60626D59
:1061300042F00202626504228A4032426FD050452A
:1061400010DC6F23C4F2020398421DDC3F23C4F22B
:106150000203984234DC1023C4F20203984256D062
:1061600028234FE048451BDC40F23F43C4F20203C2
:1061700098422DDC40F21043C4F20203984246D00C
:1061800040F228433EE000BF9F23C4F2020398423E
:1061900028DC7023C4F20203984238D0882331E00F
:1061A00040F29F43C4F20203984223DC40F2704362
:1061B000C4F2020398422AD040F2884322E000BF92
:1061C0004023C4F20203984221D058231AE000BFB2
:1061D00040F24043C4F20203984218D040F25843C0
:1061E00010E000BFA023C4F2020398420FD0B823EE
:1061F00008E000BF40F2A043C4F20203984206D078
:1062000040F2B843C4F20203984240F09F81036811
:106210009B0704D5AA60626D42F0040262651022F9
:1062200002FA01F1314200F0818050454FF008023E
:1062300010DC6F23C4F2020398421DDC3F23C4F23A
:106240000203984234DC1023C4F20203984256D071
:1062500028234FE048451BDC40F23F43C4F20203D1
:1062600098422DDC40F21043C4F20203984246D01B
:1062700040F228433EE000BF9F23C4F2020398424D
:1062800028DC7023C4F20203984238D0882331E01E
:1062900040F29F43C4F20203984223DC40F2704371
:1062A000C4F2020398422AD040F2884322E000BFA1
:1062B0004023C4F20203984221D058231AE000BFC1
:1062C00040F24043C4F20203984218D040F25843CF
:1062D00010E000BFA023C4F2020398420FD0B823FD
:1062E00008E000BF40F2A043C4F20203984206D087
:1062F00040F2B843C4F20203984218BF0422036874
:10630000134213D0A96001684903016808D4C90584
:1063100008D4016821F008010160216C21B905E071
:1063200008034FD4216C09B120468847E06D00F086
:106330001F01202000FA01F2324200F0AB802068F9
:106340001023504510DC6F27C4F20207B8421DDC51
:106350003F27C4F20207B84238DC1027C4F2020714
:10636000B8425AD0282753E048451BDC40F23F474B
:10637000C4F20207B84231DC40F21047C4F202070F
:10638000B8424AD040F2284742E000BF9F27C4F2FB
:106390000207B8422CDC7027C4F20207B8423CD096
:1063A000882735E040F29F47C4F20207B84227DC55
:1063B00040F27047C4F20207B8422ED040F288473C
:1063C00026E000BFA16C0029AED1AFE74027C4F2A0
:1063D0000207B84221D058271AE000BF40F24047D8
:1063E000C4F20207B84218D040F2584710E000BF8C
:1063F000A027C4F20207B8420FD0B82708E000BFB8
:1064000040F2A047C4F20207B84206D040F2B847B3
:10641000C4F20207B84218BF022307681F4239D0EE
:10642000AA6094F83520042A02681BD122F01602D3
:106430000260426922F080024261226C0AB9A26CB9
:106440001AB1026822F0080202603F208840A8606A
:10645000012084F83500216D0020002984F83400E3
:1064600058D161E5510301680CD4C9050ED4016807
:1064700021F010010160012084F83500002084F82B
:10648000340003E0080301D4616C00E0E16B09B162
:1064900020468847606D00283FF446AD606DC00718
:1064A00034D0042084F8350020684FEA982102682F
:1064B00022F001020260019A013201928A421AD846
:1064C0000268D20717D0019A013201928A4212D88B
:1064D0000268D2070FD0019A013201928A420AD88B
:1064E0000268D20707D0019A013201928A4202D88B
:1064F0000268D207DFD10068C0074FF0030008BF71
:10650000012084F83500002084F83400E16C002973
:106510003FF40AAD2046884702B0BDE8F08700BFCF
:10652000D00307D4616C0029F4D1FDE4216C00296B
:10653000F0D1F9E4E16B0029ECD1F5E40268042222
:106540008A4032427FF4FBAD69E600BF026866E62E
:106550002DE9F04381B0044601F096FE002C00F0D6
:10656000128140F26F4805462068C4F20208404597
:1065700016DC9F21C4F2020188422DDC5721C4F2AF
:106580000201884254DC1021C4F20201884200F06A
:106590007E802821C4F20201884278D0402171E037
:1065A00045F22F41C5F60201884229DC40F2B7418D
:1065B000C4F20201884247DC40F27041C4F2020199
:1065C000884264D040F28841C4F2020188425ED021
:1065D00040F2A04156E000BF40F22741C4F2020160
:1065E000884241DCA021C4F2020188424FD0B82188
:1065F000C4F2020188424AD040F2104142E000BF9A
:1066000045F26B41C5F60201884200F3C18045F2B4
:106610003041C5F60201884200F0CD8045F2444188
:10662000C5F60201884200F0C68045F25841BDE03F
:106630005821C4F20201884229D07021C4F202011B
:10664000884224D088211DE040F2B841C4F2020102
:1066500088421CD045F20841C5F60201884200F08C
:10666000AA8045F21C41A1E040F22841C4F2020197
:1066700088420CD040F24041C4F20201884206D068
:1066800040F25841C4F20201884240F09782022150
:1066900084F83510002184F83410016821F00101DC
:1066A00001600168C90708D001F0EEFD401B052814
:1066B00064D820680168C907F6D148F23F0204F1A6
:1066C00008060168CFF610621140D4F818C06CCEED
:1066D0001143D4F824901943E3692943256A0E43F2
:1066E000B9F1040F46EA0C0643EA060343EA050340
:1066F00003D1D4E90B6533432B43666843F480111F
:10670000A6F13F07A6F12905042FA6F1470238BFDD
:106710000B46062DA6F14F0E38BF0B46022A26F077
:10672000030238BF0B46BEF1040F38BF0B46742A74
:1067300008BF0B46B9F1040F0360416921F007015E
:1067400041EA090140F0F480D4E90A53002B41EA00
:10675000050100F0ED80BCF5005F00F0CF80BCF1DA
:10676000000F40F0D780022D00F0D780012D00F0FF
:10677000CB80002D00F0D180DAE000BF20206065E2
:10678000032084F83500012001B0BDE8F08300BF8C
:1067900045F26C41C5F6020188420CD045F28041B9
:1067A000C5F60201884206D045F29441C5F60201C1
:1067B000884240F00382022184F83510002184F8D9
:1067C00034100168A268A2F18003E768B3FA83F38A
:1067D000402A4FEA53134FEA83336FF3101108BF77
:1067E0001023226941EAD70167691943A36941EA85
:1067F000D201E26941EAD70141EAD3014CF6CD4327
:1068000041EAD2014AF6F832CAF2FD72276A02441E
:10681000CCF6CC43A2FB032341EA171101606FF0D1
:10682000030000EA9300E0652046FDF75DFDE16DA1
:10683000012201F01F0102FA01F141602068404588
:1068400040F3858045F22F41C5F60201884217DCEE
:1068500040F2B741C4F20201884229DC40F27041A3
:10686000C4F20201884200F0BC8040F28841C4F2C8
:106870000201884200F0B58040F2A041ACE000BFC8
:1068800045F26B41C5F60201884223DC45F23041F6
:10689000C5F60201884200F0A48045F24441C5F6E5
:1068A0000201884200F09D8045F2584122E000BF7D
:1068B00040F2B841C4F20201884200F0928045F2F1
:1068C0000841C5F60201884200F08B8045F21C4168
:1068D00010E000BF45F26C41C5F60201884200F0AD
:1068E000808045F29441C5F60201884200F079802B
:1068F00045F28041C5F6020170E000BF032D17D8B4
:10690000DFE805F00E0B0E02A3F1C072B2FA82F2BC
:10691000520904E0032D03D30AD1C3F300623AB154
:1069200040206065012084F8350001B0BDE8F083A7
:1069300041612046FDF7D8FCE16D3F2201F01F01C7
:1069400002FA01F18160206840453FF77BAF9F214B
:10695000C4F20201884211DC5721C4F202018842CC
:1069600020DC1021C4F2020188423AD02821C4F26E
:106970000201884235D040212EE000BF40F227417D
:10698000C4F20201884219DCA021C4F2020188424B
:1069900027D0B821C4F20201884222D040F210412F
:1069A0001AE000BF5821C4F20201884219D07021B8
:1069B000C4F20201884214D088210DE040F228413F
:1069C000C4F2020188420CD040F24041C4F20201FC
:1069D000884206D040F25841C4F20201884240F099
:1069E000E58045F2574C45F6FC0EC5F6020CC5F69F
:1069F000020E604512DC45F22F41C5F602018842C5
:106A000020DC45F20841C5F60201884234D045F247
:106A10001C41C5F6020188422ED085E045F27F4137
:106A2000C5F6020188421BDC45F25841C5F6020159
:106A3000884221D045F26C41C5F6020188421BD044
:106A400072E000BF45F23041C5F60201884213D022
:106A500045F24441C5F6020188420DD064E000BF12
:106A600045F29441C5F60201884205D045F28041C5
:106A7000C5F60201884257D16FF007014CF6CD42AE
:106A800051FA80F1CCF6CC42A1FB0212AEF1FC052A
:106A9000AEF17C061309A26803F01F01802A4FF0B3
:106AA000010205EB8305256602FA01F26666A2661D
:106AB00002D10021616000E06168CBB20139072991
:106AC0002B60726016D85E1E082E19D260450EF13A
:106AD000440219DC45F22F41C5F60201884245DC2B
:106AE00045F20841C5F60201884255D045F21C41E5
:106AF0004EE000BF00206067C4E91B0056E000BF05
:106B0000D4E91B02616F4EE045F27F41C5F60201F8
:106B1000884235DC45F25841C5F6020188423BD037
:106B200045F26C4134E000BF6FF00F014AF6AB2232
:106B300051FA80F1CAF6AA22A1FB021240F20F43D9
:106B4000C4F2020308251109984203F1AA060B4674
:106B500088BF05EB121340F60005B042C4F20205EF
:106B600005F1800628BF0B4695E700BF45F230418E
:106B7000C5F6020188420FD045F2444108E000BF4B
:106B800045F28041C5F60201884205D045F29441A4
:106B9000C5F60201884213D101210EEB8300B140FA
:106BA000E066226761670023036051600020606532
:106BB000012184F8351001B0BDE8F0834020DEE506
:106BC00040F60000C4F2020000F1FC0E00F5A072D5
:106BD000E2E7000000000000B0B500283CD0054608
:106BE00090F83400012801D10220B0BD012085F8C1
:106BF000340095F83500012828D1022085F83500A9
:106C0000002068652868046824F0010404602846B0
:106C1000FDF702FC40F20F422868C4F2020240F283
:106C20006F419042C4F2020118DC6F23C4F20203E8
:106C3000984225DC3F23C4F2020398423CDC102337
:106C4000C4F2020398425ED0282357E04FF400605C
:106C50006865002085F834000120B0BD88421BDC47
:106C600040F23F43C4F2020398422DDC40F210434D
:106C7000C4F20203984246D040F228433EE000BFEF
:106C80009F23C4F20203984228DC7023C4F202035B
:106C9000984238D0882331E040F29F43C4F2020387
:106CA000984223DC40F27043C4F2020398422AD097
:106CB00040F2884322E000BF4023C4F2020398421E
:106CC00021D058231AE000BF40F24043C4F202032F
:106CD000984218D040F2584310E000BFA023C4F2FD
:106CE000020398420FD0B82308E000BF40F2B84337
:106CF000C4F20203984206D040F2A043C4F2020359
:106D0000984240F02F8103680B2464F3440303602E
:106D10002B6C1BB1036843F008030360884219DC45
:106D20009F23C4F20203984232DC5723C4F20203C9
:106D3000984259DC1023C4F20203984200F0968076
:106D40002823C4F20203984200F090804023C4F24A
:106D5000020389E045F22F43C5F6020398422DDC79
:106D600040F2B743C4F2020398424BDC40F2704356
:106D7000C4F20203984279D040F28843C4F202037D
:106D8000984273D040F2A043C4F202036CE000BF0B
:106D900040F22743C4F20203984243DCA023C4F22A
:106DA0000203984262D0B823C4F2020398425DD035
:106DB00040F21043C4F2020356E000BF45F26B43B9
:106DC000C5F6020398423FDC45F23043C5F60203A4
:106DD00098424BD045F24443C5F60203984245D051
:106DE00045F258433EE000BF5823C4F202039842E4
:106DF0003CD07023C4F20203984237D08823C4F2F7
:106E0000020331E040F2B843C4F2020398422DD0AD
:106E100045F20843C5F60203984227D045F21C43C9
:106E200020E000BF40F22843C4F2020398421DD084
:106E300040F24043C4F20203984217D040F2584354
:106E4000C4F2020310E000BF45F26C43C5F6020332
:106E500098420BD045F29443C5F60203984205D000
:106E600045F28043C5F60203984274D12B6E1C682C
:106E7000E40303D51C6844F480741C60EB6E1BB102
:106E80001D6845F480751D60904211DC6F21C4F2CD
:106E9000020188421EDC3F21C4F20201884235DC37
:106EA0001021C4F20201884255D0282150E000BFD1
:106EB00088421BDC40F23F41C4F2020188422DDCD3
:106EC00040F21041C4F20201884244D040F228410D
:106ED0003EE000BF9F21C4F20201884228DC7021FD
:106EE000C4F20201884236D0882131E040F29F414D
:106EF000C4F20201884223DC40F27041C4F2020174
:106F0000884228D040F2884122E000BF4021C4F2EC
:106F1000020188421FD058211AE000BF40F24041D0
:106F2000C4F20201884216D040F2584110E000BF7E
:106F3000A021C4F2020188420DD0B82108E000BFB0
:106F400040F2B841C4F20201884204D040F2A041AC
:106F5000C4F202018842016841F001010160002091
:106F6000B0BD00BF0368052464F3430303602B6CCA
:106F7000002B3FF4D3AE036843F00403CDE60000DA
:106F8000B0B5044601F080F940F200010546C2F2B6
:106F90000041621C097818BF0C4400BF01F074F96D
:106FA000401BA042FAD3B0BD90F89830013B012BB2
:106FB0000ED80068836D0B4212D0836D0B408B425C
:106FC00016D1C36D43F00203C3658B0514D418E0DA
:106FD00000F19C01012002220B681A430A607047ED
:106FE000C36D43F00103C3658B0505D409E000BF01
:106FF0000323C3658B0504D5D0F8E0301343C0F8F4
:10700000E0304B0504D5D0F8E4301A43C0F8E42052
:107010004FF6FF72436DC3F6CF720A401A434265C2
:107020008A0F4AF614010020C4F200010B681A43CB
:107030000A607047000000002DE9F04390F8983096
:10704000022B19D10668D6F8C03013F07C5F1DD032
:10705000D6F8C4309B0223D4D6F8C4304D68002D36
:107060000D69C3F3044C8B6824D00C682B43234375
:1070700043F0804E22E000BFD0F89C1041F00801A0
:10708000C0F89C100120BDE8F08300BFD0F89C1030
:1070900041F02001C0F89C100120BDE8F08300BF42
:1070A000D0F89C1041F40071C0F89C100120BDE89C
:1070B000F08300BF0C682B4343EA844E836ED0F804
:1070C0008450D1E907970CFB03F48B6949EA076701
:1070D000D1F81480D1F80C901F4305EB840347EAE4
:1070E000080745F824E047EA09475F60CF6887B1A1
:1070F0004AF6F415083303320024C0F6010500BF38
:10710000171957F8037C1F51CF680434EF5DBC4258
:10711000F6D3012101FA0CF1C6F8D010C0F8941092
:107120000020BDE8F0830000704700000000000070
:1071300080B590F89820013A012A0BD80A68002AF5
:10714000CA680FD00B69072A43EA427E18D18B69BF
:107150001BE000BFD0F89C1041F00201C0F89C1069
:10716000012080BD072A19D10A69D1F81CC0120478
:107170008B6942EA0C221A4342F0605218E000BFC9
:10718000D1F808C04B6943EA8C73006F496800EB83
:10719000C10240F831E00020536080BD8B68D1F817
:1071A00010C09B0743EAC2624B6942EA0C421A4391
:1071B0004968C06E40F82120002080BD000000001A
:1071C00090F898C0BCF1010F0ED19200006842EA1D
:1071D0000111DDF800C041EA430141EA0C01C0F8A9
:1071E00080100020704700BFD0F89C1041F00401CF
:1071F000C0F89C100120704710B34AF200010068EB
:10720000C4F2000188420FD04DF20041C4F20001E7
:1072100088420BD04AF20041C4F20001884218BFF4
:107220007047012003E000BF002000E0022040F290
:107230007871C2F2004101EB4010C06A00B1004712
:1072400070470000000000007047000000000000D0
:10725000B422402908BFA4220068805800F07F00B3
:1072600070470000000000002DE9F04390F898708E
:10727000022F11D1402919D10668D6F8A07017F451
:10728000FE0F2FD0D6F8A4707F0635D0D6F8A470A4
:10729000FF013BD400273CE0D0F89C1041F00801EE
:1072A000C0F89C100120BDE8F08300BF41290FD138
:1072B0000668D6F8B07017F4FE0F13D0D6F8B47085
:1072C0007F0619D0D6F8B470FF012BD400272CE02C
:1072D000076D8F4206D900F17C04456D4FF0000C1C
:1072E0000E462BE0D0F89C1041F02001C0F89C1015
:1072F0000120BDE8F08300BFD0F89C1041F48071FC
:10730000C0F89C100120BDE8F08300BFD6F8A07043
:10731000FF0FD6F8A46000F17404C6F30526F51932
:10732000466C0AE0D6F8B070FF0FD6F8B46000F1F2
:107330007804C6F30526F519C66CAC467543246877
:1073400004EB850E54F8257017F08047576054F809
:10735000257027F0604608BFC7F38A46166054F8C8
:10736000257007F00057976054F8254004F000445A
:107370001461BEF80440D461BEF8064014F00F0456
:10738000D460DEF8044004F480145461DEF8044054
:1073900004F4001494619EF8074004F07F04146222
:1073A000DEF804404FEAD474546229D04AF6F41847
:1073B0000024C0F6010800BF0EEB0406651C377AF6
:1073C0001F55D76818F80770BD423FBF1F19757A5F
:1073D0007D70D5683EBF18F80590A51C4D450FD2AD
:1073E000B57ABD70D56818F80590E51C4D4507D2F3
:1073F000F57A0434FD70D56818F80550AC42DBD33B
:10740000402905D10068C0F8A8C00020BDE8F0837D
:10741000412905D10068C0F8B8C00020BDE8F0835C
:107420001F2909D80068012202FA01F1C0F898105A
:107430000020BDE8F08300BF006801F01F010122B9
:1074400002FA01F1C0F89C100020BDE8F0830000B2
:1074500080B590F89820022A40D10268D2F8F03026
:1074600013F47C1F42D0D2F8F4309B0646D0D2F8F9
:10747000F430D0F88000C3F3042C50F83C3013F003
:1074800080434B6050F83CE02EF0604308BFCEF3E1
:107490008A430B6050F83C3003F000538B6000EBE4
:1074A000CC0350F83C0000F0004008619888C861A7
:1074B000D88800F00F00C860586800F48010486158
:1074C000586800F400108861586800F44000486271
:1074D000D87908620020C2F8F8C080BDD0F89C10AE
:1074E00041F00801C0F89C10012080BDD0F89C102C
:1074F00041F02001C0F89C10012080BDD0F89C1004
:1075000041F48071C0F89C10012080BD0000000093
:107510000068D0F8C40000F03F0070470000000091
:1075200070470000000000002DE9F04F87B00446CE
:107530004AF61000C4F2000001684AF61400C4F2D2
:1075400000000268206802EA010A056DD0F8549034
:10755000076DD0F85480036D0293436D0193036D62
:107560000693436D0593036D0493436D0393436D3D
:10757000066D06EA030B5FEACB530BD54FF480711F
:1075800001654AF610010020C4F20001086020469F
:10759000FFF7C6FF05EA09064AF610095FEA4B50F5
:1075A000C4F200094FEA8A750ED52068D0F8DC10C5
:1075B000D0F8E42011404FF4806202650020C9F841
:1075C0000000204600F078FC08EA070806F4704640
:1075D00055B12068002101650AF00300C9F80000D8
:1075E00020462946FFF7A0FDDDE9011000EA01076A
:1075F00008F00F0546B12068314606650020C9F83D
:107600000000204600F0A8FC07F0F00645B1206815
:10761000294605650020C9F80000204600F0C8FB97
:1076200046B12068314606650020C9F800002046B2
:1076300000F0E6FB5FEA0B5000F1B6805FEA8B508A
:1076400000F1C0805FEA0B3000F1CF805FEACB3001
:1076500000F1D9805FEA4B30DDE9031000EA010553
:1076600009D520684FF4802101650020C9F8000089
:10767000204600F019FC5FEA8B30DDE9051000EAD6
:10768000010005F060710CD522684FF400331365DA
:107690000022C9F80020D4F89C2042F08002C4F8EF
:1076A0009C2000F0715539B1206801650020C9F8AF
:1076B00000002046FFF7C8FD206845B105650021A0
:1076C000C9F80010D4F89C102943C4F89C10A9F5FF
:1076D000016188425ED16068816889075AD0016A79
:1076E000426A036A476A114003EA070202F0300562
:1076F000D0F82080D0F82490026A049211F00F0193
:10770000D0F824B0026A0692426A0592466AD0F81E
:1077100020A003D00162204600F0BAFB08EA090766
:107720002DB1606829460562204600F0B9FB06EAE3
:107730000A0007F4C0754006049800EA0B060AD553
:1077400060684023C16BC26B090C02F03F02036208
:10775000204600F0A1FBDDE9051000EA010706F470
:10776000FC462DB1606829460562204600F08CFB7E
:1077700007F4F02036B161680E62D4F89C103143F2
:10778000C4F89C1030B161680862D4F89C100843BA
:10779000C4F89C00D4F89C00002847D0204607B0CD
:1077A000BDE8F04FFFF728BD20684FF40061016588
:1077B0000020C9F80000204600F0F6FB5FEA8B507D
:1077C0007FF540AF2068D0F8D810D0F8E020114005
:1077D0004FF4007202650020C9F80000204600F056
:1077E00093FB5FEA0B307FF531AF20684FF4002147
:1077F00001650020C9F80000204600F0D5FA5FEAD4
:10780000CB307FF527AF20684FF480310165002031
:10781000C9F80000204600F04BFB5FEA4B30DDE981
:10782000031000EA01053FF51CAF24E707B0BDE8EF
:10783000F08F0000000000002DE9F04F85B0A8B3E4
:107840004AF200080446C4F200080068404531D0FE
:1078500094F89810A9B3816921F01001816100F0BA
:1078600013FD054620688169090705D500F00CFD68
:10787000401B0B28F6D310E0816941F001018161C2
:1078800000F002FD054600BF20688169C90721D1CB
:1078900000F0FAFC401B0B28F6D3D4F89C0040F013
:1078A0000100C4F89C00032084F89800012005B072
:1078B000BDE8F08F08F58071616094F89810002998
:1078C000C9D1002084F89900204600F0B9F9206859
:1078D000C1E700BF816941F002018161217C8269B9
:1078E00022F04002012918BF40328261617C826926
:1078F00022F48042012908BF02F580428261A17C06
:10790000826922F48052012918BF02F580528261F7
:10791000816921F44073D4E902120B4383618369C6
:1079200023F0A4038361036923F010030361AAB168
:10793000022A0FD0012A03D1826942F004020CE02E
:107940008369032A43F080038361036943F01002D3
:10795000026103D1826942F020028261D4E905729A
:10796000E369561E6FF0FF02256A02EB0323B1F5AF
:10797000407F43EA4663A5F1010646EA030640F26A
:107980000003CFF6FF7303EB074746EA0701C16127
:1079900010D1D4E90B65D4E90917013F02EB0622A7
:1079A0006FF00F063A4306EB05173A4303EB01412C
:1079B0001143C160236E2BB1616ED0F8C02011431A
:1079C000C0F8C010E16DCDE90313D9424AF2A031ED
:1079D000C0F6010109D0D0F8C820A36E22F007023A
:1079E00051F823301A43C0F8C820D4F840A0BAF1A7
:1079F000000F09D0D0F8BC20636C22F0070251F8C8
:107A000023301A43C0F8BC20A76C57B1D0F8BC2073
:107A1000E36C22F0700251F8233042EA0312C0F8FE
:107A2000BC20D4F850C0BCF1000F0AD0D0F8BC2064
:107A3000636D22F4E06251F8231042EA0121C0F89C
:107A4000BC10404504D161688A6822F003028A6054
:107A50000021C4F89410C4F89C10012184F89810F7
:107A60004FF6FC72D0F88410D4F83C9021EA02035F
:107A7000656CD4E90D120292019543EA8103C0F8C6
:107A80008430D0F8843023F47F0343EA0243C0F803
:107A900084305318D0F888606FF38F0646EA830667
:107AA000C0F88860D0F8886003EB490326F4FE062E
:107AB00046EA0946C0F88860D0F8A0606FF38F06E8
:107AC00046EA8306C0F8A060D0F8A06005FB0A3340
:107AD00026F4FE0646EA0A46C0F8A060D0F8B06078
:107AE0006FF38F0646EA8306C0F8B060D0F8B06046
:107AF00026F4FE0646EA0746C0F8B060E66CD0F809
:107B0000AC506FF38F0506FB07337E4345EA8305D0
:107B1000C0F8AC50D4F8548008FB0C35D0F8F030E5
:107B20006FF38F0308FB0CFC43EA8503C0F8F030C9
:107B3000D0F8F0E0A36D2EF47C1242EA0342C0F8C4
:107B4000F02005EB4302D0F8C0506FF38F0545EAF3
:107B50008202C0F8C020D0F8C020DDF80CB022F4BA
:107B60007C1242EA0B42C0F8C020019AD0F8C05003
:107B700025F07C5502FB0AFE4AF20002C4F2000224
:107B8000DDF810A002EB8101029A01F5406145EA9F
:107B90000A6501EB8207C0F8C05007EBC902A56E69
:107BA00002EB8E00626700EB86060BFB05F227678F
:107BB00006EB8C07C4E91E060AFB05F007EBC303BE
:107BC00003EB8202C4F884304DF2FC33E16602EB31
:107BD0008000C4F200039842C4F88070C4F8882082
:107BE000C4F8900004D9D4F89C0040F0200058E676
:107BF000814221D20A46002042F8040BD4F890308A
:107C00009A4215D2486001F10802D4F890309A42A5
:107C10003FBF0020886001F10C02D4F8903038BFDB
:107C20009A4205D2C8601031D4F890209142E1D335
:107C300005B0BDE8F08F00BF002005B0BDE8F08FB3
:107C4000B0B586B04DF200420068C4F200020021D7
:107C500090420591CDE90311CDE9011132D04AF2EC
:107C60000041C4F20001884258D04AF20001C4F237
:107C70000001884240F0968040F6DC3144F2E0405A
:107C8000C2F20041C5F602000A68002A02F10102B0
:107C90000A6008D1C16841F48071C160C16801F413
:107CA0008071009100990168152441F0080101607C
:107CB0000068132500F00800009000980320019050
:107CC000092125E040F6DC3144F2E040C2F20041F7
:107CD000C5F602000A68002A02F101020A6008D112
:107CE000C16841F48071C160C16801F48071009184
:107CF00000990168A02441F00801016000689F25F7
:107D000000F008000090052100984FF440500190C9
:107D100040F60040C5F602002BE000BF40F6DC3123
:107D200044F2E040C2F20041C5F602000A68002AAF
:107D300002F101020A6008D1C16841F48071C1609A
:107D4000C16801F48071009100990168162441F026
:107D5000020101600068142500F002000090009804
:107D60006020019040F60040C5F602000921A0F510
:107D70000060059101A9022202920022CDE90322AE
:107D800000F07EF905210022284600F055FB284628
:107D900000F042FB05210022204600F04DFB20466A
:107DA00000F03AFB06B0B0BD7047000000000000D4
:107DB00010B34AF200010068C4F2000188420FD0FB
:107DC0004DF20041C4F2000188420BD04AF200415A
:107DD000C4F20001884218BF7047012003E000BFD1
:107DE000002000E0022040F27871C2F2004101EB75
:107DF0004010C06900B1004770470000000000005B
:107E000010B34AF200010068C4F2000188420FD0AA
:107E10004DF20041C4F2000188420BD04AF2004109
:107E2000C4F20001884218BF7047012003E000BF80
:107E3000002000E0022040F27871C2F2004101EB24
:107E40004010406A00B10047704700000000000089
:107E500090F8981001290DD1022180F8981001683E
:107E60008A6922F001028A610021C0F89C1008464C
:107E7000704700BFD0F89C1041F00401C0F89C107E
:107E80000120704700000000704700000000000063
:107E90007047000000000000704700000000000074
:107EA0007047000000000000704700000000000064
:107EB000704700000000000010B34AF200010068A3
:107EC000C4F2000188420FD04DF20041C4F200011B
:107ED00088420BD04AF20041C4F20001884218BF28
:107EE0007047012003E000BF002000E0022040F2C4
:107EF0007871C2F2004101EB4010806900B1004787
:107F0000704700000000000010B34AF20001006852
:107F1000C4F2000188420FD04DF20041C4F20001CA
:107F200088420BD04AF20041C4F20001884218BFD7
:107F30007047012003E000BF002000E0022040F273
:107F40007871C2F2004101EB4010406900B1004776
:107F5000704700000000000010B34AF20001006802
:107F6000C4F2000188420FD04DF20041C4F200017A
:107F700088420BD04AF20041C4F20001884218BF87
:107F80007047012003E000BF002000E0022040F223
:107F90007871C2F2004101EB4010006900B1004766
:107FA0007047000000000000704700000000000063
:107FB000B0B540F69C350446C007C2F2004502D079
:107FC000286800B18047A00702D5686800B18047E3
:107FD000600702D5A86800B18047200702D5E8688D
:107FE00000B18047E00602D5286900B18047A006AD
:107FF00002D5686900B18047600602D5A86900B162
:108000008047200602D5E86900B18047E00502D527
:10801000286A00B18047A00502D5686A00B1804790
:10802000600502D5A86A00B18047200502D5E86A3C
:1080300000B18047E00402D5286B00B18047A0045E
:1080400002D5686B00B18047600402D5A86B00B10F
:108050008047200406D5E86B002808BFB0BDBDE806
:10806000B0400047B0BD00008821C5F600010A6895
:10807000024208BF70470860FFF79ABF0000000087
:108080002DE9F04F85B00D680290002D00F0E680DC
:1080900002988E4600F126420A2102F1FF7342F255
:1080A0000042C5F60202002490424FEAB32208BF04
:1080B0000921082A4FF0010738BF4FEAB3210026F3
:1080C0004FF000080091CDF80CE00DE0DEF8005014
:1080D00008F1010835FA07F006F1020607F1010779
:1080E00004F1040400F0BA80A7F1010A012000FAAB
:1080F0000AF315EA0309E9D0DEF804B00BF0030532
:108100006A1E012A22D802984FEA4801D0F808C016
:108110000191032101FA06F203992CEA020CD1F82D
:108120000CE00EFA06F1DDF80CE041EA0C0181608A
:1081300041686FEA020CCBF30012994303460198A1
:1081400002FA0AF2114359600CE000BF0320032D2C
:1081500000FA06F0029B6FEA000C304602D130466E
:10816000032526E0D968DEF8082001EA0C018240E8
:10817000022D41EA0201D9601BD102466FF00300D3
:1081800000EA5A010F20194404F01C0300FA03F519
:108190001046D1F820E0039A2EEA0505DDF80CE040
:1081A00012699A40029B2A430A62DEF804B00BF07F
:1081B0000305196805FA00F001EA0C011BF4403FC1
:1081C00040EA010018603FF481AF44F2F44140F20C
:1081D0000845C5F60201C5F600050F23086840F002
:1081E00002000860086800F0020004902AF0030012
:1081F000049904F00C0142598B409A43009B03FA06
:1082000001F1114341514FF0B0452868DEF80410E8
:1082100040EA0902CB0258BF20EA09028B022A6019
:1082200040F20405C5F60005286840EA090258BF77
:1082300020EA09028B032A60D5F8800040EA09028F
:1082400058BF20EA0902C903C5F88020E86F40EA58
:10825000090258BF20EA0902EA6737E705B0BDE81E
:10826000F08F0000000000000069084018BF0120E6
:108270007047000000000000002A08BF0904816167
:1082800070470000000000004CF28830C2F200404D
:10829000006870470000000040F200004CF2883196
:1082A000C2F20040C2F2004100780A68104408603F
:1082B000704700000000000080B5032000F0ECF8DB
:1082C00001F0A6F944F218414AF20443C5F602014E
:1082D000C0F601030A68096801F00F01C2F3032226
:1082E000595C9A5C01F01F0102F01F02D04040F27D
:1082F0000C02C2F2004220FA01F1116040F20801C2
:10830000C2F2004108600F2000F00AF800281CBFEC
:10831000012080BD00F054F8002080BD0000000066
:10832000B0B58AB00F2840D804461C200022214650
:10833000002500F081F81C2000F06EF840F20400E7
:10834000C2F20040046044F2E840C5F60200016851
:1083500041F001010160006801A900F001000290F4
:10836000029802A801F0A0F8079C002C18BF012475
:1083700001F0EEF84DF68361A040C4F21B314FF0DE
:10838000FF32A0FB010141F65C30C2F200404FF029
:108390008043036002EB9141C0E9011540F2E731EF
:1083A000C0E9031502F0C8FD10B101200AB0B0BD4C
:1083B00041F65C30C2F2004002F01EFE0AB0B0BDD1
:1083C00081B044F2F4400022C5F60200016841F099
:1083D0000201016000680F2100F0020000906FF0C0
:1083E0000100009B01B000F027B800000000000071
:1083F000002848BF70474EF2801300F01F0140096B
:10840000CEF20003012202FA01F143F82010BFF37B
:108410004F8FBFF36F8F7047002848BF704700F041
:108420001F01012202FA01F14EF200124009CEF2C0
:10843000000242F82010704770B54EF60C5C4FF009
:10844000FF36CEF2000C00F16045DCF80030C3F3DB
:10845000022E8EF00703042B28BF0423BEF1030471
:1084600006FA03F321EA030100F00F0338BF0024EA
:10847000043BB0F1FF3F634406FA04F003F10C0340
:1084800001FA04F1C8BF05F5644322EA000008437D
:108490000001187070BD00004EF60C514FF6FF033E
:1084A000CEF200010A681A4060F30A2242F08060AE
:1084B00040F0FD7008607047B0B544F60C05C5F695
:1084C000020529684907296806D401F00701081A3E
:1084D00018BF0120B0BD00BF21F00701084328608C
:1084E000FFF7D2FE044600BF55F8080C800407D4FD
:1084F000FFF7CAFE001BB0F57A7FF5D90120B0BDA9
:108500000020B0BD0000000080B500F0F9FF44F28B
:1085100020414AF20442C5F60201C0F60102096890
:10852000C1F30211515C01F01F01C84080BD000081
:1085300080B544F2384EC5F6020E5EF8103C5EF887
:10854000101CC1F3053C5EF80C1CBCF1000FDEF8FA
:10855000042015D0C1F30011C2F3CC02514300EE48
:10856000101A03F003010229B8EE400A0ED089B9AF
:108570005EF8381C890611D49FED361A1CE000BF46
:1085800000218160C0E9001180BD00BF9FED301A5D
:1085900012E000BF9FED2D1A0EE000BF5EF8381C00
:1085A00049F20002C0F2D032C1F3C10122FA01F156
:1085B00001EE101AB8EE411ADEF800109FED263ACF
:1085C0006FF35F2102EE101ADEF80010C1F34621AE
:1085D000B8EE422A00EE032A00EE10CAB7EE003AC7
:1085E000B8EE400A81EE000A32EE031A02EE101ACB
:1085F000B8EE422A20EE010A32EE031A80EE011A8A
:10860000BCEEC11A80ED001ADEF80010C1F306417D
:1086100001EE101AB8EE411A31EE031A80EE011A7B
:10862000BCEEC11A80ED011ADEF80010C1F306613C
:1086300001EE101AB8EE411A31EE031A80EE010A6B
:10864000BCEEC00A10EE101A816080BD0024744A8E
:10865000001BB74B0024744C0000003900000000E0
:1086600080B544F2404EC5F6020E5EF8183C5EF846
:10867000181CC1F3055C5EF8141CBCF1000FDEF899
:10868000042015D0C1F30021C2F3CC02514300EE07
:10869000101A03F003010229B8EE400A0ED089B97E
:1086A0005EF8401C890611D49FED361A1CE000BF0D
:1086B00000218160C0E9001180BD00BF9FED301A2C
:1086C00012E000BF9FED2D1A0EE000BF5EF8401CC7
:1086D00049F20002C0F2D032C1F3C10122FA01F125
:1086E00001EE101AB8EE411ADEF800109FED263A9E
:1086F0006FF35F2102EE101ADEF80010C1F346217D
:10870000B8EE422A00EE032A00EE10CAB7EE003A95
:10871000B8EE400A81EE000A32EE031A02EE101A99
:10872000B8EE422A20EE010A32EE031A80EE011A58
:10873000BCEEC11A80ED001ADEF80010C1F306414C
:1087400001EE101AB8EE411A31EE031A80EE011A4A
:10875000BCEEC11A80ED011ADEF80010C1F306610B
:1087600001EE101AB8EE411A31EE031A80EE010A3A
:10877000BCEEC00A10EE101A816080BD0024744A5D
:10878000001BB74B0024744C0000003900000000AF
:108790002DE9F0470446C07844F22C480007C5F69E
:1087A000020833D5606E4FEA305103290CD8DFE858
:1087B00001F003111D2600BFD8F8001041F400316C
:1087C000C8F800101BE000BF01266078C0070BD07E
:1087D00020E000BF04F10800022106F0FDF9064682
:1087E00060B16078C00715D1354646E004F1280035
:1087F000022106F085FA06460028F2D1606ED8F80C
:10880000241021F440110843C8F8240000266078A1
:10881000C007E9D0A06D04280ED83546DFE800F087
:108820000412181E1E0000BFD8F80000354640F4A0
:108830000030C8F8000011E00125012760784007EA
:108840001FD453E004F10800002106F0C5F904E04C
:1088500004F12800002106F053FA05462F461DB109
:10886000607840070DD441E0D8F82400A16D20F0D5
:10887000070000250843C8F8240037466078400701
:1088800034D5D4F8A4004FEA705005280CD8DFE89E
:1088900000F00311171D1D1DD8F8000040F4003032
:1088A000C8F8000012E000BF01250126607800072B
:1088B00020D455E004F10800002106F08DF904E011
:1088C00004F12800002106F01BFA05462E461DB1D2
:1088D000607800070ED443E0D8F82C00D4F8A41038
:1088E00020F4600000250843C8F82C003E4660785C
:1088F000000735D5D4F8A8004FEA306005280DD818
:10890000DFE800F00412181E1E1E00BFD8F8000099
:1089100040F40030C8F8000012E000BF0125012734
:10892000E078800720D44EE004F10800002106F032
:1089300053F904E004F12800002106F0E1F90546AE
:108940002F461DB1E07880070ED43CE0D8F82C000B
:10895000D4F8A81020F0E06000250843C8F82C00E7
:108960003746E07880072ED5E06C4FEA30100328B8
:108970000ED8DFE800F00903130900BFD8F80000A3
:1089800040F40030C8F800002E467DB912E000BF68
:10899000012501266078C00619D44CE004F10800D6
:1089A000022106F019F905462E461DB16078C00671
:1089B0000DD440E0D8F82000E16C20F03000002514
:1089C0000843C8F820003E466078C00633D5E06D05
:1089D0004FEA303004280DD8DFE800F00412181EEA
:1089E0001E0000BFD8F8000040F40030C8F80000B6
:1089F00012E000BF01250127607880061FD44EE0F9
:108A000004F10800002106F0E7F804E004F1280072
:108A1000002106F075F905462F461DB160788006E5
:108A20000DD43CE0D8F82400E16D20F4E0400025AE
:108A30000843C8F824003746607880062FD5206E9A
:108A40004FEA3040052809D8DFE800F0040E14048E
:108A5000040400BF2E46ADB918E000BF0125012671
:108A6000607840061FD44FE004F10800012106F0B1
:108A7000B3F804E004F12800012106F041F90546AD
:108A80002E461DB1607840060DD43DE0D8F8240094
:108A9000216E20F4E02000250843C8F824003E465B
:108AA0006078400630D5D4F8AC004FEA3070052825
:108AB00008D8DFE800F0030D130303032F46ADB918
:108AC00018E000BF012501276078000620D442E0AD
:108AD00004F10800012106F07FF804E004F1280009
:108AE000012106F00DF905462F461DB160780006FC
:108AF0000ED430E0D8F82C00D4F8AC1020F0E040D0
:108B000000250843C8F82C0037466078000622D5B7
:108B1000E06E58B1B0F1005F0CD0B0F1805F2FD1A2
:108B2000D8F8000040F40030C8F800002E469DB987
:108B300008E000BF04F10800012106F04DF80546E9
:108B40002E464DB9D8F82400E16E20F040500025A3
:108B50000843C8F824003E46E078C00733D0A06C34
:108B6000032813D8DFE800F008021A08D8F800003C
:108B700040F40030C8F80000A946BDB91AE000BFB3
:108B800001250126E078C007E9D11CE001254FF05E
:108B90000109A07840061AD51CE000BF04F10800C6
:108BA000022106F019F80546A9461DB1A078400635
:108BB0000DD50FE0D8F82000A16C20F003000025AF
:108BC0000843C8F82000B146A078400602D44F46BA
:108BD00018E000BFD8F8D40340F48070C8F8D4037C
:108BE000FFF752FB064600BFD8F8D403C00507D4F0
:108BF000FFF74AFB801B6428F6D90325032701E011
:108C00002F468DB12078C00761D0A06F4FEAF000E9
:108C100005283BD8DFE800F004404604040400BF08
:108C2000002D2E4646D149E0D8F84410D4F8B000C3
:108C3000414011F4407F11D0D8F84410D8F84420B6
:108C400042F48032C8F84420D8F8442021F440711E
:108C500022F48032C8F84420C8F84410B0F5807F70
:108C600040F0D082FFF710FB064641F2883A032518
:108C7000032700BFD8F84400800700F1C182FFF746
:108C800003FB801B5045F5D9BCE700BF0125012639
:108C9000207880071FD44CE004F10800012105F082
:108CA0009BFF04E004F12800012106F029F80546A5
:108CB0002E461DB1207880070DD43AE0D8F8280060
:108CC000A16F20F0380000250843C8F828003E4670
:108CD000207880072DD5606F052809D8DFE800F0DF
:108CE000040E1404040400BF2F46ADB918E000BF01
:108CF00001250127207840071FD44DE004F108002A
:108D0000012105F069FF04E004F12800012105F0CC
:108D1000F7FF05462F461DB1207840070DD43BE0F4
:108D2000D8F82800616F20F0070000250843C8F834
:108D300028003746207840072ED5D4F89000052823
:108D400008D8DFE800F0030D130303032E46ADB986
:108D500018E000BF012601252078800620D451E0CC
:108D600004F10800012105F037FF04E004F12800B8
:108D7000012105F0C5FF05462E461DB1207880066D
:108D80000ED43FE0D8F82C00D4F8901020F0070063
:108D900000250843C8F82C003E462078800631D5CF
:108DA000D4F88C004FEA3070052809D8DFE800F0CD
:108DB000040E1404040400BF2F46ADB918E000BF30
:108DC000012701252078400620D451E004F1080055
:108DD000002105F001FF04E004F12800022105F064
:108DE0008FFF05462F461DB1207840060ED43FE088
:108DF000D8F82800D4F88C1020F0E0400025084373
:108E0000C8F8280037462078400631D5D4F89800B5
:108E10004FEAB020052809D8DFE800F0040E14045A
:108E2000040400BF2E46ADB918E000BF012601259D
:108E30002078000620D454E004F10800002105F059
:108E4000CBFE04E004F12800022105F059FF05469D
:108E50002E461DB1207800060ED442E0D8F82C0032
:108E6000D4F8981020F4E05000250843C8F82C00EE
:108E70003E462078000634D5D4F89C004FEA703086
:108E800005280FD8DFE800F004141A04040400BF1A
:108E90002F46E5B12068010727D4C1063ED4000360
:108EA00055D475E00127012520680107F5D51CE0A0
:108EB00004F10800002105F08FFE04E004F1280011
:108EC000022105F01DFF0546002D2F46E2D1D8F8FE
:108ED0002C00D4F89C1020F4604000250843C8F80A
:108EE0002C00374620680107D7D5D4F88010B1F59B
:108EF000805F0AD104F12800022105F001FF00285B
:108F000018BF01272068D4F88010D8F8282022F450
:108F100040521143C8F82810C106C0D5D4F89410A7
:108F2000B1F5807F0AD104F12800022105F0E8FEA6
:108F3000002818BF01272068D4F89410D8F82C20F6
:108F400022F440721143C8F82C10000320D5D4F845
:108F5000A000B0F5003F0FD0B0F5803F06D078BB41
:108F600004F10800002105F037FE04E004F12800B8
:108F7000022105F0C5FE05462E4655B9D8F82C004D
:108F8000D4F8A01020F4403000250843C8F82C0085
:108F90003E46A07840072BD5D4F88400B0F5401F9A
:108FA0000BD0B0F5001F11D0B0F5801F2AD1D8F832
:108FB000000040F40030C8F800002F46CDB90DE0A5
:108FC00001260125A0784007E6D411E004F128002D
:108FD000012105F095FE05462F4655B9D8F8280021
:108FE000D4F8841020F4401000250843C8F8280065
:108FF0003746A078C0070AD13E462168880016D5BA
:1090000033E000BF01270125A078C007F4D0206D10
:10901000B0F5803F10D018BBD8F8000040F4003005
:10902000C8F800002E4685B1216888001DD460680C
:109030008A0326D467E000BF04F10800022105F08E
:10904000CBFD0546002D2E46EED1D8F82000216D2F
:1090500020F4803000250843C8F82000CCE700BF8A
:109060000126012521688800E1D504F128000221AC
:1090700005F046FE002818BF0126D4E900108A0337
:1090800041D5E26F6FF0010303EB3223022B0BD3C8
:109090004FEA322343B1012B40F0AC80D8F80030C6
:1090A00043F40033C8F8003035B3CA022ED48A0224
:1090B00036D44A003ED4B1F1FF3F4BDD090253D410
:1090C000C1075CD1810765D441076ED4010778D40C
:1090D000C10600F18280800607D504F12800022134
:1090E00005F00EFE002818BF0125002D18BF012530
:1090F0002846BDE8F08700BFD8F8283023F4407335
:109100001A43C8F828203546CA02D0D5D8F82420FA
:10911000236F22F000421A43C8F824208A02C8D5DF
:10912000D8F82420A36E22F080721A43C8F82420B5
:109130004A00C0D558F81C2C22F4004248F81C2CD8
:10914000D4F8B42058F81C3C1A4348F81C2CB1F150
:10915000FF3FB3DCD8F82020636D22F040521A4361
:10916000C8F820200902ABD5D8F82810D4F88820F8
:1091700021F440011143C8F82810C107A2D004F11E
:109180000800002105F028FD002818BF054660688A
:10919000810799D504F10800012105F01DFD002883
:1091A00018BF05466068410790D504F10800022108
:1091B00005F012FD002818BF0546606801077FF51D
:1091C00087AF04F12800002105F09AFD002818BFA0
:1091D00005466068C1067FF57EAF04F128000121D5
:1091E00005F08EFD002818BF0546606880067FF5F3
:1091F0007CAF72E70125CA027FF559AF86E700BF51
:10920000D4F8B0004FF6CF7358F81C2CC0F2FF030F
:1092100000F4407122F47C5203EA10136FF31F3004
:10922000B1F5407F08BF1A43002548F81C2CD8F838
:1092300044100843C8F84400FFF7C9BC0000000010
:109240002DE9F04381B0002800F02A8142F20008A5
:109250000446C5F200288946D8F8000000F00F0047
:1092600088420ED2D8F8000020F00F0040EA090032
:10927000C8F80000D8F8000000F00F00484540F0A2
:109280000F81206844F218474107C5F602070AD546
:1092900021693A6802F07002914204D93A6822F0DA
:1092A00070021143396001070AD561697A6802F0DA
:1092B0007002914204D97A6822F0700211437960F9
:1092C000C1060AD5A1697A6802F4E062914204D924
:1092D0007A6822F4E0621143796081060AD5E16977
:1092E000BA6802F07002914204D9BA6822F07002A2
:1092F0001143B96010F002010AD0E2683B6803F044
:109300000F039A4204D93B6823F00F031A433A60D3
:10931000C20746D0386820F47061D4E90102012800
:1093200041EA0201396009D003280DD0022811D189
:1093300057F8181C890340F1B38010E057F8181C47
:10934000C90540F1AD800AE057F8181C890140F1C9
:10935000A78004E057F8181C490740F1A18057F88E
:10936000081C21F00701084347F8080CFEF78CFFA2
:10937000064641F2883500BF57F8080C616800F0D6
:109380003800B0EBC10F09D0FEF77EFF801BA8426A
:10939000F2D9032001B0BDE8F08300BF206800F0DF
:1093A000020151B1E1683A6802F00F02914204D221
:1093B0003A6822F00F0211433960D8F8001001F02A
:1093C0000F0149450DD9D8F8001021F00F0141EAED
:1093D0000901C8F80010D8F8001001F00F01494544
:1093E0005ED141070AD521693A6802F070029142C4
:1093F00004D23A6822F070021143396001070AD59D
:1094000061697A6802F07002914204D27A6822F0AF
:10941000700211437960C1060AD5A1697A6802F425
:10942000E062914204D27A6822F4E06211437960EA
:1094300080060AD5E069B96801F07001884204D25B
:10944000B96821F070010843B86000F0E1F83968AC
:109450004AF204433A68C0F60103C1F3032102F063
:109460000F02595C9A5C01F01F0120FA01F102F031
:109470001F0040F20C0221FA00F0C2F2004210601C
:1094800040F2040040F20802C2F20040C2F2004280
:109490000068116001B0BDE8F043FEF741BF00BFB6
:1094A000012001B0BDE8F0833F22026044F218427F
:1094B000C5F6020252F8083C03F007034360136844
:1094C00003F470638360136803F00F03C3601368D1
:1094D00003F070030361536803F070034361536842
:1094E00003F4E0638361926802F07002C26142F2A9
:1094F0000000C5F20020006800F00F00086070470F
:1095000080B500F085F844F218414AF20443C5F6EC
:109510000201C0F601030A68096801F00F01C2F3F5
:109520000322595C9A5C02F01F0220FA02F201F059
:109530001F0040F20C0122FA00F0C2F20041086064
:1095400040F20801C2F200410A6080BD0000000044
:1095500080B500F05DF844F2184C4AF20441C5F6BB
:10956000020CC0F60101DCF80020DCF8003003F04A
:109570000F03C2F30322CB5C8A5C02F01F02D040CF
:1095800003F01F0240F20C0320FA02F2C2F2004381
:109590001A6040F20803C2F200431860DCF80400CD
:1095A000C0F30210085C00F01F0022FA00F080BD3A
:1095B00080B500F02DF844F2184C4AF20441C5F68B
:1095C000020CC0F60101DCF80020DCF8003003F0EA
:1095D0000F03C2F30322CB5C8A5C02F01F02D0406F
:1095E00003F01F0240F20C0320FA02F2C2F2004321
:1095F0001A6040F20803C2F200431860DCF804006D
:10960000C0F30220085C00F01F0022FA00F080BDC9
:1096100044F20041C5F602010869C0F3C200032804
:1096200010D002282CD088BB0868800649F20000C0
:10963000C0F2D03058BF70470968C1F3C101C840BB
:10964000704700BF8A6A886AC0F3051CC86ABCF10B
:10965000000F4B6B20D0C3F3CC0300F00100584344
:1096600002F00302022A00EE100AB8EE400A15D0FA
:10967000C2B90868800619D49FED281A23E000BFFC
:1096800043F20060C0F26E10704700BF40F6001059
:10969000C0F23D00704700BF002070479FED1E1ACA
:1096A00011E000BF9FED1B1A0DE000BF086849F2F2
:1096B0000002C0F2D032C0F3C10022FA00F001EE85
:1096C000100AB8EE411A086B9FED153A6FF35F2050
:1096D00002EE100A086BC0F34620B8EE422A0130B1
:1096E00000EE032A00EE10CAB7EE003AB8EE400AC8
:1096F00081EE000A32EE031A20EE010A01EE100A92
:10970000B8EE411A80EE010ABCEEC00A10EE100A53
:10971000704700BF0024744A001BB74B0024744CF0
:109720000000003900000000F0B581B0002800F012
:10973000D5800446007844F20046C007C5F602060C
:1097400022D12078800768D5306910F03801B06ADE
:1097500042D0182908BF5FEA80703DD0E0683168C8
:10976000002800F0258121F0190108433060FEF740
:109770008BFD05463068400748D4FEF785FD401B49
:109780000228F7D977E100BF306900F03801B06AEC
:10979000102905D018290BD100F00300022807D1A9
:1097A00030688003CDD560680028CAD196E000BF3C
:1097B0006068002800F03281B0F5A02F00F04681EB
:1097C000B0F5803F00F04681306820F48030306092
:1097D000306820F4802040E130684007E06801D51F
:1097E00000287BD0316821F0190108433060FEF772
:1097F0004BFD05463068400708D4FEF745FD401B89
:1098000002284FF00300F5D901B0F0BD706821695E
:1098100020F0FE4040EA016070602078C00619D553
:10982000306900F03801B06A082906D0182940F0E4
:10983000818000F0030001287CD13068C00502D58A
:10984000E06980284AD1F068216A20F07C5040EA23
:109850000160F0602078000744D42078800655D459
:109860002078400700F17E80656A9DB3306900F082
:109870003800182840F01481012DB16A306B2DD0CA
:1098800001F00302A36A9A4228D1C1F30511E26AEA
:10989000914223D10146226B6FF35F21013A91423D
:1098A0001CD1C0F34622616B01398A4216D1C0F344
:1098B0000642A16B01398A4210D1C0F30660E16B08
:1098C000013988420AD1706BA16CC0F3CC0081428F
:1098D00040F09C81002001B0F0BD00BF012001B02C
:1098E000F0BD00BF60690028706F4FD040F00100EC
:1098F0007067FEF7C9FC0546706F8007ADD4FEF7B0
:10990000C3FC401B0228F7D9B5E000BFA0690028BE
:10991000306871D040F480503060FEF7B5FC0546E9
:10992000306880049CD4FEF7AFFC401B0228F7D9B6
:10993000A1E000BFE0690028306800F09F8040F09F
:1099400080003060FEF7A0FC054600BF3068C0050F
:109950003FF579AFFEF798FC401B02284FF003005B
:10996000F4D951E7D6F8000440F48070C6F800043A
:10997000FEF78AFC054600BFD6F80004C00529D4CE
:10998000FEF782FC401B6428F6D974E020F0010049
:109990007067FEF779FC0546706F80077FF55DAF55
:1099A000FEF772FC401B02284FF00300F4D92BE7AE
:1099B00021F001003060FEF767FC05463068400783
:1099C0007FF52BAFFEF760FC401B02284FF0030031
:1099D000F4D919E7A068002800F08480052800F079
:1099E0009B80012800F09C80306F20F001003067E0
:1099F000306F20F0040096E020F480503060FEF7D5
:109A000043FC0546306880047FF52AAFFEF73CFC36
:109A1000401B02284FF00300F4D9F5E6306820F42B
:109A200080303060306820F480203060FEF72CFCFD
:109A3000054600BF306880037FF583AEFEF724FC47
:109A4000401B64284FF00300F4D9DDE6306840F491
:109A500080203060306840F480303060FEF714FCC5
:109A6000054600BF306880033FF56BAEFEF70CFC87
:109A7000401B6428F6D9032001B0F0BD20F080001F
:109A80003060FEF701FC05463068C0057FF5E2AEA8
:109A9000FEF7FAFB401B02284FF00300F4D9B3E6AF
:109AA000306820F080703060FEF7EEFB022D054636
:109AB0000CD100BF3068800148D5FEF7E5FB401BA4
:109AC00002284FF00300F5D99EE600BF3068800100
:109AD0007FF500AFFEF7D8FB401B02284FF00300D4
:109AE000F4D991E6306F20F001003067306F20F03C
:109AF00004003067FEF7C8FB054641F28837306F37
:109B000080077FF5B1AEFEF7BFFB401BB8424FF0B8
:109B10000300F4D978E600BF306F40F004003067EE
:109B2000306F40F001003067FEF7AEFB054641F2B2
:109B3000883700BF306F80073FF596AEFEF7A4FB75
:109B4000401BB8424FF00300F4D95DE604F128074A
:109B5000B06A40F2F33188438ECF0843591E40EA81
:109B600002104FF47E426FF35F21B06202EB472098
:109B70004FF4FE0280B2E36B0844A16B02EB01419B
:109B80004FF0FE4201F4FE0102EB0362084402F0D2
:109B9000FE4108443063F06A4FF6F87120F001008E
:109BA000F062706BA26C884340EAC2007063F06A96
:109BB000216C20F00C000843F062F06A616C20F028
:109BC00002000843F062F06A40F48030F062F06A0C
:109BD00040F40030F062F06A40F48020F062F06AF5
:109BE00040F00100F062306840F080703060FEF7B5
:109BF0004BFB0446306880013FF56CAEFEF744FB3A
:109C0000001B02284FF00300F4D9FDE5F06A20F0B4
:109C10000100F062FEF738FB0546FEF735FBA8426F
:109C2000FBD0706B4FF6F871A26C884340EAC2001B
:109C30007063F06A40F00100F062002001B0F0BDF6
:109C400041F200410068C5F600010322884243F654
:109C50000001C4F2000108BF0122401A18BF1046DB
:109C6000032808BF704740F66041C2F2004101EB93
:109C70004010806900B100477047000000000000FC
:109C80002DE9F04381B00446066830697169D6F861
:109C9000089094F8818002070CD511F4006209D075
:109CA000B06940F40060B061204601B0BDE8F04307
:109CB00000F0DEBD01EA000505F06407042F05D1C0
:109CC000616F20468847216F2046884705F0450090
:109CD000012807D1216F2046884705F02600022879
:109CE00004D00BE005F02600022805D1616F204664
:109CF00001B0BDE8F0430847042F03D101B0BDE82F
:109D0000F08300BF280715D415F4587FF6D015F05E
:109D1000400065D1A80570D4E80505F020007CD48A
:109D2000002840F08880D4F88400002840F0938018
:109D3000E4E700BF2068816941F008018161816921
:109D400041F010018161816941F400618161016923
:109D500021F008010161806810F4404F27D02046AF
:109D600006F072FC012084F88100D4F884000028F9
:109D700040F0AB80B8F1030F00F0AE80B8F1040FF3
:109D800000F0B080B8F1050FB8D1204601B0BDE8B1
:109D9000F04301F029B800BF2068616E006B41F804
:109DA000040B6166B4F86A000138A4F86A00B4F8DC
:109DB0006A000028D3D0E0681028EDD2082805D327
:109DC000308E616E21F8020BEBE700BF206890F83F
:109DD0003000616E0870606E01306066E2E700BFBF
:109DE0002068D4F8841041F00401C4F8841081691B
:109DF00041F040018161A8058ED52068D4F8841017
:109E000041F00101C4F88410816941F4007181615D
:109E1000E80505F020007FF583AF2168D4F88420A1
:109E200042F00802C4F884208A6942F480728A6190
:109E300000283FF478AF2068D4F8841041F0800106
:109E4000C4F88410816941F020018161D4F8840054
:109E500000283FF453AF206809F4404240F26B33CE
:109E6000B2F5404F016821F001010160016921EA6A
:109E70000301016126D1816840F2197521F4404146
:109E80008160E06FC0F6010548B10565FBF7E0FDB4
:109E900028B1D4F8840040F04000C4F88400A06FDA
:109EA00000283FF42BAF0565FBF7D2FD00283FF4F7
:109EB00025AFD4F8840040F04000C4F8840001B01D
:109EC000BDE8F083012084F88100204601B0BDE8A0
:109ED000F043FFF7B5BE00BF204601B0BDE8F04338
:109EE00000F042BF204601B0BDE8F04300F080BC66
:109EF0002DE9F047002858D043F6000304460068D7
:109F0000C4F2000343F2000E43F6004C9842C4F240
:109F1000010EC4F2000C4FF00001A16203D06045B5
:109F200018BF70453ED1E16B0122E568984202EB13
:109F3000511105F108024FEAD20202FB01F118BFEC
:109F4000704525D1102930D894F8811031B90020FE
:109F500084F88000204600F09FF82068022184F8F1
:109F60008110016821F0010101608168D4F8188036
:109F7000B8F1806F01F4F81ED4F804A020D1BAF132
:109F8000000F15D0BAF5800F1AD1A36B03BB13E0F5
:109F9000604518BF082908D8704518BF6045D1D062
:109FA000D2E700BFE1680F29BDD90120BDE8F087E5
:109FB000A36BB3F1805F06D1036843F48053036061
:109FC0005FEA4A2304D4D4F80C904FF0010C0FE060
:109FD000D4F80C90B9F1070F08D3056825F4807CFC
:109FE000256D45EA0C054FF0000C04E04FF0000C25
:109FF000056825F480750560BAF1000FE769A26A6B
:10A0000047EA0E07E36B42EA0702A56842EA030249
:10A010002669676942EA090282604AEA0803626BBC
:10A02000616A42EA0302A36B41EA020141EA0301C9
:10A03000226A41EA0601E36C41EA070141EA0201B2
:10A04000A26C41EA0301A36D41EA050141EA020164
:10A0500041EA0301C16009D18168012262F3CC2188
:10A0600081608168022262F34A218160016DBCF146
:10A07000000F21F00101016505D1C168626D21F079
:10A0800000411143C1600020C4F88400012184F81C
:10A090008110BDE8F08700002DE9F04FB5B004460F
:10A0A00002A8B8210025CDE93355CDE931553095C9
:10A0B000F6F76FFB41F200412068C5F600018842C7
:10A0C00000F09A8043F60001C4F20001884240F09B
:10A0D000C3804FF48050029002A800260396199680
:10A0E000FEF756FB08B1FAF78BFC44F2E04000277C
:10A0F000C5F60200C5F6020730AD40F210088168CF
:10A100004FF0020941F4804181608168C4F2020885
:10A1100001F4804101910199016841F0040101605D
:10A1200001684FF0030A01F00401019101990168EF
:10A1300041F0020101600068294600F00200019030
:10A1400001980620309007F50060CDF8C4904FF0DC
:10A15000050B3296CDF8CCA0CDF8D0B0FDF790FF2E
:10A160004FF400502946CDE9300932A880E8400C70
:10A1700007F58060FDF784FF41F2C8552720C2F241
:10A1800000454FF48067C5E901062846C5F8008000
:10A19000EE60C5E90476C5E90666C5E90866FCF720
:10A1A000D7F908B1FAF72CFCE56708F11800AC63A1
:10A1B00041F24065C2F200452860282068604020D6
:10A1C000A8600020C5E90307C5E90500C5E9070047
:10A1D00068622846FCF7BCF908B1FAF711FC2420A4
:10A1E00005210022A567AC63FEF726F92420FEF7BF
:10A1F00013F935B0BDE8F08F4FF48040029002A80B
:10A2000003952D95FEF7C4FA08B1FAF7F9FB44F26D
:10A21000E040C5F60200416941F020014161416919
:10A2200001F0200101910199016841F001010160F3
:10A23000006830A900F0010001900198A020309042
:10A24000022031900020CDE9320008203490002017
:10A25000C5F60200FDF714FF35B0BDE8F08F000031
:10A260002DE9F04F81B0994617460E460446D0F8C6
:10A2700000A0C56BFEF708F894F8811001290DD1F4
:10A2800080460120002E18BF002F03D101B0BDE889
:10A29000F08F00BF94F88000012803D1022001B0A4
:10A2A000BDE8F08FA346012084F88000042084F8E4
:10A2B00081000020C4F884004BF8646F2646A4F89F
:10A2C000687026F86A7FE065A4F86000A4F8620070
:10A2D000A168B1F5C02FC4E91C00206804D1016851
:10A2E00021F40061016004E0C168022262F352417E
:10A2F000C16041684FF6FF72914339444160016883
:10A3000041F0010101606168B1F5800F4FF001017A
:10A3100003D1026842F400720260E36801EB551158
:10A32000102B4BD33288002A00F085818DB219F1B1
:10A33000010225D041694269D20704D1328809045B
:10A340000CD5AA420AD2016BDBF800000160043090
:10A35000CBF8000030880138308006E0FDF794FF2C
:10A36000A0EB0800484580F0C7803088002800F046
:10A370006281206841694269D207DFD0E3E700BF0C
:10A3800041694269D20704D1328809040ED5AA4234
:10A390000CD2006BDBF8001041F8040BCBF8001076
:10A3A000308801383080308830B944E1FDF76CFFE7
:10A3B0003088002800F03F812068E1E73288072BD1
:10A3C00044D9002A00F0378119F1010200F0A88079
:10A3D0008FB24FF6FF72551E41694069C00716D112
:10A3E00030880A040ED5B8420CD2BAF83010DBF827
:10A3F000000020F8041BBAF8301020F8021C29468F
:10A400000DE000BF3088890418D5012816D1BAF8AC
:10A410003010DBF8000020F8021B4FF6FF71CBF87C
:10A4200000003088084430803088002800F0038124
:10A43000206841694069C007D2D0E8E7FDF724FFF2
:10A44000A0EB08004845EFD356E000BF002A00F01B
:10A45000F28019F1010200F09F808FB24FF6FF7277
:10A46000A2F1030A41694269D20725D132880B045F
:10A470001CD5BA421AD290F83000616E087020687C
:10A48000616E4A1C626690F8300048702068616E08
:10A490004A1C626690F8300048702068616E4A1C61
:10A4A000626690F83000487050460CE0328811F433
:10A4B000C04F1BD0032A19D890F83000DBF80010E9
:10A4C00008704FF6FF70DBF800100131CBF8001078
:10A4D0003188084430803088002800F0AC80206843
:10A4E00041694269D207C1D0E6E700BFFDF7CCFE63
:10A4F000A0EB08004845EED3204606F0A5F8D4F8B6
:10A50000840040F48070C4F88400012084F8810045
:10A51000002084F88000032001B0BDE8F08F00BF68
:10A520008DB241694069C0071BD130880A0413D538
:10A53000A84211D2BAF83000DBF8001021F8040B61
:10A54000BAF83000CBF8001021F8020C308802383D
:10A550003080308898B96EE03088890416D501289B
:10A5600014D1BAF83000DBF8001021F8020BCBF858
:10A570000010308801383080308800285BD0206897
:10A5800041694069C007D0D0EBE700BFFDF77CFE12
:10A5900030880028F3D14EE08FB241694269D2077A
:10A5A0002ED132880B0425D5BA4223D290F8300040
:10A5B000616E08702068616E4A1C626690F8300017
:10A5C00048702068616E4A1C626690F830004870DE
:10A5D0002068616E4A1C626690F830004870606EB8
:10A5E00001306066B4F86A000438A4F86A00308864
:10A5F000A8B920E0328811F4C04F17D0032A15D82B
:10A6000090F83000DBF800100870DBF80000013033
:10A61000CBF80000308801383080308858B120688D
:10A6200041694269D207BCD0EAE700BFFDF72CFEC2
:10A6300030880028F3D1204606F006F8012084F87F
:10A640008100002084F88000D4F88400002818BF1E
:10A65000012001B0BDE8F08F70B5044690F881008C
:10A6600001280BD115460A4604F180060120002975
:10A6700018BF002D08D10021317070BD04F1800693
:10A6800002200021317070BD3078012802D10220F3
:10A6900070BD00BF012084F88000042084F8810090
:10A6A0000020C4F884006266A4F86850A4F86A50D8
:10A6B000C4E91C00A4F86000A4F86200A068B0F52A
:10A6C000C02F21681AD1086820F400600860E06893
:10A6D00010281BD2082829D3E06F8069B0F5005FED
:10A6E00018BFB0F5804F1DD1886820F48040886085
:10A6F000E06F8369B3F5804F24D02FE0C868022350
:10A7000063F35240C860E0681028E3D3E06F8069CB
:10A71000B0F5804F06D1886820F480408860E06FF3
:10A720001CE000BF01200021317070BD886820F45A
:10A7300080408860E06F8369B3F5804F08D0B3F53F
:10A74000005F0BD1B4F86A3001335B0804E000BF4E
:10A75000B4F86A3003339B08A4F86A3040F271738E
:10A7600040F2617CC0F60103C0F6010CC0E90F3C69
:10A7700040F231733031C0F60103C3640023036536
:10A78000B4F86A30FCF728FA60B1D4F8840040F0DD
:10A790001000C4F88400012084F881000021317089
:10A7A00070BD00BFE16FD4E90002C9694FF6FF74C4
:10A7B0004368B1F5807F23EA040318BF2B44B2F548
:10A7C000800F4360816841F480418160016941F4F8
:10A7D00050710161016841F00101016003D101681C
:10A7E00041F40071016000200021317070BD000053
:10A7F00041F200410068C5F600010322884243F699
:10A800000001C4F2000108BF0122401A18BF10461F
:10A81000032808BF704740F66041C2F2004101EBD7
:10A820004010406800B10047704700000000000081
:10A8300041F200410068C5F600010322884243F658
:10A840000001C4F2000108BF0122401A18BF1046DF
:10A85000032808BF704740F66041C2F2004101EB97
:10A860004010006900B10047704700000000000080
:10A8700070470000000000002DE9F04381B01D4644
:10A8800017460E460446D0F80090FDF7FDFC94F8FC
:10A89000811001290CD180460120002E18BF002F05
:10A8A00002D101B0BDE8F08394F88000012803D103
:10A8B000022001B0BDE8F083012184F8801003205C
:10A8C00084F881000020C4F88400E665A4F8607074
:10A8D000A4F862706066A4F86800A4F86A00A26830
:10A8E0002067B2F5C02F6067206805D10168034674
:10A8F00041F4006205E000BF034653F80C2F61F3FA
:10A9000052421A604FF6FF724168914339444160E8
:10A91000016841F0010101606168B1F5800F03D168
:10A92000016841F400710160E268102A3CD3B4F878
:10A930006210002900F01A81691C1ED04169890744
:10A9400006D4FDF7A1FCA0EB0800A8420AD339E128
:10A95000E16D51F8042B0262E165B4F86200013840
:10A96000A4F86200B4F86200002800F0FF802068BC
:10A9700041698907E5D5EBE720684169890703D478
:10A98000FDF782FC0AE000BFE16D51F8042B026282
:10A99000E165B4F862000138A4F86200B4F862001E
:10A9A0000028E9D1E2E000BFB4F86210072A5DD9BF
:10A9B000002900F0DB80691C31D04FF6FE714E1C7F
:10A9C0004169890706D4FDF75FFCA0EB0800A842A7
:10A9D0001AD3F7E0B4F86210022909D3E16B39B158
:10A9E000E16D51F8042B0262E1654FF6FE7006E05E
:10A9F000E06D30F8021BA9F82010E0653046B4F88D
:10AA000062100844A4F86200B4F86200002800F064
:10AA1000AD80206841698907DCD4D4E720684169AA
:10AA2000890703D4FDF730FC1BE000BFB4F86210C7
:10AA300002290BD3E16B49B1E16D51F8042B02629D
:10AA4000E165B4F86200023809E000BFE06D30F85B
:10AA5000021BA9F82010E065B4F862000138A4F8E0
:10AA60006200B4F862000028D8D17FE0002900F02D
:10AA70007D80691C43D04FF6FE718E1E4F1C4169CC
:10AA8000890707D4FDF700FCA0EB0800A8422CD3EF
:10AA900098E000BFB4F86210042909D3E16B4029A3
:10AAA00006D9E16D51F8042B0262E165304617E0EA
:10AAB000B4F8621002290BD3E16B49B1E06D30F8B4
:10AAC000021BA9F82010E0654FF6FE7008E000BFF9
:10AAD000E16D097880F82010E06D0130E0653846BE
:10AAE000B4F862100844A4F86200B4F862000028C8
:10AAF0003CD0206841698907CCD4C3E7206841690C
:10AB0000890703D4FDF7C0FB2CE000BFB4F8621046
:10AB100004290BD3E16B412908D3E16D51F8042BD3
:10AB20000262E165B4F86200043819E0B4F862101A
:10AB300002290BD3E16B49B1E06D30F8021BA9F893
:10AB40002010E065B4F86200023809E0E16D097890
:10AB500080F82010E06D0130E065B4F86200013843
:10AB6000A4F86200B4F862000028C7D1681C13D0B2
:10AB700020684069000713D4FDF786FBA0EB0800AE
:10AB8000A842F5D3D4F8840040F02000C4F8840033
:10AB900006E000BFFDF778FB206840690007F9D5A3
:10ABA000204605F051FD012084F88100002084F842
:10ABB0008000D4F88400002818BF012001B0BDE84F
:10ABC000F08300BF204605F03FFDD4F8840040F438
:10ABD0008070C4F88400012084F88100002084F88B
:10ABE0008000032001B0BDE8F083000000000000F9
:10ABF000F0B581B0044690F8810001280CD10029FD
:10AC00004FF0010000F0AE801546002A00F0AA8047
:10AC100094F88000012803D1022001B0F0BD00BFEC
:10AC2000012084F88000032284F881200022C4F8E7
:10AC30008420E165A4F86050A4F862506266C4E91B
:10AC40001C22A4F86820A4F86A20A268B2F5C02FDC
:10AC5000266813D13068324640F400631360E2681E
:10AC6000102A14D2A06F082A82691BD3B2F5005FA4
:10AC70002AD0B2F5804F1BD00EE000BF324652F80A
:10AC80000C3F60F352431360E268102AEAD3A06FCE
:10AC90008269B2F5804F17D0002084F8800001202F
:10ACA00001B0F0BDB2F5804F08D0B2F5005F0BD116
:10ACB000B4F862200132520804E000BFB4F8622008
:10ACC00003329208A4F8622040F2997240F269734C
:10ACD000C0F60102C0F60103C0E90F2340F2317251
:10ACE0000027C0F60102C2640765B26822F4004280
:10ACF000B260B4F8623006F12002FBF76DFF68B174
:10AD0000D4F8840040F01000C4F88400012084F8D6
:10AD1000810084F8807001B0F0BD00BFA16F4FF6D4
:10AD2000FF77D4E90002C9694368B1F5807F23EA5F
:10AD3000070318BF2B44B2F5800F4360816841F4CC
:10AD400000418160016941F448710161016841F08D
:10AD50000101016003D1016841F40071016000202C
:10AD600084F8800001B0F0BD41F200410068C5F6F2
:10AD700000010322884243F60001C4F2000108BF2B
:10AD80000122401A18BF1046032808BF704740F63A
:10AD900060414001C2F20041085808B1004700BFBD
:10ADA000704700000000000041F200410068C5F655
:10ADB00000010322884243F60001C4F2000108BFEB
:10ADC0000122401A18BF1046032808BF704740F6FA
:10ADD0006041C2F2004101EB4010C06800B1004781
:10ADE000704700000000000041F200410068C5F615
:10ADF00000010322884243F60001C4F2000108BFAB
:10AE00000122401A18BF1046032808BF704740F6B9
:10AE10006041C2F2004101EB4010806800B1004780
:10AE2000704700000000000040F20442C5F6000236
:10AE3000136823EA00000843106070470000000018
:10AE40007047000000000000704700000000000094
:10AE50007047000000000000B0B590F83C20012AC7
:10AE60004FF0020263D080F83D2040F2004C0268AF
:10AE7000C4F2010C42F4806363455368D2F808E0E1
:10AE800002BF23F470034C6823434DF6FF740D6832
:10AE9000C4F2000423F07003A24243EA05035360A6
:10AEA00014DC40F2FF73C4F200039A4222DD40F644
:10AEB0000003C4F200039A422ED040F60043C4F2CD
:10AEC00000039A4228D041F6000321E04FF6FF73B9
:10AED000C4F200039A4213DD0023C4F201039A4234
:10AEE0001AD044F20003C4F201039A4214D062451E
:10AEF00012D016E0B2F1804F0ED040F2004307E0CE
:10AF00004EF20003C4F200039A4205D04EF2004311
:10AF1000C4F200039A4204D12EF0800389681943D9
:10AF200091600022012180F83D1080F83C201046FD
:10AF3000B0BD00000000000060B310B5044690F8FA
:10AF40003D0028B9002084F83C00204600F024F899
:10AF5000022084F83D002068211D06F031FF012009
:10AF600084F8480084F83E0084F83F0084F84000EC
:10AF700084F8410084F8420084F8430084F84400D7
:10AF800084F8450084F8460084F8470084F83D00C2
:10AF9000002010BD0120704782B041F6000100681A
:10AFA000C4F20001884215D040F20041C4F2000111
:10AFB00088421CD144F2E840C5F60200016841F025
:10AFC00002010160006800F002000190019802B0E7
:10AFD000704700BF44F2E840C5F60200016841F046
:10AFE00040010160006800F040000090009802B04D
:10AFF000704700000000000090F83D10012923D1A7
:10B00000022180F83D1001684DF6FF70C4F2000087
:10B010008142C86840F00100C86017DC40F2FF7050
:10B02000C4F20000814227DD40F60000C4F20000B7
:10B03000814233D040F60040C4F2000081422DD05E
:10B0400041F6000026E000BF012070474FF6FF7078
:10B05000C4F20000814215DD0020C4F201008142EB
:10B060001CD044F20000C4F20100814216D040F22C
:10B070000040C4F201000FE0B1F1804F0ED040F269
:10B08000004007E04EF20000C4F20000814205D00B
:10B090004EF20040C4F2000081420BD107228868C2
:10B0A000C0F2010202400020062A18BFB2F5803F1C
:10B0B00000D17047086840F0010008600020704728
:10B0C00080B590F83C20012A4FF0020200F0A780E2
:10B0D00080F83D208822D0F800C0CFF6CE72DCF890
:10B0E00008301A40CCF808200B686F2B0EDDB3F146
:10B0F000101F37DAB3F5005F46DA702B00F092804C
:10B10000B3F5805F00F08480D6E000BF2F2B33DDE5
:10B110004F2B3FDC302B6FD0402B40F0CD80D1F84F
:10B1200004E0C968DCF82030DCF8202022F00102BD
:10B13000CCF82020DCF8182022F0F00242EA0111BD
:10B1400023F00A02CCF8181042EA0E01CCF82010C5
:10B150004FF68872DCF80810CFF6CF7211404731F5
:10B1600054E000BF2F21C0F210018B423ADCB3F152
:10B17000101F41D020213BE0002B18BF102B3BD0EB
:10B18000202B39D098E000BF60D0B3F5801F33D0BA
:10B1900092E000BF502B6DD0602B40F08D80D1F835
:10B1A00004E0C968DCF82030DCF8202022F010022E
:10B1B000CCF82020DCF8182022F4704242EA013159
:10B1C00023F0A002CCF8181042EA0E11CCF820109F
:10B1D0004FF68872DCF80810CFF6CF721140673155
:10B1E00014E000BF3021C0F210018B4204D0402196
:10B1F000C0F210018B425FD14FF68872DCF8081064
:10B20000CFF6CF721140194341F00701CCF8081076
:10B210000022012180F83D10002180F83C101046EA
:10B2200080BD00BFD1E901E3C968DCF8082043EA2A
:10B230000E0322F47F4243EA01211143CCF80810A7
:10B24000DCF8081041F07701E0E700BFD1E901E345
:10B25000C968DCF8082043EA0E0322F47F4243EA7F
:10B2600001211143CCF80810DCF8081041F48041AA
:10B27000CCE700BFD1F804E0C968DCF82030DCF886
:10B28000202022F00102CCF82020DCF8182022F047
:10B29000F00242EA011123F00A02CCF8181042EA47
:10B2A0000E01CCF820104FF68872DCF80810CFF6AB
:10B2B000CF7211405731A9E70122AAE70000000030
:10B2C0007047000000000000F0B581B0044600683F
:10B2D000C768066906EA0705A9071BD468072FD4C3
:10B2E000280745D4E8065BD4E80772D117F0800739
:10B2F00018BF16F402507AD1002F18BF16F48070D0
:10B3000040F08280680600F18980A80600F19080F4
:10B3100001B0F0BD6FF00201016101212177806968
:10B32000800703D02046FFF7CBFF05E0204600F062
:10B330008BF8204600F020FB002020776807CFD54F
:10B3400020686FF00401016102212177806910F407
:10B35000407F03D02046FFF7B3FF05E0204600F012
:10B3600073F8204600F008FB002020772807B9D5A5
:10B3700020686FF00801016104212177C06980070E
:10B3800004D02046FFF79CFF06E000BF204600F0F7
:10B390005BF8204600F0F0FA00202077E806A3D5FD
:10B3A00020686FF01001016108212177C06910F455
:10B3B000407F03D02046FFF783FF05E0204600F0E2
:10B3C00043F8204600F0D8FA00202077E8073FF441
:10B3D0008DAF20686FF001010161204600F02CFC68
:10B3E00017F0800718BF16F402503FF485AF2068AD
:10B3F0006FF4025101612046FFF726FD002F18BFB0
:10B4000016F480703FF47EAF20686FF480710161A4
:10B410002046FFF715FD68067FF577AF20686FF0CF
:10B4200040010161204600F00FFCA8067FF570AFD7
:10B4300020686FF020010161204601B0BDE8F040B6
:10B44000FFF706BD0000000070470000000000008C
:10B450002DE9F04190F83C30012B03D10220BDE8EA
:10B46000F08100BF4FEAB202052A31D8DFE812F0BE
:10B47000060038007600B400DA000001036843F6E5
:10B48000FF76C4F201061C6AB3421A6A24F0020471
:10B4900022F001021A621A46D3F804E052F818CFDB
:10B4A0008D6844EA0504D1F8008040F3078144F236
:10B4B0000007C4F20107BB4200F00B8144F600070D
:10B4C000C4F20107BB4200F0048144F20047FCE0F3
:10B4D0000121002280F83C200846BDE8F08100BF31
:10B4E000036840F2004E43F48067C4F2010E1C6A08
:10B4F00077451A6A24F0200422F010021A621A46D4
:10B500005D6852F818CF8E6844EA061407D1CE68F9
:10B510006FF0400724F0C00407EA0616344343F6F0
:10B52000FF76D1F80080C4F20106B34240F3EC800C
:10B5300044F20007C4F20107BB4200F0EC8044F67D
:10B540000007C4F20107BB4200F0E58044F2004767
:10B55000C4F20107BB4200F0DE80E4E0036840F281
:10B56000004E43F48067C4F2010E1C6A77451A6AE4
:10B5700024F4007422F480721A621A465D6852F84C
:10B580001CCF8E6844EA062407D1CE6840F2FF47FC
:10B59000360224F44064BE43344343F6FF76D1F8C8
:10B5A0000080C4F20106B34240F3D48044F20007A5
:10B5B000C4F20107BB4200F0D48044F60007C4F295
:10B5C0000107BB4200F0CD8044F20047C4F20107FE
:10B5D000BB4200F0C680CCE0036843F6FF77C4F2BC
:10B5E0000107D3F820C0BB421A6A22F480521A62C3
:10B5F0001A465C6852F81C6F0D68D1F808E040F3F9
:10B60000CF8044F20007C4F20107BB4200F0D380B0
:10B6100044F60007C4F20107BB4200F0CC8044F2BC
:10B620000047C4E0036843F6FF77C4F20107D3F88C
:10B6300020C0BB421A6A22F480321A621A465C6841
:10B6400052F8546F0D68D1F808E040F3D38044F20B
:10B650000007C4F20107BB4200F0D78044F60007A0
:10B66000C4F20107BB4200F0D08044F20047C8E0BA
:10B67000036843F6FF77C4F20107D3F820C0BB424A
:10B680001A6A22F480121A621A465C6852F8546FE1
:10B690000D68D1F808E040F3D98044F20007C4F205
:10B6A0000107BB4200F0DD8044F60007C4F2010749
:10B6B000BB4200F0D68044F20047CEE00027C4F23F
:10B6C0000107BB4205D040F20047C4F20107BB426C
:10B6D00005D1CF6824F00C0427F004073C43B342A3
:10B6E00040F3E28044F20006C4F20106B34200F0E7
:10B6F000E68044F60006C4F20106B34200F0DF80A3
:10B7000044F20046D7E000BF0027C4F20107BB4265
:10B7100001D0734507D14F6925F440658E6945EA2C
:10B72000870747EA860548F6FF475D60CFF6FF6763
:10B7300007EA0C0747EA08279F614F6809699F637A
:10B740001C629F6947F400679F619F6927F48067C7
:10B750009F61A6E00027C4F20107BB4201D07345F8
:10B7600007D14F6925F440558E6945EA071747EA26
:10B7700006154FF68C775D60CFF6FE7707EA0C076B
:10B7800047EA0807DF614F680969DF631C62DF6908
:10B7900047F00807DF61DF6927F00407DF61ACE0ED
:10B7A0000027C4F20107BB4205D040F20047C4F2B3
:10B7B0000107BB4204D14F6924F4804444EA871452
:10B7C00048F6FF475C60CFF6FF673E402CF4005719
:10B7D00046EA0524DC614E6809691E6447EA0E37B3
:10B7E0001F62DF6947F40067DF61DF6927F4806764
:10B7F000DF6156E00027C4F20107BB4205D040F2EA
:10B800000047C4F20107BB4204D14F6924F48034DD
:10B8100044EA07244FF68C775C60CFF6FE77033757
:10B820003E402CF4003746EA05045C654E68096921
:10B830009E6547EA0E471F625F6D47F008075F6528
:10B840005F6D27F004075F6557E000BF0027C4F273
:10B850000107BB4205D040F20047C4F20107BB42DA
:10B8600004D14F6924F4802444EA872448F6FF4732
:10B870005C60CFF6FF6707F540773E402CF4001779
:10B8800046EA05245C654E680969DE6547EA0E579D
:10B890001F625F6D47F400675F655F6D27F4806727
:10B8A0005F65090229E000BF0026C4F20106B34229
:10B8B00005D040F20046C4F20106B34206D12EF490
:10B8C0004077D1E90565374347EA050E4FF68C7599
:10B8D000C3F804E0CFF6FE750CEA050747EA08074F
:10B8E0009F614F6809695F631C629F6947F00807A1
:10B8F0009F619F6927F004079F61136819431160D6
:10B900000021002280F83C200846BDE8F0810000BC
:10B9100060B310B5044690F83D0028B9002084F8C3
:10B920003C00204600F024F8022084F83D00206806
:10B93000211D06F045FA012084F8480084F83E00F5
:10B9400084F83F0084F8400084F8410084F8420005
:10B9500084F8430084F8440084F8450084F84600E5
:10B9600084F8470084F83D00002010BD0120704796
:10B970007047000000000000704700000000000059
:10B9800071B10A1F4FEAB202032A11D8DFE802F0B0
:10B9900002161E2400F13F031B78012B13D120E077
:10B9A00090F83E20012A0ED1022280F83E2032E09B
:10B9B00000F143031B78012B05D112E000F1400395
:10B9C0001B78012B0DD00120704700BF00F141030F
:10B9D0001B78012B05D0F6E700F142031B78012B01
:10B9E000F1D1032A08D8DFE802F0030B0F1300BFE0
:10B9F000022280F83F200EE0022280F843200AE075
:10BA0000022280F8402006E0022280F8412002E075
:10BA1000022280F84220026801F01F00012101FA91
:10BA200000F0116A814311624EF2FF31C4F200014D
:10BA30008A42116A40EA0100106215DC40F6FF30CC
:10BA4000C4F20000824227DCB2F1804F4ED040F2B7
:10BA50000040C4F20000824248D040F60000C4F228
:10BA60000000824242D053E043F6FF700021C4F24E
:10BA70000100C4F20101824244F20000C4F201005C
:10BA80001EDC4EF20043C4F200039A422ED08A42DA
:10BA900024D040F200431DE040F60040C4F2000014
:10BAA000824223D041F60000C4F2000082421DD041
:10BAB0004EF20000C4F20000824217D028E000BF1E
:10BAC00082420BD044F60003C4F201039A4205D02F
:10BAD00044F20043C4F201039A4219D1536C8A42E2
:10BAE00043F40041516418BF82420BD10721906892
:10BAF000C0F2010101400020062918BFB1F5803FC6
:10BB000006D1704740F20040C4F201008242EDD0FD
:10BB1000106840F001001060002070470000000035
:10BB2000026801F01F0C012303FA0CFC136A23EADC
:10BB30000C0343F6FF7CC4F2010C13626245136AE6
:10BB4000136213DD44F20003C4F201039A4218D0D9
:10BB500044F60003C4F201039A4212D044F20043B7
:10BB6000C4F201039A420CD019E000BF0023C4F2D2
:10BB700001039A4205D040F20043C4F201039A4205
:10BB80000DD1D2F820C041F211131CEA030F06D1E7
:10BB9000D2F820C040F244431CEA030F12D0D2F87E
:10BBA00020C041F211131CEA030F16D1D2F820C0B5
:10BBB00040F244431CEA030F0FD1136823F0010342
:10BBC00013600AE0536C23F400435364D2F820C09E
:10BBD00041F211131CEA030FE8D04FEAB101042926
:10BBE0000AD8DFE801F0030F151B2100012180F8BE
:10BBF0003E100020704700BF012180F84310002054
:10BC0000704700BF012180F83F100020704700BF3F
:10BC1000012180F840100020704700BF012180F80A
:10BC200041100020704700BF012180F84210002021
:10BC300070470000000000000068B0F1804F18BF9E
:10BC40007047FCF729BB00007047000000000000AF
:10BC500090F88410012901D1022070472421C0F8F6
:10BC6000881002681368116823F0005321F0010165
:10BC700011600021416613602022C0F8882080F8FE
:10BC80008410084670470000704700000000000064
:10BC9000704700000000000070B590F88420012A71
:10BCA00002D1022070BD00BF2422C0F888200268A3
:10BCB000D0F864E0BEF1000FD2F800C0136823F0A2
:10BCC00001031360936823F0606341EA030191600C
:10BCD0001AD091684AF6042E9368C0F6010E5B0FE5
:10BCE0004AF60C25C1F34266C0F601051EF8034072
:10BCF000E95C2301B3FBF1F11EF80630AE5D1B01D8
:10BD0000B3FBF6F302E000BF01210123A0F86A10A3
:10BD10002021A0F86830C2F800C0C0F888100021C7
:10BD200080F88410084670BD70B590F88420012A10
:10BD300002D1022070BD00BF2422C0F88820026812
:10BD4000D0F864E0BEF1000FD2F800C0136823F011
:10BD500001031360936823F0604341EA030191609B
:10BD60001AD091684AF6042E9368C0F6010E5B0F54
:10BD70004AF60C25C1F34266C0F601051EF80340E1
:10BD8000E95C2301B3FBF1F11EF80630AE5D1B0147
:10BD9000B3FBF6F302E000BF01210123A0F86A1013
:10BDA0002021A0F86830C2F800C0C0F88810002137
:10BDB00080F88410084670BD704700000000000045
:10BDC000704700000000000045F200010068C4F266
:10BDD0000001042301F54C42904208BF0123401AA0
:10BDE00018BF1846042808BF704700EBC00040F693
:10BDF000A041C2F2004101EB8000C06900B10047E0
:10BE0000704700000000000010B50446206850E8AC
:10BE1000000F216820F4907041E80002002A1FBF43
:10BE2000206850E8000F216820F490701CBF41E8A2
:10BE30000002002A12D0206850E8000F216820F488
:10BE4000907041E800024AB1206850E8000F216874
:10BE500020F4907041E80002002AD7D14FF6FE701E
:10BE6000CEF6FF70216851E8021F2268014042E8C7
:10BE70000213002B1FBF216851E8021F22680140F6
:10BE80001CBF42E80213002B10D0216851E8021FAA
:10BE90002268014042E8021343B1216851E8021FC1
:10BEA0002268014042E80213002BDBD1E06E01283A
:10BEB00028D100BF206850E8000F216820F0100052
:10BEC00041E80002002A1FBF206850E8000F2168E7
:10BED00020F010001CBF41E80002002A12D02068A8
:10BEE00050E8000F216820F0100041E800024AB13C
:10BEF000206850E8000F216820F0100041E800029F
:10BF0000002AD7D12068816849060FD40021A4F8FF
:10BF10005E10A1650F2202622020C4F88C0020462A
:10BF2000E166FFF751FF002010BD00BF50E8020F8F
:10BF3000216820F0400041E80202FAB1206850E890
:10BF4000020F216820F0400041E80202002A1FBFD2
:10BF5000206850E8020F216820F040001CBF41E833
:10BF60000202002A0AD0206850E8020F216820F05F
:10BF7000400041E802020AB12068D7E7D4F8800007
:10BF800070B143F2D961C0F601010165F9F760FDB6
:10BF90000028C8D0D4F88000016D8847002010BD6B
:10BFA0000020A4F85E002168A0650F220A628A6959
:10BFB00042F008028A612021C4F88C10E066204615
:10BFC000FFF702FF002010BD45F200010068C4F237
:10BFD0000001042301F54C42904208BF0123401A9E
:10BFE00018BF1846042808BF704700EBC00040F691
:10BFF000A041C2F2004101EB8000006900B100479E
:10C000007047000000000000B0B50446006840F62C
:10C010002F01C26905681140D0F808E020290BD132
:10C0200005F020010EF08053C91823D0616FD1B301
:10C030002046BDE8B040084740F60F010A4219D03B
:10C04000012140F22013C1F20001C0F200430EEAC8
:10C05000010C05EA030111EB0C010BD0D10718BF4D
:10C0600015F4807140F0C68191070EF0010300F1D4
:10C07000CD81D4E105EA0203D906E16E14D5012988
:10C0800012D1102101628168490600F19D80B4F847
:10C090005C10B4F85E20B4F85E30002B1CBF891A27
:10C0A0005FEA01422FD1B0BDD10240F159811EF4A7
:10C0B000800100F055814FF4801101622046BDE8F7
:10C0C000B040FFF77DBE00BF206850E8000F226837
:10C0D00020F4907042E80003002B1FBF206850E856
:10C0E000000F226820F490701CBF42E80003002B70
:10C0F00012D0206850E8000F226820F4907042E8C7
:10C1000000034BB1206850E8000F226820F49070C3
:10C1100042E80003002BD7D14FF6FE70CEF6FF7039
:10C12000226852E8022F2368024043E80225002DCE
:10C130001FBF226852E8022F236802401CBF43E859
:10C140000225002D10D0226852E8022F23680240F9
:10C1500043E8022545B1226852E8022F23680240D5
:10C1600043E80225002DDBD12020C4F88C000020FC
:10C17000E0666067206850E8000F226820F0100039
:10C1800042E80003002B1FBF206850E8000F226820
:10C1900020F010001CBF42E80003002B12D02068E2
:10C1A00050E8000F226820F0100042E800034BB175
:10C1B000206850E8000F226820F0100042E80003D9
:10C1C000002BD7D189B227E2D4F8803019684A68A9
:10C1D000B4F85CC091B2002900F01682614580F08D
:10C1E0001382A4F85E20D969B1F5807F00F0AC809D
:10C1F00050E8000F216820F4807041E80002FAB195
:10C20000206850E8000F216820F4807041E80002A7
:10C21000002A1FBF206850E8000F216820F48070BA
:10C220001CBF41E80002002A0AD0206850E8000F35
:10C23000216820F4807041E800020AB12068D7E745
:10C24000206850E8020F216820F0010041E8020256
:10C25000002A1FBF206850E8020F216820F001006B
:10C260001CBF41E80202002A26D0206850E8020FD5
:10C27000216820F0010041E80202EAB1206850E89C
:10C28000020F216820F0010041E80202002AD7D104
:10C2900012E000BF206850E8020F216820F0400043
:10C2A00041E80202EAB1206850E8020F216820F05C
:10C2B000400041E80202A2B1206850E8020F216864
:10C2C00020F0400041E80202002A1FBF206850E829
:10C2D000020F216820F040001CBF41E80202002A42
:10C2E000D8D12020C4F88C000020E066206850E8F7
:10C2F000000F216820F0100041E80002002A1FBF53
:10C30000206850E8000F216820F010001CBF41E8B1
:10C310000002002A12D0206850E8000F216820F0A7
:10C32000100041E800024AB1206850E8000F21687F
:10C3300020F0100041E80002002AD7D1D4F8800094
:10C34000F9F7EAF8B4F85CC002202067B4F85E00A0
:10C35000ACEB000081B22046BDE8B040FFF794BCD2
:10C3600011060BD505F0800C0EF4000111EB0C0149
:10C3700004D0A16F00297FF45BAE94E659060BD47C
:10C38000100240F17D8115F0804000F07981204657
:10C39000BDE8B040FFF710BD50E8000F216820F065
:10C3A000400041E80002002A00F04681206850E881
:10C3B000000F216820F0400041E80002002A1FBF62
:10C3C000206850E8000F216820F040001CBF41E8C1
:10C3D0000002002A00F03081206850E8000F216838
:10C3E00020F0400041E80002002A00F0258120688A
:10C3F000D2E700BF01210162D4F8901041F00101A1
:10C40000C4F8901091070EF0010308D53BB102214A
:10C410000162D4F8901041F00401C4F89010510763
:10C4200008D53BB104210162D4F8901041F002011B
:10C43000C4F8901011070CD505F0200151EA0C0149
:10C4400007D008210162D4F8901041F00801C4F827
:10C45000901011050BD515F0806108D04FF40061E4
:10C460000162D4F8901041F02001C4F89010D4F883
:10C47000901000293FF417AE12F020010AD005F009
:10C4800020010EF08052891804D0616F11B120464E
:10C4900088472068D4F89010826802F0400201F0CA
:10C4A0002801891800F0C08050E8000F216820F4AE
:10C4B000907041E80002FAB1206850E8000F21684E
:10C4C00020F4907041E80002002A1FBF206850E865
:10C4D000000F216820F490701CBF41E80002002A80
:10C4E0000AD0206850E8000F216820F4907041E8DD
:10C4F00000020AB12068D7E74FF6FE70CEF6FF7053
:10C50000216851E8021F2268014042E80213002B13
:10C510001FBF216851E8021F226801401CBF42E88A
:10C520000213002B10D0216851E8021F226801403D
:10C5300042E8021343B1216851E8021F226801401A
:10C5400042E80213002BDBD1E06E012828D100BFA6
:10C55000206850E8000F216820F0100041E8000238
:10C56000002A1FBF206850E8000F216820F010004B
:10C570001CBF41E80002002A12D0206850E8000FDA
:10C58000216820F0100041E800024AB1206850E81C
:10C59000000F216820F0100041E80002002AD7D1E6
:10C5A0002020C4F88C000021E16620686167816862
:10C5B00049065FD550E8020F216820F0400041E8AD
:10C5C0000202002A42D0206850E8020F216820F0C1
:10C5D000400041E80202002A1FBF206850E8020F15
:10C5E000216820F040001CBF41E80202002A2DD043
:10C5F000206850E8020F216820F0400041E8020264
:10C6000022B32068D6E700BF8C457FF44CADD869D3
:10C61000B0F5807F7FF447AD022020672046BDE85B
:10C62000B040FFF731BB00BF2046FFF7CDFC002034
:10C63000C4F89000B0BD00BF2020C4F888000020DE
:10C64000A0672046BDE8B04000F002BCD4F88000EE
:10C6500080B143F21131C0F601010165F9F7F8F933
:10C6600000283FF420ADD4F88000016DBDE8B04053
:10C67000084700BF2046BDE8B040FFF7A5BC00BF9B
:10C68000D0017FF510ADB5F1FF3FC8BFB0BD20466A
:10C69000BDE8B040FFF7FCBA10B5E0B10446D0F8F1
:10C6A000880028B9002084F88400204600F028F88B
:10C6B0002420C4F888002068A16A0268002922F0BA
:10C6C0000101016002D0204606F0F6FC204607F08A
:10C6D000A7FD012802D1012010BD00BF20684168DC
:10C6E00021F490414160816821F02A018160016854
:10C6F00041F0010101602046BDE8104006F04CBD4C
:10C700002DE9F043B5B0044602A8B8210025CDE9D3
:10C710003355CDE931553095F4F73BF841F60041FA
:10C720002068C4F20101884274D045F20001C4F2CD
:10C730000001884240F0F18002A8002603964FF0E5
:10C740000208CDF808801F96FCF722F808B1F8F728
:10C7500057F944F2E04041F20007C5F60200C5F681
:10C76000020730AD4FF00809816841F48011816003
:10C77000816801F4801101910199016841F004017F
:10C780000160016801F0040101910199016841F023
:10C79000080101600068294600F008000190019836
:10C7A0004FF48050CDE93008A7F50060CDF8D09067
:10C7B000CDE93266FBF764FC04202946CDE9300858
:10C7C000A7F58060CDF8D090CDE93266FBF758FC34
:10C7D00041F2B8655820C2F20045C4F20200286058
:10C7E0004120C5E901064FF48060EE60C5E904060A
:10C7F0004FF40030C5E908062846C5E90666F9F792
:10C80000A7FE08B1F8F7FCF8C4F8805005F138002D
:10C81000352579E00120029002A803952095FBF7C9
:10C82000B7FF08B1F8F7ECF844F2E04041F2000538
:10C83000C5F60200C5F6020530AE40F2580801699F
:10C840004FF0020941F0800101610169002701F008
:10C85000800101910199016841F0100101600068B7
:10C86000314600F010000190019804203090C4F28D
:10C87000020834902846CDF8C490CDE93277FBF712
:10C88000FFFB08203146CDE930090B2034902846C3
:10C89000CDE93277FBF7F4FB41F2307508F574709F
:10C8A000C2F200454FF4806628607620C5E9010792
:10C8B0002846EF60C5E90467C5E90677C5E908774A
:10C8C000F9F746FE08B1F8F79BF8C4F8805008F570
:10C8D0007A70AC6341F2A875C2F2004528607720F7
:10C8E00068604020C5E902072846C5E90467C5E934
:10C8F0000677C5E90877F9F72BFE08B1F8F780F855
:10C90000E56705F138009C250460052100222846D2
:10C91000FBF792FD2846FBF77FFD35B0BDE8F083BD
:10C92000B0B50446D0F88C00202807D115460A4639
:10C930000120002918BF002D02D1B0BD0220B0BDDA
:10C940004FF0000CC4F86CC040F600402168C5F6FA
:10C950000000814234D04868000231D551E8000F10
:10C96000D4F800E040F080604EE8000141B300BF21
:10C97000206850E8000F216840F0806041E8000323
:10C98000002B1FBF206850E8000F216840F0806036
:10C990001CBF41E80003002B12D0206850E8000FB4
:10C9A000216840F0806041E800034BB1206850E806
:10C9B000000F216840F0806041E80003002BD7D1D0
:10C9C000A2652220A4F85C50C4F890C0C4F88C0082
:10C9D000D4F88000F0B143F2395143F2B963C0F6A4
:10C9E0000101C0F60103C0E90F1343F22131002316
:10C9F000C0F60101C1642168036524312B46FAF7B2
:10CA0000EBF838B11020C4F890002020C4F88C0056
:10CA10000120B0BD206938B3206850E8000F2168BC
:10CA200040F4807041E80002002A1FBF206850E8EF
:10CA3000000F216840F480701CBF41E80002002A0A
:10CA400012D0206850E8000F216840F4807041E85F
:10CA500000024AB1206850E8000F216840F480705D
:10CA600041E80002002AD7D1206850E8020F21686F
:10CA700040F0010041E80202002A1FBF206850E890
:10CA8000020F216840F001001CBF41E80202002AA9
:10CA90001DD0206850E8020F216840F0010041E8F5
:10CAA0000202A2B1206850E8020F216840F00100A4
:10CAB00041E80202002AD7D109E000BF206850E80F
:10CAC000020F216840F0400041E80202EAB120680C
:10CAD00050E8020F216840F0400041E80202A2B194
:10CAE000206850E8020F216840F0400041E802024F
:10CAF000002A1FBF206850E8020F216840F0400064
:10CB00001CBF41E80202002AD8D10020B0BD0000BD
:10CB100080B5D0F88C30202B06D10123002918BF16
:10CB2000002A03D1184680BD022080BD0023C366C1
:10CB300040F60043D0F800C0C5F600039C4503D082
:10CB4000DCF804301B0205D407F08AFE00231846E7
:10CB500080BD00BF5CE800CFD0F800E04CF08063FF
:10CB60004EE8003CBCF1000FEED0036853E800CF64
:10CB7000D0F800E04CF080634EE8003CBCF1000FC0
:10CB80001FBF036853E800CFD0F800E04CF080638B
:10CB90001CBF4EE8003CBCF1000FD5D0036853E841
:10CBA00000CFD0F800E04CF080634EE8003CBCF1D0
:10CBB000000FC9D0036853E800CFCDE700000000A4
:10CBC00045F200010068C4F20001042301F54C4263
:10CBD000904208BF0123401A18BF1846042808BF16
:10CBE000704700EBC00040F6A041C2F2004101EBEB
:10CBF0008000C06800B100477047000000000000DE
:10CC000045F200010068C4F20001042301F54C4222
:10CC1000904208BF0123401A18BF1846042808BFD5
:10CC2000704700EBC00040F6A041C2F2004101EBAA
:10CC30008000806800B100477047000000000000DD
:10CC4000B0B50446D0F88800202831D100294FF033
:10CC5000010061D0002A134608BFB0BD2165002540
:10CC6000A4F854302120A4F85630C4F89050C4F8E9
:10CC70008800E06FF0B143F2213243F2017CC0F64C
:10CC80000102C264226843F2C17E2832C0F6010C60
:10CC9000C0F6010E0565C0E90FCEF9F79DFF48B15A
:10CCA0001020C4F890002020C4F888000120B0BDF6
:10CCB0000220B0BD20684021016250E8020F2168C7
:10CCC00040F0800041E8020242B300BF206850E813
:10CCD000020F216840F0800041E80202F2B12068B2
:10CCE00050E8020F216840F0800041E80202AAB13A
:10CCF000206850E8020F216840F0800041E80202FD
:10CD000062B1206850E8020F216840F0800041E8DD
:10CD100002020020002AD9D1B0BD00BF0020B0BD62
:10CD2000D0F88830202B07D10123002918BF002A12
:10CD300004D11846704700BF0220704701650021EA
:10CD4000A0F85420A0F85620C0F890102121C0F877
:10CD50008810416EB1F1005F816835D1B1F5805F17
:10CD600002D10169002963D044F66951C0F601017E
:10CD70008167016851E8021F026841F4000142E83E
:10CD80000213002B52D0016851E8021F026841F4DF
:10CD9000000142E80213002B1FBF016851E8021F87
:10CDA000026841F400011CBF42E80213002B3DD091
:10CDB000016851E8021F026841F4000142E80213D1
:10CDC000002BD6D132E000BFB1F5805F01D10169FF
:10CDD000A1B344F69941C0F601018167016851E8A9
:10CDE000001F026841F0800142E8001363B301684C
:10CDF00051E8001F026841F0800142E80013002B57
:10CE00001FBF016851E8001F026841F080011CBF8C
:10CE100042E80013002B09D0016851E8001F0268A6
:10CE200041F0800142E80013002BD7D10020704769
:10CE300044F6A931C0F601019AE700BF44F6D921B2
:10CE4000C0F60101C9E700BF002318467047000083
:10CE500045F200010068C4F20001042301F54C42D0
:10CE6000904208BF0123401A18BF1846042808BF83
:10CE7000704700EBC00040F6A041C2F2004101EB58
:10CE80008000406800B100477047000000000000CB
:10CE900045F200010068C4F20001042301F54C4290
:10CEA000904208BF0123401A18BF1846042808BF43
:10CEB000704740F6A04100EBC000C2F2004151F8BB
:10CEC000200008B1004700BF7047000000000000CC
:10CED000FEE700000000000010EE100AB6EE001A97
:10CEE00045F6DF11B7EE083AC5F6377120EE010AB4
:10CEF000A1EB6000B0EE434A01EE100A20EE012AD9
:10CF000002EE414A24EE011A20EE010A01EE403AF7
:10CF100021EE030A7047000030B3B0EE403A90EDC6
:10CF2000011A90ED062A90ED074A80ED072A02EEDD
:10CF3000413A90ED021A04EE413A13EE101A21F034
:10CF40000041B1F1FF4F00FE031A90ED030A90ED8E
:10CF5000043A80ED061A20EE010A02EE030A90ED73
:10CF6000053A04EE030A70479FED010A704700BFBF
:10CF70000000000000000000002808BF704710B546
:10CF80000446F5EE400AC0ED000A0020F1EE10FA6A
:10CF9000A061E06132DD80EE200A9FED201A81EE73
:10CFA000000A0CF043FF9FED1E1AB7EE002A20EE98
:10CFB000011A20EE004A31EE023A32EE410ABFEE8B
:10CFC000002A34EE031A34EE022A34EE000A84EE0C
:10CFD000013A32EE022A84ED033A80EE010A84ED32
:10CFE000053A33EE034A82EE011A84ED044A84EDD9
:10CFF000011A84ED020ABDE8104070474FF07E51DF
:10D000006061C4E9031060609FED030A84ED020AC9
:10D01000BDE81040704700BF00000000DB0F494032
:10D02000F304B53F0000000080B390ED031A90EDCB
:10D03000042A31EE023A90ED054AB0EE406A90EDD6
:10D04000015A33EE043A80EE033A13EE101A01F05F
:10D05000FF41B1F1FF4F00FE033A80ED073A03EEC6
:10D06000456A90ED025A03EE456A16EE101A21F059
:10D070000041B1F1FF4F00FE065A80ED065A21EE45
:10D08000050A02EE030A04EE030A70479FED010A47
:10D09000704700BF0000000010B584B0002841D0E8
:10D0A00090F800C0BCF1020F38D840F60C51C2F223
:10D0B000004151F82C1089B391F8842072B30B1DF4
:10D0C00004E000BF013A03F1040327D0D3F800E0E5
:10D0D000BEF1000FF6D09EF800106145F2D1BEF807
:10D0E00002104488A142EDD1BEF8040069460090C8
:10D0F00008208DF804004FF0FF30CDF805000290B5
:10D10000FC208DF80C009EF80000F5F729FA0028A5
:10D1100018BF4FF0FF3040B204B010BDFC2040B249
:10D1200004B010BDFE2040B204B010BD00000000ED
:10D13000B0B518B390F800C0BCF1020F1ED840F68D
:10D140000C51C2F2004151F82C10B9B191F8843061
:10D15000A3B101F1040E002203E000BF01329A42A4
:10D160000ED25EF822100029F8D00C786445F5D173
:10D170004C884588AC42F1D10846B0BD0020B0BD16
:10D1800000210846B0BD0000B0B584B0FE220028E2
:10D1900018BF002902D150B204B0B0BD90F800C051
:10D1A000BCF1020F00F2968040F60C52C2F200422F
:10D1B00052F82C20002A00F08D8092F88430002B49
:10D1C00000F08880043204E0013B02F1040200F028
:10D1D0008180D2F800E0BEF1000FF5D09EF800404B
:10D1E0006445F1D1BEF802404588AC42ECD19EF8CE
:10D1F0000700002872D0B3EE0E0A91ED021A9FEDDF
:10D20000732A91ED013A32EE411A9FED712A30EE08
:10D21000430A9FED705A91ED003A91ED034A21EED9
:10D22000021A9FED6D2A20EE020A91ED046A24EEA7
:10D23000024AB1EE047A81EE051A9FED685A80EE3B
:10D24000050AB2EE085A26EE026ABEF80400BDEEE8
:10D25000C11A009035EE433A9FED615A84EE054ABB
:10D26000082086EE075A11EE101A23EE022AB3EEBA
:10D27000083ABDEEC00A8DF80400080A8DF80610C1
:10D2800082EE032A8DF80500BDEEC43A10EE102A96
:10D29000BDEEC54ABDEEC22A13EE103A100914EED7
:10D2A000105A8DF8070012EE104A8DF80930190A4D
:10D2B00041EA02108DF8080029018DF80C40280978
:10D2C0008DF80A0041EA14208DF80B009EF800004A
:10D2D000694671E0FC2250B204B0B0BDB3EE0E2A34
:10D2E00091ED020A9FED391AB2EE084A30EE010ABA
:10D2F00091ED011A31EE021A9FED353A9FED362A73
:10D3000091ED035A20EE030A9FED323A21EE021A04
:10D3100091ED046A25EE025AB1EE047A80EE030A1A
:10D320009FED2E3A81EE031A91ED003A33EE043A66
:10D330009FED2B4A26EE026ABEF8040085EE044AF1
:10D34000009023EE022AB3EE083A86EE075A082030
:10D35000BDEEC00A8DF8040082EE032ABDEEC11AAC
:10D36000BDEEC43A10EE101ABDEEC54ABDEEC22A9B
:10D3700011EE102A13EE103A080A14EE105A8DF826
:10D38000061012EE104A11018DF8050010098DF8F3
:10D39000070041EA1320210A8DF8080028098DF8BA
:10D3A00009308DF80A0041EA05108DF80B00694636
:10D3B0008DF80C409EF80000F5F7D2F802460028E0
:10D3C00018BF4FF0FF3250B204B0B0BDDA0F494180
:10D3D00000FF7F47DA0FC94100F07F45000070422F
:10D3E0000000FA4300000000F0B581B0002841D0F1
:10D3F00006780446022E4FD840F60C57C2F200477A
:10D4000057F82600D0B357F82660002E44D096F87F
:10D410008400002846D0002103E000BF043181428F
:10D420003ED206EB810253681BB15B886788BB4222
:10D430001BD04B1C834233D293681BB15B88678837
:10D44000BB4212D08B1C83422AD2D3681BB15B88AB
:10D450006788BB4209D0CB1C834221D21269002AC3
:10D46000DCD0528863889A42D8D1FD2040B201B006
:10D47000F0BD00BFFE2040B201B0F0BD8820F5F73E
:10D480003BFA47F8260038B188210546F3F781F9C1
:10D490002E702678022EB6D9FF2040B201B0F0BD22
:10D4A0001F28F9D83020F5F727FA0028F4D03021CA
:10D4B0000546F3F76EF920686168C5E900010020B0
:10D4C00028722078E27961882A760322F4F780FBBB
:10D4D00030B12846F5F75CF9FF2040B201B0F0BD4D
:10D4E00096F8840006EB8001013086F88400002065
:10D4F0004D6040B201B0F0BD2DE9F0438BB048B1B2
:10D500008146007802280BD9FC2148B20BB0BDE857
:10D51000F08300BFFE2148B20BB0BDE8F08300BF2E
:10D5200040F60C58C2F2004858F82020002A4DD08E
:10D5300092F88430002B49D0002703E00437FC2107
:10D540009F42E2D202EB87056E6826B17188B9F876
:10D550000240A1421ED0791C994237D2AE6826B152
:10D560007188B9F80240A14214D0B91C99422DD259
:10D57000EE6826B17188B9F80240A1420AD0F91CC0
:10D58000994223D22E69002ED8D07188B9F8025062
:10D59000A942D3D16A460023F4F7C2F9E0B1F5F706
:10D5A000DFFAD6E90423801A48F2A162C0F2010230
:10D5B0009941801A71F10000C0F0FC8000203072A7
:10D5C000FF2148B20BB0BDE8F08300BFFC2148B298
:10D5D0000BB0BDE8F08300BF377A01203072F5F759
:10D5E000BFFABDF80E209FED761AC6E904011204B9
:10D5F0009DF81110B3EE084ABAEE085A10BA00EEC0
:10D60000100A9DF8100001F00F039DF81220000190
:10D61000B8EEC00A40EA111042EA032102EE100AF5
:10D6200003EE101A20EE010A9FED661A9DF8130012
:10D63000B8EEC22AB8EEC33A80EE010A9FED631A33
:10D6400022EE011A9FED602A23EE043ABBEE0E4A49
:10D6500030EE020A9FED5E2A81EE021A86ED070A7D
:10D6600083EE023AB5EE400A31EE042A33EE051A93
:10D6700003EE100AF1EE10FA86ED082AB8EE433AEE
:10D6800086ED091A86ED0A3A4ADA9FED523A30EEF3
:10D69000030AB5EE400AF1EE10FABFBF30EE030AFE
:10D6A000B5EE400AF1EE10FA30EE030ABCBFB5EE5B
:10D6B000400AF1EE10FA06DA30EE030AB5EE400A3F
:10D6C000F1EE10FAE3DB86ED070A9FED423AB4EE85
:10D6D000430AF1EE10FA2ADB9FED3F4A30EE040ACE
:10D6E000B4EE430AF1EE10FAA1BF30EE040AB4EE34
:10D6F000430AF1EE10FA30EE040AA4BFB4EE430A76
:10D70000F1EE10FA06DB30EE040AB4EE430AF1EE55
:10D7100010FAE3DA86ED070AF07950B915E000BF98
:10D720009FED2C3AB4EE430AF1EE10FAD4DAF07918
:10D7300058B133EE400AB1EE422A86ED070AB1EE47
:10D74000410A86ED082A86ED090A77BB99F80000A0
:10D7500002282AD858F8201039B391F8842022B32F
:10D760000B1D06E0013A03F104034FF000013FF402
:10D77000CCAE19680029F5D00F788742F2D14F88D6
:10D78000B9F80260B742EDD18888079008208DF87B
:10D7900020004FF0FF30CDF821000990FC208DF8DB
:10D7A0002800087807A9F4F7DBFE002148B20BB087
:10D7B000BDE8F083FF2148B20BB0BDE8F08300BFA5
:10D7C000DA0FC94100FF7F47DA0F49C100007042FC
:10D7D00000F07F45DB0FC940DB0FC9C0000000002F
:10D7E00080B584B0B0B30146007802282ED840F648
:10D7F0001852C2F2004252F820203AB34988A1F2EE
:10D8000001210A296ED8012303FA01F10B0725D162
:10D8100011F0F00F40D0518940F2FF13009393892B
:10D820004FF0080C8DF804C009BA090CADF80510CA
:10D830001BBAD1891B0CADF807300BBA118A1A0C30
:10D84000ADF809200A0A8DF80B203EE0FC2040B21A
:10D8500004B080BDFE2040B204B080BD4FF4007122
:10D86000009108218DF80410D1788DF80510917879
:10D870008DF8061051798DF8071011798DF8081080
:10D88000D1798DF8091091798DF80A10517A8DF8B7
:10D890000B10117A19E000BF40F2FF21009108211E
:10D8A0008DF80410918A538AD28A8DF80A2009BA19
:10D8B0001BBA090CADF80710110A8DF809100021E8
:10D8C0001B0CADF805308DF80B108DF80C10694667
:10D8D000F4F746FE002818BF4FF0FF3040B204B006
:10D8E00080BD00BFFF2040B204B080BD000000003A
:10D8F000B0B5E8B3017802293AD840F61852C2F21E
:10D90000004252F821C0BCF1000F31D09CF844E035
:10D91000BEF1000F2CD0002204E000BF0432002131
:10D92000724528D20CEB8203996919B14C8845885D
:10D93000AC4220D0511C71451CD2D96919B14C8818
:10D940004588AC4217D0911C714511D2196A19B1A2
:10D950004C884588AC420ED0D11C714508D2596A1A
:10D960000029DBD04B884488A342D7D103E000BF15
:10D970000020B0BD00210846B0BD0000000000003E
:10D98000F0B581B0002841D006780446022E4FD869
:10D9900040F61857C2F2004757F82600D0B357F8A0
:10D9A0002660002E44D096F84400002846D000217E
:10D9B00003E000BF043181423ED206EB810293694D
:10D9C0001BB15B886788BB421BD04B1C834233D2A0
:10D9D000D3691BB15B886788BB4212D08B1C834222
:10D9E0002AD2136A1BB15B886788BB4209D0CB1C63
:10D9F000834221D2526A002ADCD0528863889A423C
:10DA0000D8D1FD2040B201B0F0BD00BFFE2040B231
:10DA100001B0F0BD4820F4F76FFF47F8260038B199
:10DA200048210546F2F7B5FE2E702678022EB6D9AB
:10DA3000FF2040B201B0F0BD0A28F9D85020F4F719
:10DA40005BFF0028F4D0054620686168C5E9000145
:10DA500005F118002821F2F79CFE20786279618890
:10DA600085F828200322F4F7B3F838B12846F4F7F4
:10DA70008FFEFF2040B201B0F0BD00BF96F8440019
:10DA800006EB8001013086F8440000208D6140B231
:10DA900001B0F0BD000000009FED010A00F004B8E5
:10DAA0000000000000000000F0B5002860D0017800
:10DAB000022959D840F61852C2F2004252F82110F9
:10DAC000002951D0B7EE001A4279002A91F844207B
:10DAD00080FE410ABFEE001A80FE010AB1EE402A24
:10DAE00000FE020A002A3FD0C2F1000CA2F1010E92
:10DAF000002303E00433FC249A4252D001EB830557
:10DB0000AC691CB164884688B4421AD09E452BD0BB
:10DB1000EC691CB164884688B44212D00CEB030651
:10DB2000B41C21D02C6A1CB164884788BC4208D040
:10DB3000F41C19D06C6A002CDCD064884588AC4297
:10DB4000D8D10079022817D2A4F20122082A2BD2B8
:10DB500001289FED182A02FE011A00289FED162ABF
:10DB600002FE011A0FE000BFFC2460B2F0BD00BF4E
:10DB7000FE2460B2F0BD00BF16D1A4F20520072834
:10DB800012D29FED0B1A20EE010A4FF07F4000EBFE
:10DB900004600024BDEEC00A01EBE05010EE101A44
:10DBA000418060B2F0BD00BFFF2460B2F0BD00BF95
:10DBB0000060EA460000804600401C46000000006D
:10DBC000F0B587B040B102460078022808D9FC21A0
:10DBD00048B207B0F0BD00BFFE2148B207B0F0BDAB
:10DBE00040F61851C2F2004151F820C0BCF1000FBC
:10DBF0003FD09CF84430E3B3002403E00434FC211C
:10DC00009C42E5D20CEB8405AF691FB17988568838
:10DC1000B1421BD0611C99422BD2EF691FB17988A8
:10DC20005688B14212D0A11C994222D22F6A1FB14C
:10DC300079885688B14209D0E11C994219D26F6A9D
:10DC4000002FDBD079885688B142D7D16A460023AD
:10DC5000F3F766FE90B1F4F783FFD7E90823801A43
:10DC600040F2E9329941801A71F1000028D3002076
:10DC70003876FC2148B207B0F0BD00BF01203876ED
:10DC8000F4F76EFFBDF80D2097F90430C7E90801DD
:10DC9000BDF80F10022B10BABDF811204FEA10404A
:10DCA00009BA12BA4FEA11414FEA12420CD872A6D1
:10DCB0006EA506EB830655F8233096ED004A07E083
:10DCC000FF2148B207B0F0BDB7EE004A4FF0FF3376
:10DCD00012B200EE100A5A439FED6A1A09B29FED84
:10DCE0006B5AB8EE400A02EE102A20EE011A9FEDA0
:10DCF000660AB8EEC23A02EE101AB97921EE001A9D
:10DD0000B8EEC22A23EE053A41B1B7F84010411AE5
:10DD1000B1F5805F3ADD796C01393CE0A7F840004D
:10DD20000020C7E9110087ED021A07F1080087ED0E
:10DD3000032A87ED043AB4EE401AF1EE10FA72DBD2
:10DD40009FED534A31EE041AB4EE401AF1EE10FA88
:10DD5000A1BF31EE041AB4EE401AF1EE10FA31EE22
:10DD6000041AA4BFB4EE401AF1EE10FA06DB31EE4D
:10DD7000041AB4EE401AF1EE10FAE3DA80ED001A5C
:10DD800097F82800002851D15CE000BF11F5805FB2
:10DD9000796C01DA0131796405EE101A82EE042AF9
:10DDA00024EE033AA7F8400007F1080087ED032AA4
:10DDB000B8EEC55A87ED043A05EE001A81EE041A52
:10DDC00087ED121A87ED021AB5EE401AF1EE10FA3D
:10DDD00024DA31EE001AB5EE401AF1EE10FABFBFA8
:10DDE00031EE001AB5EE401AF1EE10FA31EE001ADB
:10DDF000BCBFB5EE401AF1EE10FA06DA31EE001AA9
:10DE0000B5EE401AF1EE10FAE3DB80ED001AB4EE45
:10DE1000401AF1EE10FA06DB92E700BFB4EE401AAA
:10DE2000F1EE10FA8CDA97F8280058B130EE410A7A
:10DE3000B1EE421A87ED020AB1EE430A87ED031AEA
:10DE400087ED040A9DF8130000EE100AD7E90201DD
:10DE5000F8623869B8EE400A396387ED050A7969D6
:10DE6000C7E90D01002148B207B0F0BD102700003E
:10DE70000040000030750000000010422CA09941C5
:10DE80000000803F00000039DB0FC94000008038EF
:10DE9000DB0FC9C00000000080B582B044F2D8405A
:10DEA0000022C5F60200016841F00101016001682D
:10DEB00001F0010101910199016841F00201016045
:10DEC0000068052100F00200009000980B20FAF78E
:10DED000B3FA0B20FAF7A0FA0C2005210022FAF77A
:10DEE000ABFA0C20FAF798FA0E2005210022FAF777
:10DEF000A3FA0E20FAF790FA392005210022FAF74A
:10DF00009BFA3920FAF788FA3A2005210022FAF71D
:10DF100093FA3A2002B0BDE88040FAF77DBA0000DB
:10DF200080B541F620004AF20001C2F20040C4F27E
:10DF300000010122052301600021C0E902110282D3
:10DF40004FF00E0C8274C0E90533C0E907C3C0E985
:10DF50000933C0E90BC3C0E90D12C2631022026489
:10DF60000423C0E91131C0E91331C0E91531C0E91A
:10DF70001712C0E91913F9F75FFC002808BF80BD2C
:10DF8000BDE88040F6F73CBD80B541F6C0004AF2DE
:10DF90000041C2F20040C4F20001012205230160E9
:10DFA0000021C0E9021102824FF00E0C8274C0E918
:10DFB0000533C0E907C3C0E90933C0E90BC340F228
:10DFC0003F33C0E90D32C0E90F210422426414231B
:10DFD0008266C0E91232C0E91412C0E9161110239A
:10DFE000C0E91831F9F728FC002808BF80BDBDE85A
:10DFF0008040F6F705BD000080B541F660104DF297
:10E000000041C2F20040C4F2000101220523016078
:10E010000021C0E9021102824FF00E0C8274C0E9A7
:10E020000533C0E907C3C0E90933C0E90BC340F2B7
:10E030007E63C0E90D32C0E90F210422426410233F
:10E040008266C0E91232C0E91412C0E91611C0E9B3
:10E050001831F9F7F1FB002808BF80BDBDE880400A
:10E06000F6F7CEBC0000000080B541F651304AF60C
:10E070001422C0F60100C0F60102002107F06CFE78
:10E0800041F2282C41F63973C2F2004CC0F601036C
:10E090004AF264620021C0F60102CCF80000184682
:10E0A000BDE8804007F058BE2DE9F04186B044F24B
:10E0B000E0404FF00008C5F60200CDF8148040F6AD
:10E0C000000400220168C5F6020441F0100101605D
:10E0D00001684FF4604501F010010091009901685A
:10E0E00041F004010160016801F004010091009910
:10E0F000016841F080010160016801F08001009138
:10E100000099016841F001010160016801F001011D
:10E1100000910099016841F002010160016801F07D
:10E12000020100910099016841F008010160006856
:10E130004FF4604100F00800009000982046FAF784
:10E140009BF809210122204609270126FAF794F8B5
:10E1500001A8CDF8108080E8600101AD2046294675
:10E16000F9F78EFF20462946CDE90176CDE9036611
:10E17000F9F786FF4FF4A05001904FF404102946A0
:10E18000CDE9020604F50060F9F77AFF4FF400408C
:10E1900001904FF488102946CDE90208A4F50060EB
:10E1A000F9F76EFF4FF000600021FCF73DFE2820DC
:10E1B00005210022FAF740F92820FAF72DF906B0D8
:10E1C000BDE8F0810000000010B541F6002443F6E0
:10E1D0000000C2F20044C4F20000072120604FF4A6
:10E1E000800060600020A060E1604FF0007121615C
:10E1F0004FF0807161614FF08061A1614FF040513B
:10E20000C4E90710C4E90900E0624FF08040606390
:10E2100004F138002421F2F7BCFA2046FBF768FE2F
:10E22000002808BF10BDBDE81040F6F7E9BB0000AC
:10E2300010B541F6882441F20040C2F20044C5F610
:10E2400000004FF0806120604FF4800060604FF468
:10E250000030A0600320E0600020C4E90400C4E9AD
:10E260000610C4E90800C4E90A004FF0804060636A
:10E2700004F138002421F2F78CFA2046FBF738FE2F
:10E28000002808BF10BDBDE81040F6F7B9BB00007C
:10E29000B0B594B041F6103041F60005C2F200402E
:10E2A00000210D91C4F20005CDE90B11CDE9081153
:10E2B000CDE90611CDE90411CDE90211CDE9001136
:10E2C00005601722C0E9012140F2CF728161C0E9E7
:10E2D0000321FCF731FE08B1F6F792FB4FF48050B2
:10E2E0000A9041F610300AA9C2F20040FCF7E8FE9D
:10E2F00008B1F6F785FB41F61030C2F20040FDF799
:10E3000007FB08B1F6F77CFB41F6103007A9C2F213
:10E310000040002407940994FCF79EFD08B1F6F72D
:10E320006FFB60200294CDE90004049441F61034A0
:10E33000C2F20044694604222046FDF789F808B17C
:10E34000F6F75EFB20680021A8421391CDE9111178
:10E3500010910F9114D040F20041C4F200018842A4
:10E360002BD144F2E040C5F60200016841F0020101
:10E370000160006800F002000E900E9802200EE08E
:10E3800044F2E040C5F60200016841F0020101607C
:10E39000006800F002000E900E984FF400400F90BD
:10E3A000022010900021139040F20040CDE911119D
:10E3B000C5F602000FA9F9F763FE14B0B0BD000066
:10E3C000B0B594B041F6A83040F20045C2F200402A
:10E3D00000210D91C4F20005CDE90B11CDE9081122
:10E3E000CDE90611CDE90411CDE90211CDE9001105
:10E3F00005601722C0E9012142F20F728161C0E974
:10E400000321FCF799FD08B1F6F7FAFA4FF48050B2
:10E410000A9041F6A8300AA9C2F20040FCF750FE6B
:10E4200008B1F6F7EDFA41F6A830C2F20040FDF768
:10E430006FFA08B1F6F7E4FA41F6A83007A9C2F27C
:10E440000040002407940994FCF706FD08B1F6F794
:10E45000D7FA60200294CDE90004049441F6A83470
:10E46000C2F2004469460C222046FCF7F1FF08B1D5
:10E47000F6F7C6FA41F600022068C4F20002002155
:10E4800090421391CDE91111CDE90F1110D0A8429E
:10E490002BD144F2E040C5F60200016841F00201D0
:10E4A0000160006800F002000E900E9802200EE05D
:10E4B00044F2E040C5F60200016841F0020101604B
:10E4C000006800F002000E900E984FF400400F908C
:10E4D000022010900021139040F20040CDE911116C
:10E4E000C5F602000FA9F9F7CBFD14B0B0BD0000CE
:10E4F00080B541F6884045F20001C2F2004048F282
:10E50000A062C4F20001C0F20102C0E900124FF49F
:10E51000805181600021C1604FF480620261042259
:10E52000C0E90521C0E90711C0E90911FEF7B4F8F7
:10E5300008B1F6F765FA41F688400021C2F20040C2
:10E54000FDF7F2FB08B1F6F75BFA41F688400021CF
:10E55000C2F20040FDF7A0FB08B1F6F751FA41F610
:10E560008840C2F20040FDF773FB002808BF80BD61
:10E57000BDE88040F6F744BA80B541F6F43041F684
:10E580000041C2F20040C4F201010C2201604FF4CC
:10E59000E13141600021C0E902110161C0E90521BA
:10E5A000C0E90711C0E90911FEF776F808B1F6F7DE
:10E5B00027FA41F6F4300021C2F20040FDF7B4FB27
:10E5C00008B1F6F71DFA41F6F4300021C2F200401E
:10E5D000FDF762FB08B1F6F713FA41F6F430C2F228
:10E5E0000040FDF735FB002808BF80BDBDE8804036
:10E5F000F6F706BA00000000FEE700000000000089
:10E60000B0B5002800F097800078052808D8DFE82A
:10E6100000F00D4D6103036D012B6CDA8BE000BF40
:10E62000012B35DA002040B2B0BD00BF042BF3D17E
:10E6300091ED001A91ED012A31EE421A91ED022A74
:10E6400031EE021A82ED001A91ED001A91ED012AC5
:10E6500031EE021A91ED022A31EE021A82ED011A10
:10E6600091ED001A91ED012A32EE411A91ED022A44
:10E6700031EE021A82ED021A91ED001A91ED012A93
:10E6800031EE021A91ED022A32EE411A82ED031A9E
:10E690005FFA83FC4FF0FF3050FA83F003F0030E73
:10E6A00003284BD29FED971A00216CE0042BB3D1C5
:10E6B00091ED000AB1EE400A82ED000A0868506050
:10E6C0000868906091ED000AB1EE400A82ED030AFD
:10E6D00010E000BF022B9FD191ED000AB1EE400A7D
:10E6E00082ED000A0868506004E000BF012B93D15E
:10E6F00008681060DBB24FF0000C0024002100BF5E
:10E7000041F0010042F824C0C0B2834213DD41F061
:10E71000020542F820C0ECB2A3420CDD41F0030038
:10E7200042F824C0C0B2834205DD043142F820C063
:10E73000CCB2A342E4DCFF2040B2B0BD0CF0FC0040
:10E74000A2F110049FED6F1A002100BF94ED042A7E
:10E7500094ED053AB0EEC22A0431884282FE011AD5
:10E76000B0EEC32A94ED063A82FE011AB0EEC32A37
:10E7700094ED073A04F1100482FE011AB0EEC32AA8
:10E7800082FE011AE2D1BEF1000F19D002EB810026
:10E79000BEF1010F90ED002AB0EEC22A82FE011AEE
:10E7A0000ED090ED012ABEF1020FB0EEC22A82FE19
:10E7B000011A05D090ED022AB0EEC22A82FE011A9B
:10E7C000B7EE002AB4EE421AF1EE10FA49DD4FF02E
:10E7D000FF3050FA83F0032802D2002124E000BF6A
:10E7E0000CF0FC00A2F11004002100BF94ED042AFB
:10E7F00094ED053A94ED064A82EE012A83EE013A41
:10E8000084ED042A84EE012A84ED053A94ED073A5A
:10E8100084ED062A04F11005043183EE012A8842B2
:10E8200084ED072A2C46E1D1BEF1000F19D002EB8E
:10E830008100BEF1010F90ED002A82EE012A80EDE9
:10E84000002A0ED090ED012ABEF1020F82EE012ABD
:10E8500080ED012A05D090ED022A82EE011A80EDAA
:10E86000021A4FF0FF3050FA83F0032802D2002042
:10E8700024E000BF0CF0FC01A2F11003002000BF57
:10E8800093ED041A93ED052A93ED063A21EE001A52
:10E8900022EE002A83ED041A23EE001A83ED052AE6
:10E8A00093ED072A83ED061A03F11005043022EEDA
:10E8B000001A814283ED071A2B46E1D1BEF1000F09
:10E8C0003FF4B0AE02EB8000BEF1010F90ED001AF4
:10E8D00021EE001A80ED001A3FF4A4AE90ED011A6B
:10E8E000BEF1020F21EE001A80ED011A3FF49AAE3C
:10E8F00090ED021A21EE000A80ED020A002040B2DB
:10E90000B0BD00BF0000000020B10170002040B287
:10E91000704700BFFF2040B27047000000000000B9
:10E92000FEE700000000000010B52DED0A8B10EE90
:10E93000101A044601F0FF41B1F1FF4F00F0998039
:10E9400010EE900AB0EE60BA00F0FF40B0F1FF4F59
:10E9500000F08F8011EE100AB0EE419A00F0FF40F7
:10E96000B0F1FF4F00F0858011EE900AB0EE618AA1
:10E9700000F0FF40B0F1FF4F7BD06068F0EE4B0A33
:10E9800090ED071AF5F74CFC6068B0EE40AA90EDE8
:10E99000001A04F11C0020EE01CA21EE0B0AFEF75A
:10E9A000BBFA207860B101280CD194ED051A94EDE2
:10E9B000022A30EE411A88FE022A81EE029A01E014
:10E9C0009FED2E9A19EE100A9FED2C1A94ED032A52
:10E9D00084ED04AA0CEE082A84ED050A00F0FF403D
:10E9E000B0F1FF4F606801FE091A90ED013A2CEE7C
:10E9F000033A90ED034A90ED025A01EE443A9FED3E
:10EA0000201A22EE054AB4EE415AF1EE10FA1CDD4E
:10EA100012EE101A01F0FF41B1F1FF4F15D033EEA5
:10EA2000040A90ED055AB0EEC00AB4EE450AF1EEC4
:10EA300010FA0ADCB0EEC20A90ED045AB4EE450AB0
:10EA4000F1EE10FAD8BF84ED032A33EE040A10EE7B
:10EA5000101A01F0FF41B1F1FF4F0AD0D0ED050AC5
:10EA6000F4EE410AF1EE10FA01DDF2F7C1FB84ED9C
:10EA7000060A94ED060ABDEC0A8B10BD00000000EA
:10EA8000BD3786350000000070B550B304465068AD
:10EA900000F0FF40B0F1FF4F23D0906800F0FF403E
:10EAA000B0F1FF4F1DD0D06800F0FF40B0F1FF4F34
:10EAB00017D0106900F0FF40B0F1FF4F11D050693E
:10EAC00000F0FF40B0F1FF4F0BD0B7EE001A6260CC
:10EAD00081EE001A11EE100A00F0FF40B0F1FF4F76
:10EAE00002D1FF2568B270BD04F11C06D2ED060A02
:10EAF00030460D4684ED021AFEF73EFA9FED060AF7
:10EB0000304625700025C4E90355C4E90555FEF7D4
:10EB10008BFA68B270BD00BF00000000000000006A
:10EB200010B568B100F11C010024C0E90344446140
:10EB30009FED050A84610846FEF776FA60B210BDC3
:10EB4000FF2460B210BD00BF000000000000000004
:10EB500020B10021C16048B2704700BFFF2148B218
:10EB600070470000000000000000000000000000EE
:10EB7000EFF30980BFF36F8F154B1A681EF0100F6B
:10EB800008BF20ED108A20E9F04F10602DE9090040
:10EB90004FF0500080F31188BFF34F8FBFF36F8F9A
:10EBA00008F08AFE4FF0000080F31188BDE80900EC
:10EBB00019680868B0E8F04F1EF0100F08BFB0ECFD
:10EBC000108A80F30988BFF36F8F704700BF00BFC2
:10EBD0009C06002400000000F0B581B044F22C47F0
:10EBE000C5F6020757F8042C02F00302032A03D1EA
:10EBF000012001B0F0BD00BF054657F82C0C0C46B3
:10EC000020F0806047F82C0CF9F73EFB064600BF69
:10EC100057F82C0C000105D5F9F736FB801B0228AC
:10EC2000F6D964E057F8040CEE6895E80E0020F47D
:10EC30007C30012C40EA0130A2F101016FF35F2129
:10EC40004FF47E4202EB432247F8040C92B24FF09D
:10EC5000FE4302EB01004FF4FE012A6901EB06417D
:10EC600001F4FE0103EB0262084402F0FE41084495
:10EC7000F8603868696920F0C00040EA0100386037
:10EC80003868A96920F0200040EA0100386038683F
:10EC90004FF6F87120F0100038603869EA6920EA10
:10ECA00001004FF4001140EAC2003861386808BF23
:10ECB0004FF4801140F01000002C386008BF4FF472
:10ECC000002138680843386057F82C0C40F0806009
:10ECD00047F82C0CF9F7D8FA044600BF57F82C0C6B
:10ECE000000107D4F9F7D0FA001B0328F6D303205C
:10ECF00001B0F0BD002001B0F0BD00000000000038
:10ED0000F0B581B044F22C47C5F6020757F8042C41
:10ED100002F00302032A03D1012001B0F0BD00BFBD
:10ED2000054657F82C0C0C4620F0805047F82C0C68
:10ED3000F9F7AAFA064600BF57F82C0C800005D553
:10ED4000F9F7A2FA801B0228F6D964E057F8040C00
:10ED5000EE6895E80E0020F07C70012C40EA01502E
:10ED6000A2F101016FF35F214FF47E4202EB4322D7
:10ED700047F8040C92B24FF0FE4302EB01004FF44F
:10ED8000FE012A6901EB064101F4FE0103EB026278
:10ED9000084402F0FE41084478613868696920F44B
:10EDA000406040EA010038603868A96920F40070CA
:10EDB00040EA0100386038684FF6F87120F480703E
:10EDC0003860B869EA6920EA01004FF0807140EAD2
:10EDD000C200B861386808BF4FF4000140F4807089
:10EDE000002C386008BF4FF4800138680843386051
:10EDF00057F82C0C40F0805047F82C0CF9F744FAE7
:10EE0000044600BF57F82C0C800007D4F9F73CFAF1
:10EE1000001B0328F6D3032001B0F0BD002001B091
:10EE2000F0BD00000000000040F624004FF48071A7
:10EE3000C2F20040406806F093BE000000000000EF
:10EE400040F624004FF40071C2F20040406806F022
:10EE500087BE00000000000040F624008021C2F2BE
:10EE60000040406806F07CBE002101707047000041
:10EE700080B50120F3F79CFEBDE88040FCF7C4BFDD
:10EE8000F0B581B0002853D040F624070446C2F202
:10EE90000047387820B1FD2670B201B0F0BD00BF48
:10EEA00015460E4606F054FF0028786040D04FF615
:10EEB00031120120C0F600020321C6F8C15101251C
:10EEC000F3F7D2FE4EF659620120C0F60002072188
:10EED000F3F7CAFE4EF671620120C0F60002082167
:10EEE000F3F7C2FE4EF629600121C0F600000022B1
:10EEF0000023002606F09CFFC4F8D0034EF64160C4
:10EF0000C0F6000001210022002306F091FFC4F8A2
:10EF1000D403D4F8D003142106F0D6FFD4F8D403D8
:10EF200041F2883106F0D0FF3D7070B201B0F0BD03
:10EF3000FE2670B201B0F0BD0246097800201170C3
:10EF40007047000000000000B1F831C08B8F02460E
:10EF500000EE10CAB8EE400A80ED020A00EE103A48
:10EF6000B8EE400A80ED030A886B506009780020F3
:10EF70001170704700000000B1F831C08B8F02465D
:10EF8000097800EE10CA1170B8EE400A80ED010A4F
:10EF900000EE103AB8EE400A80ED020A00207047F9
:10EFA000B1F840300246A0F80D30D1F834C08B6B78
:10EFB000C86BC2F80900C2F80530C2F801C091F868
:10EFC0003300D076D1F827C0D1F82B30D1F82F00FC
:10EFD000C2F81700C2F81330C2F80FC0D1F85900B8
:10EFE000CB6DD061C2F81F300020097811707047D6
:10EFF000F0B581B0044601200D46F3F7D9FDD0F8F5
:10F000008800202812D194F8AB0128B994F8AA11ED
:10F0100011B994F8AC1149B194F8AC1151B1072968
:10F020003ED9FF2568B201B0F0BD00BF002568B22F
:10F0300001B0F0BD94F8AA110729F2D8DFE811F069
:10F040009200D80008010800080008006A006A0061
:10F0500040F6E536A520C2F200460421FF223070BA
:10F060005120A6F801003046F4F712FD95F827204C
:10F07000307140F20130A6F80500F01D40F2031196
:10F0800000F05EFC06F10D004B222146F1F7E0FA9C
:10F090004B212046F1F75BFB5A25582603E100BFC0
:10F0A00040F6E536A520C2F200460421FF2230706A
:10F0B0000820A6F801003046F4F7EAFC95F827206E
:10F0C000307140F20130A6F80500F01D4FF4807158
:10F0D00000F036FC94F8AC0100254FF6FF720138C1
:10F0E00084F8AC01C1B204EB4101B1F8A401A6F867
:10F0F0000D003046A1F8A4510F21F4F7F5FBA6F856
:10F100000F000120112201233146F3F7C9FD68B237
:10F1100001B0F0BD40F6E536A520C2F2004604215C
:10F12000FF2230706F20A6F801003046F4F7B0FCE3
:10F1300095F82720307140F20130A6F80500F01D47
:10F140004FF4827100F0FCFB06F10D0069222146AC
:10F15000F1F77EFA69212046F1F7F9FA782576264B
:10F16000A1E000BF002800F0B08007283FF659AFAB
:10F1700040F6E536A520C2F200460421FF22307099
:10F180003320A6F801003046F4F782FC95F82720DA
:10F19000307140F20130A6F80500F01D4FF488717F
:10F1A00000F0CEFB94F8AB012D22013884F8AB01BE
:10F1B000C1B206F10D0011FB02412D2201F16904DB
:10F1C0002146F1F745FA2D212046F1F7C0FA3A2100
:10F1D0004FF6FF723046F4F787FB708701203C2220
:10F1E00001233146F3F75CFD002568B201B0F0BDA4
:10F1F00040F6E536A520C2F200460421FF22307019
:10F200001520A6F801003046F4F742FC95F82720B7
:10F21000307140F20130A6F80500F01D40F20111F6
:10F2200000F08EFB20681E256168A268D4F80B30C0
:10F23000B361C6F81520C6F81110C6F80D000020FD
:10F24000C4F80B001C26A060606020602BE000BFAB
:10F2500040F6E536A520C2F200460421FF223070B8
:10F260002420A6F801003046F4F712FC95F8272078
:10F27000307140F20130A6F80500F01D4FF48171A5
:10F2800000F05EFB06F10D001E222146F1F7E0F9C9
:10F290000020206060602D25A0602B26E0602061AA
:10F2A0006061A061A08340F6E5374FF6FF72C2F2BD
:10F2B000004731463846F4F717FBB85301200123C5
:10F2C00039462A46F3F7ECFC20B1FE2568B201B0BE
:10F2D000F0BD00BF002584F8AA5168B201B0F0BDAE
:10F2E0002DE9F04FA3B0044610250120C4F2020519
:10F2F00020700120F3F75CFCD0F880000068A84281
:10F3000000F097800120F3F753FCD0F8800005F15E
:10F3100018010068884200F08C800120F3F748FC57
:10F32000D0F8800005F130010068884200F081804B
:10F330000120F3F73DFCD0F8800005F1480100689A
:10F34000884276D00120F3F733FCD0F8800005F135
:10F350006001006888426CD00120F3F729FCD0F8E6
:10F36000800005F178010068884262D00120F3F73F
:10F370001FFCD0F8800005F190010068884258D049
:10F380000120F3F715FCD0F8800005F1A801006812
:10F3900088424ED00120F3F70BFCD0F8800005F531
:10F3A00080610068884244D00120F3F701FCD0F866
:10F3B000800005F58361006888423AD00120F3F7A8
:10F3C000F7FBD0F8800005F586610068884230D0F0
:10F3D0000120F3F7EDFBD0F8800005F589610068A6
:10F3E000884226D00120F3F7E3FBD0F8800005F532
:10F3F0008C61006888421CD00120F3F7D9FBD0F85B
:10F40000800005F58F610068884212D00120F3F773
:10F41000CFFBD0F8800005F592610068884208D0E3
:10F420000120F3F7C5FBD0F8800005F59561006871
:10F4300088420120F3F7BCFBD0F88000006804305C
:10F440000068D0F1FF00229000F0868142F2A067B0
:10F450004FF00008C2F200474FF0000904F5697050
:10F46000059004F56070049004F55E70039004F25A
:10F470006E30029004F26230019004F546701C90E8
:10F4800004F2FA201B9004F2BA201A9004F51470CA
:10F49000199004F24230189004F50E70179004F29F
:10F4A0003630169004F50B70159004F537701490F3
:10F4B00004F1A900139004F1A800129004F1A20035
:10F4C000119004F1A000109004F178000F9004F165
:10F4D00070000E9004F168000D9004F160000C9033
:10F4E00004F159000B9004F158000A9004F14E0009
:10F4F000099004F14200089004F13400079004F1EF
:10F500002700069004F2BE30219004F121002090E3
:10F5100004F10D001F9004F10C001E90601C1D9062
:10F5200017F80800A52840F0178109F10500229975
:10F53000C5B2A5EB0800884280F0028107EB080401
:10F5400005212046F4F7ECFA002800F0F980207835
:10F55000A52840F0F58009F10700229B5FFA80FBA7
:10F56000ABEB0801994280F0EB803A467A5BFF21D1
:10F57000B2F5007F0EDC022A2ADD032A3ED0B2F566
:10F58000827F3FD040F205139A4240F0D48001259B
:10F59000219EAFE0A2F201230D2B21D9A2F201336B
:10F5A0000F2B37D8DFE813F01000440048004C0060
:10F5B0005000540058005C006000C700C700C7003E
:10F5C000C700C700C70040007625139E92E000BF29
:10F5D000012A1BD0022A40F0AE8001251E9E89E040
:10F5E000DFE803F008464A4EA952565A5E62666A40
:10F5F0006E7200BF0D25069E7CE000BF10251F9E89
:10F6000078E000BF0325209E74E000BF0B251D9EFF
:10F6100070E000BFA2F60122052A00F28C80DFE82C
:10F6200002F003575B5F63671E251C9E62E000BF0C
:10F630001E25149E5EE000BF0C25159E5AE000BFFB
:10F640000C25169E56E000BF1825179E52E000BFFD
:10F650000825189E4EE000BF6A25199E4AE000BFAB
:10F6600022251A9E46E000BF1E251B9E42E000BFD9
:10F670000E25079E3EE000BF0C25089E3AE000BF25
:10F680000A25099E36E000BF01250A9E32E000BF30
:10F6900007250B9E2EE000BF08250C9E2AE000BF28
:10F6A00008250D9E26E000BF06250E9E22E000BF25
:10F6B00028250F9E1EE000BF0225109E1AE000BF05
:10F6C0000625119E16E000BF0125129E12E000BF24
:10F6D0000C25019E0EE000BF0A25029E0AE000BF35
:10F6E0000825039E06E000BF2425049E02E000BF1B
:10F6F0000625059E2844229AC0B2A0EB080191423B
:10F700001ED200F1020905F109015FFA89FAAAEB9C
:10F710000800884214D12046F4F74EF980B107EB77
:10F720000B0130462A46F0F793FF2298D0468245D7
:10F73000FFF4F6AE002148B223B0BDE8F08F00BF61
:10F7400041F22C20C2F20040016801310160FF212A
:10F7500048B223B0BDE8F08F002148B223B0BDE825
:10F76000F08F000000000000F0B587B002290446C9
:10F7700072D0012976D0002940F0B48094F8AB1102
:10F7800000260020062906D82D2011FB004001315B
:10F7900084F8AB116930642161A2CDE90211C8215E
:10F7A0000491CDE9051260A10122012300960127F1
:10F7B000019705F05DFD94F8AA01062805D8411CC3
:10F7C000C0EB0010261884F8AA114FF470704FF4A3
:10F7D0000771CDE903104AF62B310290C0F6010102
:10F7E00001220123F020059030460025CDE9005785
:10F7F00005F0D2FD94F8AA110020062905D8481C6E
:10F80000C1EB011184F8AA0160184FF4FA710122CA
:10F8100001924FF46172CDE902214AF629310122A9
:10F82000C0F60101012300950A27049705F06CFD3D
:10F8300094F8AC01022806D8411C04EB400000F506
:10F84000D27584F8AC1101210122284605F0B4FCE0
:10F850000025284607B0F0BD94F8AC01022845D930
:10F8600000204AE094F8AB1100250020062906D8B4
:10F870002D2011FB0040013184F8AB116930D4F820
:10F88000C1110A239FED221BB6EE003B0A8849886E
:10F89000019300EE102A322302EE101A0293012384
:10F8A0000095B8EE400B1CA7B8EE422B069720EE51
:10F8B000010B22EE031BBCEEC00BBCEEC11B10EE15
:10F8C000101A11EE102ACDE903314AF629310592BA
:10F8D000C0F601010122012305F0CAFC284607B049
:10F8E000F0BD00BFFF25284607B0F0BD411C04EB6A
:10F8F000400000F5D27084F8AC110121012205F01E
:10F900005BFCFF25284607B0F0BD00BF00BF00BF6D
:10F910009A9999999999E93F4155544F00000000EF
:10F9200044656D6F00000000300000000000000022
:10F9300040F624008021C2F20040406806F010B971
:10F94000092A018014D8013AFF21082A00F2818097
:10F95000DFE802F006222A323A424A7F4C0000BF1A
:10F960000121C0F20111C0F80210002148B2704715
:10F97000653AFF21082A00F26C80DFE802F00539C1
:10F9800041495159616A67006521C0F26511C0F8AB
:10F990000210002148B270470221C0F20211C0F8E3
:10F9A0000210002148B270470321C0F20311C0F8D1
:10F9B0000210002148B270470421C0F20411C0F8BF
:10F9C0000210002148B270470521C0F20511C0F8AD
:10F9D0000210002148B270470621C0F20611C0F89B
:10F9E0000210002148B2704707212AE0092128E0CF
:10F9F0006621C0F26611C0F80210002148B27047BB
:10FA00006721C0F26711C0F80210002148B27047A8
:10FA10006821C0F26811C0F80210002148B2704796
:10FA20006921C0F26911C0F80210002148B2704784
:10FA30006A21C0F26A11C0F80210002148B2704772
:10FA40006B214180002148B2704700BF6D21418089
:10FA5000002148B27047000080B542F2A061012049
:10FA6000C2F20041FF220023F3F7D6F8002818BFA6
:10FA70004FF0FF3080BD00002DE9F04381B02DED47
:10FA8000088B88B0044606F053F8C00540F19A830D
:10FA90004FF4807006F01CF840F65D40C2F2004062
:10FAA0000178042928D804F2AD16DFE801F0033DFF
:10FAB0000D151D0094F8AC1101220270022940F2CC
:10FAC0007181002075E100BF94F8AC11032202702F
:10FAD000022933D9002038E094F8AC1104220270D6
:10FAE00002294BD9002050E094F8AC110522027095
:10FAF000022965D900206AE094F8AC1102294FF080
:10FB00000001017008D894F8AB01072804D894F8D4
:10FB1000AA010828C0F056830120F3F749F82021F4
:10FB2000C0F888104EE300BF94F8AC1102220270B6
:10FB3000022940F24B8100204FE100BF481C04EB3A
:10FB4000410184F8AC0101F5D2700121042205F0D5
:10FB500033FB94F9BF0102284AD80FF6282101EBA4
:10FB6000800090ED000A94F8AA01062846D8411CAE
:10FB7000C0EB0010204484F8AA1140E0481C04EBBC
:10FB8000410184F8AC0101F5D2700121052205F094
:10FB900013FB94F9BE014AF2F835C0F601050228BC
:10FBA0006CD805EB800090ED008A94F8AA01062835
:10FBB0006AD8411CC0EB0010204484F8AA1164E00C
:10FBC000481C04EB410184F8AC0101F5D27001211D
:10FBD000062205F0F1FA94F8C01194F8AA01002960
:10FBE00000F0BA81062840F23582002038E200BFDA
:10FBF0009FEDDC0A94F8AA010628B8D90020D4F8B1
:10FC0000C1119FEDD92A9FEDD93ABAEE0C5A0A8854
:10FC10009FEDD74A4988022601EE102A0096012658
:10FC2000B8EE411A21EE021A02EE101AB8EE422A7C
:10FC300031EE033A31EE041A20EE020AB1EE002A48
:10FC4000BCEEC33ABCEEC11A30EE022A30EE050A11
:10FC500013EE101A11EE103ABCEEC22ABCEEC00A26
:10FC6000CDE9016112EE102A0FF6241110EE107A80
:10FC7000CDE9032301220423A1E200BF9FEDB98A4D
:10FC800094F8AA01062894D90020D4F8C1119FED58
:10FC9000B6AAB1EE009ABAEE0CBA0A889FEDD92A3C
:10FCA00049889FEDD93A00EE102A022601EE101A7B
:10FCB00000960126B8EE400AB8EE411A20EE0A0A74
:10FCC00028EE011A30EE022A30EE030A31EE093A2C
:10FCD00031EE0B1ABCEEC22ABCEEC33ABCEEC00A2F
:10FCE000BCEEC11A12EE101A13EE102A10EE103AE2
:10FCF00011EE107ACDE90161CDE903230FF67C0105
:10FD000001220523059705F093FB94F9BD01022814
:10FD10009CBF05EB800090ED008A94F8AA010628AC
:10FD200002D9002006E000BF411CC0EB00102044B7
:10FD300084F8AA11D4F8C1119FEDB42A9FEDB43A0A
:10FD400002260A884988009600EE102A012601EE54
:10FD5000101AB8EE400AB8EE411A20EE0A0A28EE50
:10FD6000011A30EE022A30EE030A31EE093A31EE82
:10FD70000B1ABCEEC22ABCEEC33ABCEEC00ABCEE03
:10FD8000C11A12EE101A13EE102A10EE103A11EEEC
:10FD9000107ACDE90161CDE903230FF2E47101226C
:10FDA00005230CE2481C04EB410184F8AC0101F589
:10FDB000D270012102224FF0020805F0FDF994F8FB
:10FDC000AA01062854D94FF0000958E0481C04EB5A
:10FDD000410184F8AC0101F5D2700121032205F044
:10FDE000EBF994F8B101012800F0C480002840F03C
:10FDF000E98194F8AA2100210020062A05D8501C88
:10FE0000C2EB021284F8AA01A018D4F8C12101277C
:10FE10009FED811B1388528800EE103A02EE102AE3
:10FE20009FED7F3BB8EE400BB8EE422BCDE9007161
:10FE300020EE010B4FF4B47122EE031B0291052159
:10FE40003227BCEEC00B0797BCEEC11B10EE102A88
:10FE500011EE103ACDE903124AF62D310122CDE917
:10FE60000537C0F60101032305F0B2F9AAE100BF8E
:10FE7000411CC0EB001004EB000984F8AA11D4F86F
:10FE8000C1019FED692B0188408800EE101A03EE36
:10FE9000100AF0689FED624BB8EE401BB8EE433B92
:10FEA000B8EE408A00EE100A21EE021B23EE042B6E
:10FEB000BCEEC11BBCEEC22B11EE105A12EE107A32
:10FEC00009F0B8FE9FED5A9AD4F8C10120EE090A54
:10FED0009FED581A408808EE010ABCEEC01A00EEE9
:10FEE000100AF068B8EE408A00EE100A11EE106AAF
:10FEF00009F014FD20EE090A9FED4F1A01AA0C210A
:10FF00000223CDF8008008EE010A0496A2C20FF287
:10FF100084610122BCEEC00A10EE100A059048462A
:10FF200005F03AFA94F9B501C1B2042900F24A8108
:10FF3000172222FA01F1C90700F044810FF258623A
:10FF400094F8AA1102EB8000062990ED000A40F215
:10FF5000F3800020F6E000BF062840F2A5800020D4
:10FF6000A8E000BF000000009A99593F00005842E5
:10FF70000000CC4294F8AA2100210020062A05D8CE
:10FF8000501CC2EB021284F8AA01A018D4F8C121B7
:10FF900037689FED211B138802EE107A52880226E3
:10FFA00000EE103A03EE102A9FED1D4BB8EE400B09
:10FFB000B8EE433BCDE9006120EE010B05219FED3A
:10FFC0001F1A322622EE011A079623EE042BBCEEEE
:10FFD000C00BBCEEC11ABCEEC22B10EE103A11EEF3
:10FFE000102A12EE107ACDE903134AF62D3102924F
:10FFF000C0F6010101220323CDE9057605F0E8F8FA
:020000040801F1
:10000000E0E000BF0000E4420000224300002E4375
:1000100000005E4300BF00BF333333333333E33F6D
:100020009A9999999999C93F9A9999999999D93F82
:1000300000003842CDCCCC3ECDCC4C3E0000B44389
:100040000000C0420000F042000060420000A042F8
:1000500000003042411CC0EB0010204484F8AA117B
:10006000D4F8C1111FED403A1FED112BBAEE0C4B25
:100070000A88498800EE102A01EE101AB8EE400AEC
:10008000B8EE411B20EE030A1FED133A21EE021BCE
:10009000B1EE002B30EE033A31EE022B31EE041BB1
:1000A0001FED184A28E000BF411CC0EB001020449F
:1000B00084F8AA11D4F8C1111FED553A1FED262B73
:1000C000BAEE0C4B0A88498800EE102A01EE101A8D
:1000D000B8EE400AB8EE411B20EE030A1FED263AA7
:1000E00021EE021BB1EE002B30EE033A31EE022B73
:1000F00031EE041B1FED2B4A30EE040A0226BCEE43
:10010000C33A0096BCEEC22B0126BCEEC00ABCEE80
:10011000C11B13EE101A12EE102A10EE103A11EE57
:10012000107ACDE901614AF64B31CDE90323C0F6DF
:1001300001010122062342E0481CC1EB011184F8B1
:10014000AA016018D4F8C1111FED792A1FED404AA9
:10015000BAEE0C5A0A8802264988009601EE102A47
:10016000012603EE101AB8EE411AB8EE433A21EE1A
:10017000021AB9EE082A20EE030AB1EE003A31EE77
:10018000022A31EE041A30EE033A30EE050ABCEED4
:10019000C22ABCEEC33ABCEEC11ABCEEC00A12EED3
:1001A000101A13EE102A11EE103A10EE107ACDE963
:1001B0000161CDE903230FF2F431012202230597F7
:1001C00005F036F905F0B4FC800540F1AD814FF43F
:1001D000007005F07DFC94F8AC01022802D90020E3
:1001E00007E000BF411C04EB400000F5D27084F82A
:1001F000AC1101210022002504F0DEFF94F8AB01D0
:10020000062807D82D2110FB0141013084F8AB01ED
:1002100001F16905D4F8C1019FEDD78A9FEDCC2B80
:10022000018801224088002300EE101A022701EE07
:10023000100A00974FF00A09CDF80490B8EE400A72
:100240004FF05008B8EE411BD9A6CDE9028720EE49
:10025000080A069621EE021B0026BCEEC00ABCEE80
:10026000C11B10EE100A11EE101ACDE904014AF676
:1002700029312846C0F6010104F0FAFF94F8AB01D9
:10028000062807D82D2110FB0141013084F8AB016D
:1002900001F16906D4F8C10101229FEDAF2B01885D
:1002A00000234088002500EE101A01EE100ACDE967
:1002B0000079B8EE400AB8EE411BCDE9028720EE86
:1002C000080AC1A721EE021B0697BCEEC00ABCEECD
:1002D000C11B10EE100A11EE101ACDE904014AF606
:1002E0002B313046C0F6010104F0C2FF94F8AB0197
:1002F000062807D82D2110FB0141013084F8AB01FD
:1003000001F16905D4F8C10101229FED952B018807
:1003100000234088022700EE101A009701EE100A11
:100320004FF00A09CDF804904FF05008B8EE400A9B
:10033000ABA6B8EE411B0696CDE9028720EE080A6F
:10034000002621EE021BBCEEC00ABCEEC11B10EE63
:10035000100A11EE101ACDE90401A7A1284604F0F5
:1003600087FF94F8AB01062807D82D2110FB014127
:10037000013084F8AB0101F16906D4F8C101012212
:100380009FED792B018800234088002500EE101A8C
:1003900001EE100ACDE90079B8EE400AB8EE411B33
:1003A000CDE9028720EE080A94A721EE021B0697EA
:1003B000BCEEC00ABCEEC11B10EE100A11EE101A02
:1003C000CDE9040193A1304604F052FF94F8AA014C
:1003D000062805D8411CC0EB0010251884F8AA1186
:1003E000D4F8C10103229FED589B01880023408867
:1003F000022700EE101A009701EE100A9FED4EAB97
:10040000B8EE400BB8EE411B9FED592B20EE0A0BC6
:1004100021EE091BBCEEC00B31EE022BBCEEC11B62
:1004200010EE100ABCEEC22B11EE101ACDE901201D
:1004300012EE106A0122CDE9031077A12846059635
:10044000002604F0A9FF94F8AB01062807D82D2157
:1004500010FB0141013084F8AB0101F16906D4F8C9
:10046000C1010A2200234FF050080188002540886E
:10047000019200EE101A012201EE100A0097CDE958
:100480000287B8EE400A65A7B8EE411B069720EE3A
:10049000080A21EE0A1BBCEEC00ABCEEC11B10EE1E
:1004A000100A11EE101ACDE9040160A1304604F0E3
:1004B000DFFE94F8AB01062807D82D2110FB01417F
:1004C000013084F8AB0101F16905BBEE0A2BD4F8C9
:1004D000C101B2EE044B0222018800234088009241
:1004E00000EE101A142203EE100A9FED151BB8EE51
:1004F000400BB8EE433BCDE9012800EE012B04226E
:1005000003EE094BBCEEC20BBCEEC41B10EE100A8E
:1005100011EE101ACDE90320059146A1012244A055
:100520000690284604F0A4FE002008B0BDEC088B1D
:1005300001B0BDE8F08300BF9A9999999999D93F84
:10054000333333333333E33F9A9999999999C93FB8
:10055000666666666666E63FC3F5285C8FC2E53F61
:100560001F85EB51B81EE53F7B14AE47E17AE43FAF
:1005700000000000000049409A99593F62000000C5
:10058000660000007B142E3F0AD7233FC3F5283FA7
:1005900061000000360000007B142E3F7B142E3FCC
:1005A000C3F5283F7B142E3F0AD7233F38000000B5
:1005B000434841532020474D424C202053484F543C
:1005C0002020464952450000464C4C5720205245B9
:1005D0004C58202052454C582020534E474C000088
:1005E000464C333520204142534C20205341464550
:1005F000202042525354000033000000524F545206
:100600002020524C545620204C4F41442020434F30
:100610004E54000034000000350000004354524C9A
:1006200020205243202050430000000064000000BE
:10063000434150006500000041F60020C2F2004036
:10064000F9F71EBB00000000016840F26F32D1F8DC
:1006500014C08B6943F008038B618B6943F010036E
:100660008B610B6823F001030B600B6923EA020224
:100670000A618A6822F440428A6090F881305FEA19
:100680008C620BD5042B09D0D0F8842042F0800274
:10069000C0F884208A6942F020028A6190F8813093
:1006A0005FEA4C620BD5032B09D0D0F8842042F0CE
:1006B0000402C0F884208A6942F040028A615FEA3D
:1006C0008C5209D45FEACC5213D40021A0F86210F6
:1006D000A0F86A10704700BFD0F8842042F00102F1
:1006E000C0F884208A6942F400728A615FEACC52C1
:1006F000EBD5D0F8842042F00802C0F884208A6943
:1007000042F480728A610021A0F86210A0F86A1099
:100710007047000000000000806B0021A0F86A1004
:10072000A0F86210012180F88110F9F789BA000061
:1007300010B5846BF5F7ECFA022808BF10BD20460F
:10074000FFF782FFD4F8840040F01000C4F8840062
:10075000012084F881002046BDE81040F9F770BA06
:10076000806BFAF765B80000806BFAF71DBB0000DC
:10077000806B90F88110072908BF7047C16FC96965
:10078000B1F5807F02D1FAF733B800BF0068016984
:1007900041F0080101617047806B90F881100729D2
:1007A00008BF7047816FC969B1F5807F02D1FAF740
:1007B000DBBA00BF0068016941F0080101617047C0
:1007C000074B19680868B0E8F04F80F30988BFF359
:1007D0006F8F4FF0000080F31188704700BF00BF9B
:1007E0009C0600240000000090ED000A91ED001A24
:1007F00030EE011AB7EE002AB4EE421AF1EE10FA0A
:10080000D8BF704782EE011A20EE010A80ED000A7F
:1008100091ED000A21EE000A81ED000A7047000008
:10082000B0B52DED088B044600284FF0FF0028D00E
:100830000D4631B3B4F8640110B3A069416929B31E
:1008400090F82C1041B394F8E01079B394ED391A74
:1008500094ED472A94ED3B0A31EE421AB5EE400A78
:1008600084ED3E1AF1EE10FA2EDD94ED3A2A82EE76
:10087000000A94F8E01084ED3F0A61BB46E000BF37
:10088000FF2040B2BDEC088BB0BD00BFFF2040B2DE
:10089000BDEC088BB0BD00BF0021C4F8F810816921
:1008A000C4F8FC1090ED069A3BE000BF90ED060AFC
:1008B0009FED511A0021C4F8F81094F8E01084ED6F
:1008C0003F0A41B922E000BF9FED4B0A94F8E010C7
:1008D00084ED3F0AD1B194ED392AB5EE402AF1EE0C
:1008E00010FA13DD94ED3A2AB5EE402AF1EE10FA33
:1008F0000CDD90ED0D3A90ED0C2AB4EE431AF1EEBA
:1009000010FA5DDDB0EE420A02E000BF90ED060A8B
:10091000B4F82211C08D9FED389A814288BFB0EEA5
:10092000409A9FED368AD4ED5A0AB0EE481A94EDFB
:10093000790A94ED00AA94ED58BAF3F771FCB5EE7C
:10094000409AF1EE10FA0ADDB7EE001A3AEE4B2AA1
:1009500081EE093AB4EE432AF1EE10FA04DA0020EF
:1009600040B2BDEC088BB0BDB0EEC00A0020B4EEC2
:10097000410AF1EE10FA3FF784AFA97800293FF45D
:1009800080AFA069F0EE480A2168C4F8601190EDCC
:10099000050A04F5F270B8EE400A88EE000AF3F793
:1009A0001FFCB4F86401B4F866110138A4F86401BE
:1009B000481CA4F86601002040B2BDEC088BB0BD15
:1009C00090ED0E4AB4EE441AF1EE10FA0ADD31EE63
:1009D000441A33EE443A32EE402A81EE031A01EE15
:1009E000020A95E790ED0F2AB4EE421AF1EE10FAE2
:1009F0008EDC9FED010A8BE700000000DB0FC94091
:100A0000B0B52DED028B044600284FF0FF0000F03A
:100A10003F820D46002900F03B82F2F7A1F809F071
:100A20000AFC00EE100A9FED528A80EE080A84ED5F
:100A3000000AF2F795F8D4E90223801A994109F0E7
:100A4000FAFB00EE100A80EE080A84ED040AF2F7C1
:100A500087F8A269C4E9020113782BB1012B07D1F1
:100A60009FED440A02E000BF9FED430A84ED780A3F
:100A700092F82C0020B394F8E00008B394F8000139
:100A8000032800F2A981DFE800F003213B4B00BFFF
:100A900094F8D0000138012800F2A1819FED370AB7
:100AA0001079B0EE401A002800F01781411E00F0C6
:100AB000030C032980F0D0809FED301A0022EFE074
:100AC000002084F8000184F81401DCE194F8D0E0FF
:100AD000AEF10100012800F27C819FED280A117916
:100AE000B0EE401A002900F05681481E01F0030CB8
:100AF000032880F00F819FEDE91A00232EE100BF4B
:100B00009FEDE60A1079B0EE401A00287AD0411E17
:100B100000F0030C032933D29FEDE01A002254E0C9
:100B2000012B07D063B9B2EE040A94ED461A31EEF8
:100B3000000A0BE094ED460A9FEDD71A04E000BFCF
:100B400094ED3B0A94ED461A30EE010A94ED391A01
:100B500084ED460AB4EE410AF1EE10FAC8BF84ED06
:100B6000461AB4F820010130A4F8200162E000BF69
:100B70000024744900007A4500409C4500000000B4
:100B8000A4F11003A0EB0C019FEDC41A002200BFDA
:100B900093ED4D2A93ED4E3AB0EEC22A04329142C3
:100BA00031EE021AB0EEC32A93ED4F3A31EE021A3B
:100BB000B0EEC32A93ED503A03F1100331EE021A5E
:100BC000B0EEC32A31EE021AE2D1BCF1000F19D007
:100BD00004EB8201BCF1010F91ED492AB0EEC22A6B
:100BE00031EE021A0ED091ED4A2ABCF1020FB0EE9E
:100BF000C22A31EE021A05D091ED4B2AB0EEC22A7C
:100C000031EE021A02EE100A0028B8EEC22A81EE76
:100C1000021A9FEDA12A00FE010A94ED781A84EDD4
:100C2000420A31EE401A84ED441AB4EE421AF1EE53
:100C300010FA01DA0120D0E094ED000A94ED411A97
:100C400030EE410A9FED961AB4EE410AF1EE10FA29
:100C5000C0F2C5800320C0E0A4F11003A0EB0C019A
:100C60009FED8E1A002293ED4D2A93ED4E3AB0EE91
:100C7000C22A0432914231EE021AB0EEC32A93ED39
:100C80004F3A31EE021AB0EEC32A93ED503A03F117
:100C9000100331EE021AB0EEC32A31EE021AE2D18D
:100CA000BCF1000F19D004EB8201BCF1010F91EDF2
:100CB000492AB0EEC22A31EE021A0ED091ED4A2A2C
:100CC000BCF1020FB0EEC22A31EE021A05D091ED4E
:100CD0004B2AB0EEC22A31EE021A02EE100A0028A8
:100CE000B8EEC22A81EE021A9FED6E2A00FE010ABA
:100CF00094ED781A21EE021A84ED420AB4EE410A0C
:100D0000F1EE10FA6BDB012084F8000184ED430A58
:100D100065E000BFA4F11002A1EB0C009FED5F1A8B
:100D2000002392ED4D2A92ED4E3AB0EEC22A0433E2
:100D3000984231EE021AB0EEC32A92ED4F3A31EEEC
:100D4000021AB0EEC32A92ED503A02F1100231EECF
:100D5000021AB0EEC32A31EE021AE2D1BCF1000F42
:100D600019D004EB8300BCF1010F90ED492AB0EEDD
:100D7000C22A31EE021A0ED090ED4A2ABCF1020FBF
:100D8000B0EEC22A31EE021A05D090ED4B2AB0EE39
:100D9000C22A31EE021A02EE101A0029B8EEC22A57
:100DA00081EE021A9FED3C2A00FE010A94ED781AAA
:100DB00084ED420A31EE401A84ED441AB4EE421A30
:100DC000F1EE10FA05DD022084F800012068C4F875
:100DD0000401BEF1000F02D1002084F8000194ED5F
:100DE000460AB5EE400AF1EE10FA16DD94ED3A1A15
:100DF000B5EE401AF1EE10FA0FDD94ED042A01EE83
:100E0000420A84ED460AB5EE400AF1EE10FA04DA21
:100E10009FED220A0020C4F8180194ED391AB5EEAE
:100E2000401AF1EE10FA13DD94ED3C2AB5EE402A9B
:100E3000F1EE10FA0CDB94ED3D0AB4EE402AB0EE70
:100E4000420AF1EE10FA1CBF84ED462A84ED3D2AD9
:100E500094ED3B2A84ED470AB5EE402AF1EE10FAF4
:100E60000EDD31EE400AB5EE400AF1EE10FA07DD74
:100E700080EE020ABCEEC00A10EE100A01E000BFCC
:100E80000020A4F822012046294600F0C9F80020DD
:100E900040B2BDEC028BB0BD0000C84200000000B3
:100EA0006F12033A3333733FB0F8660108800020B5
:100EB000C4F24010486070472DE9F04F81B02DED2D
:100EC000028BFF2400281CBF8846002906D160B28F
:100ED000BDEC028B01B0BDE8F08F00BFB0EE408AE0
:100EE000B5EE400AF1EE10FAF1DD98F804408346C1
:100EF000C0F81880F0F770FDBCB308F1840908F160
:100F0000A40A08F140050BF5F6760BF2345700BF42
:100F10002846FCF735FDB0EE480A012130464A4626
:100F2000FDF7B2FDB0EE480A06F5B4700121524655
:100F3000FDF7AAFDDBF81800B0EE480AD0ED510A23
:100F40003846FCF719F8DBF81810B0EE480A07F13C
:100F5000C000D1ED520AFCF70FF8013C05F10A057B
:100F600006F13C0607F12007D2D108F17C00FCF71E
:100F700007FDDBF8180090F8800078B1012845D112
:100F8000B0EE480A0BF2BC4008F582720121FDF771
:100F90007BFD0BF59F6008F592720CE0B0EE480AFD
:100FA0000BF2BC4008F1C4020121FDF76DFD0BF509
:100FB0009F6008F1E402B0EE480A0121FDF764FDEC
:100FC000DBF81810B0EE480A0BF2B460D1ED530A0A
:100FD000FBF7D2FFDBF81810B0EE480A0BF2D46032
:100FE000D1ED540AFBF7C8FF0BF1E00044210024C7
:100FF000CBF87041CBE95844CBE95A44EFF7C9FB31
:1010000060B2BDEC028B01B0BDE8F08FFC2460B291
:10101000BDEC028B01B0BDE8F08F000000000000C5
:1010200070B518B3044680690D4690F8201009B3D6
:1010300094F8DC10032900F27480DFE801F0036506
:10104000274200BF94ED240A9FED4A1A80EE010A60
:1010500090ED091AB4EE410AF1EE10FA73DD0120A9
:1010600084F8DC002068C4F8D8006CE0FF2670B279
:1010700070BD00BF20462946002684F8DC6084F855
:10108000D46000F0C5F870B270BD00BFD4F868112C
:10109000C4F8E41190ED050A9FED331AB8EE400A4A
:1010A0000020A4F8640104F5F270DFED300A81EE4F
:1010B000000AF3F795F8032084F8DC002068C4F8F0
:1010C000D8002046294600F0A3F894ED000A94EDDC
:1010D000361A30EE410A9FED261AB4EE410AF1EEBF
:1010E00010FA34DB94ED240A9FED221A80EE010AF7
:1010F000B3EE041A0026B4EE410AF1EE10FAC2DA99
:1011000070B284F8DC6070BD94ED240A9FED191A6A
:1011100080EE010A90ED091AB4EE410AF1EE10FAE0
:1011200004DA002670B284F8DC6070BD94ED000A29
:1011300094ED361A30EE410A90ED0A1AB4EE410AE7
:10114000F1EE10FA06DA2046294600F061F8002692
:1011500070B270BD012084F8D400022084F8DC0055
:10116000002670B270BD00BFDB0FC9C0DB0FC940E5
:101170009A99993E00007A44002843D0F0B581B096
:101180002DED028B044680690779EFB104F5F67501
:1011900004F234569FED1D8A2846FDF7C1FC05F583
:1011A000B470FDF7BDFCB0EE480A3046FBF73CFFDB
:1011B000B0EE480A06F1C000FBF736FF013F05F12B
:1011C0003C0506F12006E7D104F2BC40FDF7A8FC7F
:1011D00004F59F60FDF7A4FC9FED0C8A04F2B46057
:1011E000B0EE480AFBF720FFB0EE480A04F2D460E4
:1011F000FBF71AFF0020BDEC028B01B0BDE8F04008
:1012000040B27047FF2040B2704700BF00000000AE
:101210002DE9F04F81B02DED0C8B84B006460028EF
:101220004FF0FF0000F053838946002900F04F8300
:10123000B069317F40F62C0504790029C2F20045DF
:1012400000F0A88096F8D0100396002900F0C08026
:10125000022900F09D81012940F04082002CCDF848
:10126000049000F03D82B7EE00AA6FF0030101EB9D
:1012700084014FF0240A4827002440F2F4599FEDDE
:10128000D39A9FEDD3BA00259FEDD28A02919FEDAC
:10129000D2CA00BFC15DB0EE4B2A96ED781A013973
:1012A000CAB2017800EB820292ED020A29B1B0EED7
:1012B00048DA01291CD1B0EE4C2A284406EB0A0179
:1012C00022EE025A90ED023A91ED004A11EE034AE5
:1012D00024EE043AB0EEC44A83EE053AB4EE442A52
:1012E000F1EE10FA3AEE433A33FE08DA86ED57DAB9
:1012F00020EE010A06EB0508B0EE481A06EB040BD7
:101300000BF5F670D8ED4F0A80EE090AD6ED041AF7
:10131000FDF70AFBB06988ED5D0AB0EE481AD8ED1A
:101320004F0AC05D06EB80010BF5557008F5BA76E3
:1013300091ED540A0399D1ED041AFDF7F5FA2DEE5B
:10134000000A08F5C671304688ED630A039EFFF770
:101350004BFA98ED5D0A98ED631A30EE010A06EB40
:10136000090088ED690AFBF7D7FDB06988ED6F0ABF
:1013700038440838FCF798FB0298A84200F0B08186
:10138000B0690AF1100A04350A373C3409F1200922
:1013900080E700BF94B140302F46FCF77DFB012C65
:1013A0000AD064424A2500BFB0692844FCF774FBA8
:1013B00001340A35601CF7D1B0693D467C30FCF73A
:1013C0006BFB96ED5A0A86ED790A85ED010A6BE210
:1013D000CA46D4B304EB840000254FEA40084FF41A
:1013E000F6796FF0030B40F2F4579FED7A8A00BF55
:1013F000039800EB09063046FDF7AAFB0398B0EE10
:10140000480A00EB0B040398B0EE481AD4ED500ADA
:10141000D0ED041A3046039EFDF786FAF01984EDEC
:101420005E0A84ED6A0AFBF777FDB06984ED700A05
:1014300028444030FCF738FB0A3509F13C09A8453F
:101440000BF1040B07F12007D2D140F62C059FEDDC
:10145000618AC2F20045B0EE481A06F2BC48D6EDE9
:10146000041A95ED010AD6ED5A0A4046FDF75CFADA
:10147000B0EE481A06F59F67D6ED041A3846D6ED49
:101480005C0A86ED750AFDF74FFA06F2D46086ED28
:10149000760AFBF741FDB06986ED770A7C30FCF7F0
:1014A00003FB9AF80100D146002800F0FD81304688
:1014B000FFF762FEB06904796CB1039800F55576C8
:1014C000A6F5B470FDF744FB3046FDF741FB013C47
:1014D00006F13C06F4D14046FDF73AFB3846FDF7ED
:1014E00037FB039EB0690779002F4AD0791E07F0B9
:1014F000030003294FF000024FF000011AD306F554
:10150000E4733F1A002100BF043143F8042C43E97F
:10151000152243E9132243E90F2243E90D2243E94F
:10152000092243E9072243E903228F421A6003F1AB
:101530001003E9D128B306EB810300220128C3F888
:101540007421C3F88C21C3F8A421C3F8BC2118D09E
:101550004B1C022806EB8303C3F87421C3F88C21CB
:10156000C3F8A421C3F8BC210BD0881C002106EBD2
:101570008000C0F87411C0F88C11C0F8A411C0F834
:10158000BC110020C6F8DC01C6E97500012089E124
:1015900030464946CDF80490FFF742F9002C00F0A0
:1015A000ED80B7EE00AAA0004FF0240948244FF0C8
:1015B000000B40F2F4579FEDCF9A00259FEDCEBA75
:1015C00002909FEDCE8A9FEDCECA70E000C0DA4552
:1015D00000004842000000000000C843284406EB19
:1015E000090122EE025A90ED023A91ED004A11EE05
:1015F000034A24EE043AB0EEC44A83EE053AB4EE50
:10160000442AF1EE10FA3AEE433A33FE08DA86ED58
:1016100057DA20EE010A06EB0508B0EE481A06EB91
:101620000B0A0AF5F670D8ED4F0A80EE090AD6EDDE
:10163000041AFDF779F9B06988ED5D0AB0EE481A31
:10164000D8ED4F0A005D06EB80010AF5557008F5EC
:10165000BA7691ED540A0399D1ED041AFDF764F9B5
:101660002DEE000A08F5C671304688ED630A039E28
:10167000FFF7BAF898ED5D0A98ED631A30EE010AAB
:10168000F01988ED690AFBF747FCB06988ED6F0A2D
:1016900020440838FCF708FA0435029809F11009CB
:1016A0000A34A8420BF13C0B07F1200766D0B06961
:1016B000B0EE4B2A96ED781A015D0139CAB2017875
:1016C00000EB8202002992ED020A87D0B0EE48DAE0
:1016D00001299ED1B0EE4C2A80E700BF0020E1E056
:1016E00040F62C059FED858AC2F20045B0EE481AFF
:1016F00006F2BC40D6ED041A95ED010AD6ED5A0A61
:10170000FDF712F9B0EE481A06F59F60D6ED041AFF
:1017100086ED750AD6ED5C0AFDF706F906F2D4608F
:1017200086ED760AFBF7F8FBB06986ED770A7C3028
:10173000FCF7BAF9DDF8049099F8010000285BD0B5
:101740002878002840F0B08099F80200002800F0C6
:10175000AB80307F022186F8D010D6F868110328BC
:10176000C6F8E41100F0BA80022800F0BD8001281C
:101770003DD10120A6F8640196E000BF9FED5F8A8D
:1017800006F2BC40B0EE481AD6ED041AD6ED5A0A5D
:1017900096ED790AFDF7C8F8B0EE481A06F59F6095
:1017A000D6ED041A86ED750AD6ED5C0AFDF7BCF895
:1017B00006F2D46086ED760AFBF7AEFBB06986EDE3
:1017C000770A7C30FCF770F9DDF8049040F62C05C0
:1017D000C2F2004599F80200002865D1012086F880
:1017E000D00096ED5A0A85ED010A86ED790A0020AF
:1017F000A6F8640158E000BF3046FFF7BDFCB069B1
:101800000779002F49D0791E07F0030003294FF014
:1018100000024FF0000119D306F5E4733F1A0021CE
:10182000043143F8042C43E9152243E9132243E928
:101830000F2243E90D2243E9092243E9072243E944
:1018400003228F421A6003F11003E9D128B306EB9B
:10185000810300220128C3F87421C3F88C21C3F846
:10186000A421C3F8BC2118D04B1C022806EB83032B
:10187000C3F87421C3F88C21C3F8A421C3F8BC2198
:101880000BD0881C002106EB8000C0F87411C0F852
:101890008C11C0F8A411C0F8BC110020C6F8DC01FE
:1018A000C6E9750086F8D000B0694030FBF798FFB4
:1018B000B0694168052903D36830FBF791FFB0692F
:1018C0007C30FBF78DFF99F802002870002040B2B1
:1018D00004B0BDEC0C8B01B0BDE8F08F41F60A20DE
:1018E000A6F86401E0E700BFB069C069A6F864012A
:1018F000DAE700BF00C0DA450000484200000000FF
:101900000000C8430000000020B10177002040B271
:10191000704700BFFF2040B2704700000000000089
:10192000002800F0BB802DE9F0472DED068B8246A4
:10193000806990F80480B8F1000F4DD0B7EE008AAE
:10194000BFEE009A4FEA88094827002540F2345636
:1019500024249FED7BAA26E00AEB04010AEB060093
:1019600091ED000AFBF7D8FA80EE0A1ADAF81800AF
:101970000AEB05010435C25D0A3781FE481A81ED84
:10198000490AA94506F120060AEB820204F1100477
:1019900081FE090A81ED4F0A92ED541A31EE000AD8
:1019A00082ED540A18D038440838FCF709F9DAF8FF
:1019B000180038440838FBF79BFF0028CCD00AEB0E
:1019C000850100F12C0C01F1200E806B9CE80C10BD
:1019D0008EE80C10C862BFE700EE108A9AED561A26
:1019E0007C30B8EEC00A81EE000AB6EE001A20EE96
:1019F000010A8AED560AFCF7E3F8DAF818007C30A1
:101A0000FBF776FF01460AF180005022EEF765FEF3
:101A1000DAF818009AED321A90ED040A20EE010A65
:101A20008AED5A0AB5EE400AF1EE10FA3ADB9FED64
:101A3000451AB4EE410AF1EE10FA5ADA9AF8A80003
:101A400018B131EE400A8AED5A0A0AF2B4609AEDF2
:101A5000230AFBF761FA9AED231A9FED3C2A81EEE7
:101A6000021AB7EE002A8AED5B0A9AED090A9AED8E
:101A70000D3A0AF2F46081FE421ABFEE002A30EEFF
:101A8000430A80ED000A002081FE021A8AED5C1AEA
:101A9000BDEC068BBDE8F04740B27047FF2040B276
:101AA000704700BF9FED271A30EE010AB5EE400ADD
:101AB000F1EE10FABFBF30EE010AB5EE400AF1EECA
:101AC00010FA30EE010ABCBFB5EE400AF1EE10FA92
:101AD00006DA30EE010AB5EE400AF1EE10FAE3DB69
:101AE0008AED5A0A9FED171AB4EE410AF1EE10FA88
:101AF000A4DB9FED152A00BF30EE020AB4EE410AC6
:101B0000F1EE10FAA1BF30EE020AB4EE410AF1EE96
:101B100010FA30EE020AA4BFB4EE410AF1EE10FA58
:101B200006DB30EE020AB4EE410AF1EE10FAE3DA17
:101B30008AED5A0A9AF8A80000287FF482AF84E759
:101B400000C0DA45DB0FC940DB0FC9C000401C45AF
:101B500080B504F0FDF8BDE8804004F04DB9000008
:101B600010B540F60C04C2F20044207860B902209F
:101B70004FF440710322F0F72BF818B1FF2040B268
:101B800010BD00BF01202070002040B210BD000039
:101B900010B588B040F60C04C2F200442078012849
:101BA00007D101AA02204FF440710023EFF7B8FEDD
:101BB00020B1FF2040B208B010BD00BFF6F764FBB3
:101BC0006060BDF811009DF81410A0829DF813000C
:101BD000207448006082BDF81500E082002040B209
:101BE00008B010BD0000000080B54EF21000CEF22B
:101BF0000000006806F074FF012808BF80BDBDE842
